:020000040800F2
:100000000050002089B6000835B70008E9A10008B3
:1000100035B7000835B7000835B700080000000004
:1000200000000000000000000000000035B70008DC
:1000300035B700080000000035B70008D9A1000856
:1000400035B7000835B7000835B7000835B70008E0
:1000500035B7000835B7000835B7000835B70008D0
:1000600035B7000835B7000835B7000835B70008C0
:1000700035B7000835B7000871A0000835B700088B
:10008000A9A0000835B7000835B7000835B7000843
:1000900035B7000835B7000835B7000835B7000890
:1000A00035B7000835B7000835B70008BD9F000810
:1000B000B59F0008A99F00089D9F0008E5A00008C3
:1000C000DDA00008E1A00008D9A0000835B70008AD
:1000D00035B7000835A0000835B70008C99F0008EB
:1000E00035B7000835B7000835B700080000000034
:1000F0000000000000000000000000000000000000
:0C01000000000000000000005FF808F1A3
:100110002DE9F04F684B694C9FB02360002363606A
:1001200009F08CF918B907F025F809F0ABF903F0DC
:1001300073FD00230993624D0A930B934FF4E01370
:100140000C932B685F4A43F48033917B2B60AB693F
:10015000904643F01003AB612B6803F400330A931D
:10016000099B013309930A9B1BB9099BB3F5A06F47
:10017000F2D12A68524B12F4003201D0022315E06A
:10018000186840F00100186009922B6803F0020320
:100190000A93099B013309930A9B1BB9099BB3F589
:1001A000A06FF2D12B689B073BD501230B93464BE5
:1001B00046481A6842F010021A601A6822F00302D8
:1001C0001A601A6842F002021A606B686B606B6812
:1001D0006B606B6843F480636B603D4B1A68043B53
:1001E00022F070425A603B4A10606868914620F4E1
:1001F0007C106860586840F000405860D86820F46F
:100200000040D8609B6813F4004F17BF324B4FF487
:10021000E01313604FF480130C930B9B012B01D15F
:1002200017E0FEE7022B18D169B10C9BB3F5801FD4
:1002300002D14FF4A01305E00C9BB3F5E01F02D1EF
:100240004FF400130C936A680C9B134343F4803300
:1002500002E06B6843F460136B602B6843F08073BB
:100260002B602A68164B9701FBD55A6822F00302CF
:100270005A605A6842F002025A606A68104B02F0F3
:100280000C02082A0592F8D15A68144F02F00C02A9
:10029000042A03D0082A05D00C4B01E0D9F800301D
:1002A0003B6028E05A685968C2F38342CE0302F1EA
:1002B000020217D40A4B1CE0B92300086C06002088
:1002C000001002400C1700200020024000127A00AB
:1002D0000410014014000020001BB700780000202B
:1002E00000093D005B6813F4003FD9F8003018BFE7
:1002F0005B085A433A606B681EAEC3F303134B446A
:100300001A793B68DFF820B3D340B44A3B60B44B62
:10031000B448DA60AB69DFF814A343F00103AB61C2
:100320006B6A43F080736B62AB6943F01C03AB6193
:1003300000238DF84E304FF6FF7326F82C3D3146E2
:1003400002F014FD5846314602F010FDA648314631
:1003500002F00CFD9AE80300A44B0AF1080A5A685F
:1003600042F000725A60AB6986E8030043F008036C
:10037000AB610823CBF81030139814A902F0F6FCF7
:100380009AE80300AB6986E8030043F0040314A96C
:10039000AB61139802F0EAFC954AD9F800300020CE
:1003A00093420CBF934A944A944B4FF0070A1A6049
:1003B00001F0CDFE924B93E80300AB6986E80300A1
:1003C00043F00803AB6114A9139802F0CFFC304648
:1003D00009F01AFD139B8B4AF021B3FBF2F33A6844
:1003E000A3604FF47A73B2FBF3F2874B013A5A6081
:1003F0007B4A002782F823109F60C3F800A009F011
:1004000073FE07F077FB642001F097FE3946102257
:100410007E480DF06AF9734A012384F80FA0A37394
:1004200013683946934601228A4002F00100904247
:1004300005D18A000F2000FA02F223EA02030131FB
:100440000829F0D1CBF800306B69714F43F00103FC
:100450006B61AB69384643F40073AB6101F082FB1A
:100460006C4B002513936C4B4FF0010A14934FF41F
:10047000807319934FF480631A9320231B933146A2
:100480004FF4005338461C931595CDF858A0179596
:1004900018951D9501F048FB3B68604A43EA0A0342
:1004A0003B60536823F4702323F480735360916896
:1004B0005B4B0B4043F4602343F002039360D36A29
:1004C00023F47003D3625346504A511988780028A8
:1004D00051D0AA5C581C092ACF78C0B24F4910D914
:1004E000A2F10A0606EB46064FF0070E0EFA06FECC
:1004F000B740D1F80CC02CEA0E0E4EEA0706CE60CB
:100500000DE002EB42064FF0070E0EFA06FEB74072
:10051000D1F810C02CEA0E0E4EEA07060E61062B2B
:100520003E490CD8013B03EB83031F269E409A40B3
:100530004F6B27EA060646EA02034B631CE00C2BCE
:100540000CD8073B03EB83031F269E409A400F6B9A
:1005500027EA060646EA02030B630DE00D3B03EBB8
:1005600083031F269E409A40CF6A27EA060646EA82
:100570000203CB6200E018460435102D01D003467B
:10058000A2E7264B9A6842F480729A609A6842F019
:1005900001029A609A6842F008029A6099681F4ABC
:1005A0000D07FBD4936843F0040393601B4A9368E0
:1005B00013F00403FAD19168B8F8E60041F4A00101
:1005C0009160184AA8BBB2F9E8308BBBB2F9EA30A7
:1005D000D3F1010338BF00232BE000BF0005FA056B
:1005E00000ED00E000080140001001400000014063
:1005F000001BB700F117000805180008E01C0020D8
:10060000C4F2000840420F0010E000E0780600202D
:10061000080002404C2401408806002000240140CC
:10062000FDF7F1FF0C170020000C0140B4F20008A8
:10063000034613F0010340F08D8089F8143000B2B6
:1006400009F03AFFA4A3D3E9002309F09BFF0AF0C5
:10065000CBF9A34F0646B7F9E80009F02DFF9EA39A
:10066000D3E9002309F08EFF0AF0BEF90546B7F979
:10067000EA0009F021FF98A3D3E9002309F082FFE3
:100680000AF0B2F9814630460DF05EFA0746304670
:100690000DF0CEFA804628460DF056FA064628465A
:1006A0000DF0C6FA054648460DF04EFA8246484619
:1006B0000DF0BEFA3946814650460AF0F3FA394643
:1006C000039048460AF0EEFA5146049040460AF07C
:1006D000E9FA4946069040460AF0E4FA31460790A6
:1006E00050460AF0DFFA4946606206F100400AF01F
:1006F000D9FA2946A062E56206980AF0D3FA0146C3
:1007000004980AF0C7F92946206307980AF0CAFA44
:10071000014603980AF0BCF93146606308F10040D5
:100720000AF0C0FA2946A06303980AF0BBFA014612
:1007300007980AF0ADF92946E06304980AF0B2FA86
:10074000014606980AF0A6F93946206430460AF0B8
:10075000A9FA6064634E644A3368002143F00203DF
:10076000336013685E4DB3F85A30A4F84810049310
:100770005E4BB5F8EE80197094F84A1095F8ED705C
:10078000994609B908F090FFB8F1140F1CD009D8A8
:10079000B8F1050F1ED0B8F10A0F18D0B8F1000F4C
:1007A0000FD11AE0B8F1BC0F1AD0B8F5807F05D090
:1007B000B8F1620F05D14FF0020813E04FF00008C6
:1007C00010E04FF003080DE04FF004080AE04FF08E
:1007D000050807E04FF0060804E04FF0070801E0C5
:1007E0004FF00108424B4FF0100A1A881A2022F0ED
:1007F00040021204120C1A801A8822F038021204E5
:10080000120C42F030021A801A8892B242F0400272
:100810001A80CBF814A004F06BFC404604F068FC8E
:100820000120CBF810A001F07DFC13A808F0EEFC2D
:100830009DF94E30013303D19DF94C30013303D083
:10084000B4F848309BB22BB100230320A4F8483001
:1008500001F0C8FCDFF8B880264B6420C8F80030EF
:10086000254BC8F80430254BC8F80C3001F065FC66
:1008700001200423039089F80030DFF890B00022B3
:10088000062F8BF80020DFF88CA008D0082F01D0AD
:10089000DFB904E0336823F00203336015E000227F
:1008A000A4F8482094F84A200AB908F0FDFE144A3A
:1008B0001449642011601449516001F03EFC062285
:1008C0008AF8002004228BF800209AF800303BBB05
:1008D00017B31F46D1E700BF399D52A246DF913FB3
:1008E0000C17002068020020F801002012020020EE
:1008F00000300140E51A00080D92000890C1793DD2
:100900006C020020D51A0008999100087E02002090
:10091000FC010020DD1C0020336823F0020333605B
:1009200095F8E2300BB189F8003095F8E3300BB15F
:10093000BF490B7095F8E4300BB1BE4A13703368B1
:100940009C0702D5BC4B1B689847D8F800309847E5
:100950003368BA4C13F0080F1BD0049A4FF06409A7
:100960000FFA82FA9AFBF9F738460AF047F98346FC
:1009700009FB17A000B20AF041F9B1490AF092F957
:10098000014658460AF086F8AE490AF08BF9E06451
:1009900001E00023E364AC4B08221A614FF00A091E
:1009A000A94F1920FB6809F1FF3983F00803FB60A8
:1009B00001F0C3FB012001F0CAFB192001F0BDFBCF
:1009C000002001F0C4FB19F0FF09E9D108233B61C5
:1009D0009E4B9F4F1B6893F90C0009F06DFD90A38F
:1009E000D3E9002309F0CEFD09F0FEFF0DF0ACF8CD
:1009F000814638880AF002F949460AF053F90DF0A9
:100A0000D9F8944B188038880AF0F8F801469248D3
:100A10000AF0FCF991490AF0F9F92065D8F80C00C0
:100A200009F05CFD7EA3D3E9002309F0ABFD7EA3B2
:100A3000D3E9002309F0A6FD09F0D6FF884B894AC7
:100A4000186089496879894B107001EBC000407EBD
:100A50006365874B794F1860A868984610F0200F9F
:100A600018BF01234FF000014FF4A07207F15800A6
:100A700018BFC8F800300CF038FE7E4A536823F4E3
:100A8000406343F0706343F4006353607A4BDA6968
:100A900042F00702DA619A6942F4006242F00C0205
:100AA0009A61764BC4F8983108F0F0FF152207F5EB
:100AB000CE70FF210CF019FE002384F89C313368BE
:100AC0000122980784F8B12107D587F89D210322D8
:100AD00087F8B121022287F89E21590708D594F89A
:100AE000B121511C84F8B1112244032182F89C11D8
:100AF00013F00A0F14D094F8B1310421E21882F8EF
:100B00009C115A1CD2B22244052182F89C11DA1C95
:100B10000233DBB284F8B1212344062283F89C21FE
:100B2000AB689A0608D594F8B121511C84F8B1112C
:100B30002244072182F89C111F060ED594F8B1219A
:100B40000920A11881F89C01911C0132D2B284F8CD
:100B5000B11122440A2182F89C116A79082A01D035
:100B60000E2A08D194F8B121511C84F8B111224405
:100B70000B2182F89C1194F8B1210C27A618511C66
:100B8000C9B286F89C715E072C4884F8B11106D56D
:100B9000023280F8B1210144102281F89C2194F89E
:100BA000B1211227A61886F89C7195F84161511C55
:100BB000C9B2002E0CBF002303F001031F4884F8C4
:100BC000B11133B102320144132380F8B12181F80D
:100BD0009C3194F8B1312A485A1C84F8B12123443D
:100BE000142283F89C21002198220CF07EFD00261F
:100BF000D5F82C214FF0000A002700970120394634
:100C0000032306F0BDFD8146E0BBBAF1000F53D1CE
:100C10004FF496424FF0010AEEE700BFAFF30080B9
:100C2000399D52A246DF913F000000A0F7C6B03EBA
:100C30007E020020E41C00206C0200206C060020D4
:100C40008988883C00002041000C0140B802002047
:100C500000000020DC0200200AE81C4100401C4685
:100C6000B4020020DA030020B4F200081C170020B0
:100C7000FC04002000000140001002403418002055
:100C800020080020012EB3D84C2202FB06F3DFF827
:100C900064A306F1010B0AEB0306304639460293C2
:100CA0000CF023FD029B5FFA8BFB4AF803900123B3
:100CB00086F84A305E469BE7022001F020F90146A3
:100CC000C4F84C0248B9009103230220D5F8302122
:100CD00006F056FDB84BC3F84C020EA800211222B4
:100CE0000CF003FD6B790E2B01D0082B02D10123F0
:100CF0008DF84130AE6816F4005618D1AF4A002383
:100D0000B05CD75CD118874203D01033602BF8D188
:100D1000002108F043FB83681B78012B04D01036B8
:100D2000602EEBD10023039303988DF83B00D8F895
:100D30000010A3480031AB6818BF01218DF83F10A7
:100D40000168C3F340028DF83C2091F82611C3F3EB
:100D500080128DF83D20C3F34032C1F38001B5F815
:100D6000E0008DF83820C3F3C0328DF83A208DF8BA
:100D70004010C3F30042B5F8DE108DF83E20ADF808
:100D8000440003F001024FF47A70DB048DF839203F
:100D9000ADF84210ADF8460004D58A4BB3F8DA300E
:100DA000ADF84630B1F5FA7F864E84BF0023ADF82A
:100DB0004630B6F818318449ADF8483096F82031FD
:100DC00084F85032002384F851324B709DF8413042
:100DD000002B14BF0223002302B101337B490027FB
:100DE00001EB8303D3F83031BA460393039A4FF6ED
:100DF000FF71D35B8B42DAB20CD1754B94F8512260
:100E00001A70744B93F80080B8F1160F40F04A81C5
:100E100000253AE19DF83B1019B1911E012940F2DD
:100E200021819DF83D1019B1111F032940F21A814B
:100E3000DFF8C4919DF83E104FEA021809EB08054F
:100E400029B159F808106448814200F00B819DF8DF
:100E50003A1011B1012A00F005819DF83C1011B142
:100E6000042A00F0FF801B0A022B05D19DF83810E0
:100E7000002908BF002303E0012B08BF9DF839308B
:100E80009DF83F1039B19DF8411021B9A2F1080138
:100E9000012998BF04239DF8401031B19DF84110FD
:100EA00019B9043A032A40F2C480012B36D1424BCF
:100EB0004FF0000BFF2283F854B2C3F858B2C3F8C6
:100EC0005CB2C3F860B2C3F894B283F8982283F896
:100ED000992283F89AB283F89BB283F89CB2C3F844
:100EE000A852AB68EA7B6868ADF84C3013A90223BE
:100EF0008DF84F308DF84E2001F038FF297B5A468F
:100F000059F8080008F05DFE284604F027FB284643
:100F10005946324A324B04F03DF8A3E0022B30D15F
:100F2000DFF8D8E05FFA8AFB4FEA0B110EEB010005
:100F300000224FF0010C8270827280F801B00EF82E
:100F400001C0E97BC560A8688DF84E10ADF84C0073
:100F500013A968688DF84F30029201F007FF297BD2
:100F6000029A59F8080008F02CFE284604F0F6FA18
:100F7000284659461B4A1C4B04F00CF80AF1010A9A
:100F800070E0032B53D1BDF84230DFF82C80B3F56D
:100F9000FA7F98F8529233D9144A2846B2FBF3F2FA
:100FA0000821BDF8463092B203F02CFE08EB89030D
:100FB000C3F81C030E4B32E06C06002084F30008DB
:100FC000F80100200C170020BD080020B4F2000832
:100FD000B8040020DA030020000400408B19000848
:100FE000911A0008BD9D0008651A000800127A00D9
:100FF000B11A00082008002058080108080900203C
:10100000904A2846B2FBF3F20121BDF8463092B275
:1010100003F0F8FD08EB8903C3F81C038A4B8360D7
:101020008A4B93F85222013283F852221AE0042BA1
:1010300018D1BDF84430834ADFF8108292FBF3F2F6
:101040002846BDF84830012192B298F8519203F039
:10105000D9FD08EB8903C3F84C0398F851320133EA
:1010600088F851320237182F7FF4C0AEC5E6784FAA
:1010700099E80F002F4487E80F00764B10351A7857
:10108000C02D02F101021A7008D0636D0021585979
:1010900003EB050909F09AFF0028E8D0B368DF04E4
:1010A0001ED418E06C496B4A01EBC80393F818E0B2
:1010B000D3F81CC082F800E0BCF1000FEED0002590
:1010C0007545EBDA624F2B011F4463440FCB0135AA
:1010D00087E80F00F4E7B8F1080F604F26D128E049
:1010E0005C4B93F80090B9F1010FF4D95C4D0027E7
:1010F0004F4505F11005EEDA55F8100C4FF07C5114
:1011000009F0D0FD4FF07C5145F8100C55F8140C47
:1011100009F0C8FD4FF07C5145F8140C55F80C0C43
:1011200009F0C0FD013745F80C0CE1E7B8F10E0FEE
:1011300003D13B7843F0100302E03B7823F0100327
:101140003B7004F0C3F94749474B4848484AC4F844
:101150006C13C4F8703301600023B6F81811A4F8BA
:10116000763384F87833C4F87C23C4F8802391461E
:10117000404A99520233242BFAD13F4B334CC3F8E7
:101180000090B36813F0080F00F0A4803B4B0022DE
:1011900093F81631042B00F29780DFE803F0030385
:1011A0002A448100012B4FF0030208D184F88423E4
:1011B000072284F8863384F885230C2308E0022371
:1011C00084F88433002384F8863384F88523072346
:1011D00084F88733002300930820012328494FF423
:1011E000E13206F0CDFA274BC4F88C03C4F89033F3
:1011F00066E001230093244905230820234A06F0D2
:10120000BFFAB6F81811C4F89403A1F57771490034
:1012100000231F4A99500433302BFAD11D4BC4F8D8
:1012200090330C234AE00092012308201A494FF41E
:10123000E13206F0A5FA194BC4F89803C4F89033CC
:1012400010233BE040420F00A11A00086C0600206A
:10125000E0030020B01C0020B4F20008DE020020F1
:10126000E80300201A180020F4F30008F40000201E
:10127000DC090020BA040020E80100200C1700203F
:10128000BD1F000811170008C9200008A086010032
:1012900014010020C517000855200008B5170008E4
:1012A000009201230820BD494FF4E13206F068FAAC
:1012B000BB4BC4F89C03C4F89033082384F88733ED
:1012C000003018BF012028B9082001F0ABFB002333
:1012D000C4F89033B3685D0405D5082284F88723E9
:1012E000B04AC4F8902342F201021A4003F001010F
:1012F00003F400505AB1AC4AC4F8902318B1AB4A79
:10130000082082F8870311B10C2284F8872394F80F
:1013100087231806A2F1040284F8882346D5A34B3C
:10132000A34AD6F83411C3F8A0230023A14A02EB44
:101330000310D0F86C011546884204D00133DBB2AB
:10134000042BF3D9002384F8A5339B4B0020C4F869
:10135000C03304F0A3FA994B94F8A5231B6800212D
:10136000C4F8AC3396F8263105EB02128B42C4F870
:10137000A8134FF010000091D2F86C210CBF01238C
:10138000032306F0FDF9C4F8C40318B9802001F066
:1013900049FB02E0012004F081FA894B1868894B6F
:1013A00000F5947204301A6001F04AFCB368D90366
:1013B00040F1C880002140F22A3283480CF095F9B0
:1013C00082498B6943F008038B61814B1A680023C3
:1013D0000120984000F01005854208D198000F25A3
:1013E000854022EA05020B2505FA00F0024301338D
:1013F000082BEDD1764B774D1A60CB694FF0010A7F
:1014000043F00203CB61744B4FF000081A68734B32
:10141000DFF8F0B1B2FBF3F22B88013A23F45C73EE
:101420001B041B0C2B8092B21D23AB852A85A5F8CB
:1014300014A02B8C23F001031B041B0C2B842B8C7E
:10144000A8882A8B23F0020322F0730212041B04E3
:10145000120C1B0C42F0600280B243EA0A03A8801F
:101460002A83A5F834802B842B8B584623F008035D
:101470001B041B0C43F008032B83B5F844306FEAC0
:1014800043436FEA53439BB2A5F844304B6943EAA8
:101490000A034B6100F066FB514B40F22A32139372
:1014A0001692494B802218924FF48072149319922D
:1014B00010234FF40052584613A915931C9202931F
:1014C000CDF85C80CDF86880CDF86C80CDF8748064
:1014D00000F02AFBAA89029B92B242F40072AA8110
:1014E000DBF800200DA842F00202CBF800208DF8B6
:1014F000343002238DF835A08DF836308DF837A0C2
:1015000000F0A8FB374B1A68374B48F8032008F166
:101510000408B8F1800FF5D104F03DF804F03BF871
:10152000324A334B13608033C4F8F436314BC3F87E
:10153000009001F0BDFA01F0F9FA01F0D1FA2E4B5A
:1015400001221A70B3685A0540F19280042008F015
:1015500039F80146042007F021FF18B14368187AD2
:1015600000F00100B36884F8F80613F480690BD02A
:10157000042008F027F80146042007F00FFF10F1BF
:10158000000918BF4FF001091C4B83F800901C4B59
:101590001D682B78C3BBC4F8FC565FE00920000827
:1015A000A1170008D9170008E51700086C060020ED
:1015B00034180020B4F20008321800200817002068
:1015C000F8010020C8030020340A00200010024067
:1015D000000C0140000400407800002000366E013D
:1015E0003404004074F20008CC050020C805002037
:1015F0005018002050060020B805002000050020EB
:10160000040500206C000240012B27D1DFF8F88090
:10161000002140462C22C4F800570CF066F88E23B7
:1016200088F801304FF07C0BE0234FF07D0A88F8FA
:10163000033088F800B088F82BA0DFF8D0800021B4
:1016400040462C220CF051F88A2388F80130A02360
:1016500088F800B088F8033088F82BA02B78022B8C
:1016600008BFC4F80457B9F1000F01D006F0DCF848
:1016700000F08AFC1D4B18607379052B03D11C4BBD
:101680004FF4C8721A801B4B4FF47A721A803B7861
:1016900043F008033B70184B1A7822F002021A70CC
:1016A000B3689B071ED5154BC4F8083700F0C6FB7E
:1016B000282000F042FD059901390591F6D1104B23
:1016C00096F8051118780A460123904203D3013396
:1016D000082B0A44F9D10B4A137096F8062153439C
:1016E000A4F80C371FB0BDE8F08F00BF280300201E
:1016F00080020020D81C0020DC1C002010180020D4
:1017000014050020740000202C050020590500203D
:101710001E4B2DE9F0431A781D460AB31C4B07787F
:101720001E781C4B93F800C002231B4A03F10108EA
:10173000D45C344104F00F04BC420CD20B2C0AD808
:1017400012F8039012F8088002EB840209EA0C04F4
:1017500008EB042414610233102BE6D100232B7014
:1017600003788B420FD90C4B93F8400060B10B4AC1
:10177000890012780B44186902B1400800F57770AF
:1017800080B2BDE8F0830020BDE8F083F8000020BF
:10179000F0090020F10900207C0D0020F209002052
:1017A00007299ABF024B33F821000020704700BF81
:1017B000C4010020024B53F82100C0F3CF00704752
:1017C0006C010020034B53F82100400800F57770AE
:1017D00080B2704714010020014B33F811007047AC
:1017E000BA040020014B33F811007047481600205E
:1017F000034B4FF4004208B11A6170475A617047B9
:1018000000080140034B4FF4004208B15A61704791
:101810001A61704700080140032810B5114B0FD81A
:10182000114A126894888C420AD2D2888A4207D917
:10183000012202FA00F093F84120104383F841009E
:1018400093F841300F2B0CD1064B002283F8412036
:10185000064B998808B2142802DD1439998010BD0E
:101860009A8010BD7C0D0020C40F0020DC090020F0
:10187000024B9A8801329A80704700BFDC09002031
:10188000074B1A68074B1178B3F9040053780B44DF
:1018900003EB83039842D4BF00200120704700BFB0
:1018A000C40F0020DC090020064BB3F90400064BEE
:1018B0001B681B7803EB83039842D4BF00200120F0
:1018C000704700BFDC090020C40F002010B504469B
:1018D000FFF7EAFF002814BF2046002000F00100B7
:1018E00010BD024B01221A72704700BFDC090020B4
:1018F000014B187A704700BFDC090020034BB3F995
:101900000400D0F1010038BF00207047DC0900203E
:10191000014B00229A807047DC09002003685A1CA2
:10192000026019707047016B0346C26810B54069C8
:1019300041B1196C541A005D013918BF0A46C0B292
:101940001A6410BD196A405C0131B1FBF2F402FB6C
:101950001412C0B21A6210BD026B03691AB1516849
:10196000013B026C02E0C169026A013B881A18401F
:10197000C0B27047436B13B190F844007047826A5D
:10198000436AD31A584258417047334A10B5136C12
:1019900090681944081A40F68C2398429160D060F0
:1019A000516013463CD9127893F945108A420BD105
:1019B000111F082908D893F84610182901D80131B9
:1019C00003E083F8442002E0002183F8461093F9F5
:1019D00044108A421CD1204991F84710C1B100211E
:1019E00091421E4806DA03EB8104246920F8114075
:1019F0000131F5E7511E00EB41011630814203D061
:101A0000002421F8024FF9E71549087801300870E1
:101A100083F84520002201211A7083F8471010BD79
:101A200092F84710B9B1A0F2EF2440F2DA518C429B
:101A300008D811780B2905D80B1D0131117042F817
:101A4000230010BD002283F847209918043200209B
:101A5000302A0861F9D110BDC008002048160020C6
:101A6000DF100020084B03EB0010837A0133DBB258
:101A70000A2B837207D983781BB94178034A22F86D
:101A80001130002383727047080900204816002097
:101A9000024B1A6C11441964704700BFC008002043
:101AA000024B53F820301B681980704788090020CA
:101AB000074BA1F57A7153F820304FF47A701A6809
:101AC0009B884B4393FBF0F39BB21380704700BF9E
:101AD00088090020024B4FF480521A80704700BFE3
:101AE00000000020704738B50C68054620460BF012
:101AF0003DFE214602462868BDE838400BF03EBE58
:101B0000084BDA68D10709D4DA68520708D4DB68D1
:101B100013F0100F0CBF0420032070470120704702
:101B200002207047002002408A6810B50C6A0368E2
:101B300014430A6923F4FF4314434A6923F07003F2
:101B400014438A691443CA6914434A6A14438A6A6B
:101B5000224313430360CB6843600B6883604B6888
:101B6000C36010BD02684FF6FE731340036000238C
:101B7000036043608360C3602A4B984222D02A4BA3
:101B8000984229D0294B984230D0294B984237D0DF
:101B9000284B98423ED0284B984206D153F8682CE7
:101BA00042F4700243F8682C7047244B984206D1E7
:101BB00053F87C2C42F0706243F87C2C7047204B29
:101BC000984206D153F8042C42F00F0243F8042C3B
:101BD00070471C4B984206D153F8182C42F0F00283
:101BE00043F8182C7047184B984206D153F82C2C08
:101BF00042F4706243F82C2C7047144B984206D183
:101C000053F8402C42F4704243F8402C7047104B7C
:101C1000984205D153F8542C42F4702243F8542CC6
:101C2000704700BF080002401C0002403000024024
:101C300044000240580002406C0002408000024014
:101C4000080402401C0402403004024044040240E4
:101C50005804024010B5104B4178DB688478DB43B0
:101C6000C3F30223C3F1040201FA02F20F21D940A7
:101C700021401143094B02780901C9B21A4482F884
:101C8000001302780120510902F01F0200FA02F24B
:101C900043F8212010BD00BF00ED00E000E100E0AE
:101CA0002DE9F843574B0C460168013AC3F842103E
:101CB0008188A3F84610072A42D8DFE802F0040A18
:101CC000101822292F35B3F842202280B3F844207F
:101CD00013E0B3F844202280B3F8422005E0B3F8C3
:101CE000422052422280B3F84420524205E0B3F829
:101CF000442052422280B3F842206280B3F846303A
:101D00001DE0B3F8422052422280B3F8442012E092
:101D1000B3F844202280B3F842200CE0B3F842200C
:101D20002280B3F8442005E0B3F8442052422280D8
:101D3000B3F8422052426280B3F846305B42A3803F
:101D4000314B1B78002B5AD1B4F9000008F056FF34
:101D50008046B4F9020008F051FF0746B4F90400C8
:101D600008F04CFF294D06462968404608F09AFFC6
:101D7000E9688146384608F095FF0146484608F074
:101D800089FEA9698146304608F08CFF0146484625
:101D900008F080FE0BF00EFF69682080404608F0D6
:101DA00081FF29698146384608F07CFF0146484694
:101DB00008F070FEE9698146304608F073FF01467D
:101DC000484608F067FE0BF0F5FEA96860804046C3
:101DD00008F068FF69698046384608F063FF0146ED
:101DE000404608F057FE296A0746304608F05AFF79
:101DF0000146384608F04EFE0BF0DCFEA080BDE840
:101E0000F88300BF7C0D00202800002090060020F1
:101E1000074B084A1B7812889A4207D3064A126871
:101E2000907898428CBF00200120704700207047B6
:101E300014050020780D0020740D002010B5194BFA
:101E400093F84820511C83F84810174902F0070204
:101E50004878164903EB420331F81010A3F84A10F2
:101E600000231846124A9A5A02331044102B80B2AB
:101E7000F8D1C00808F0C2FE0E4908F013FF0E4961
:101E800008F0C4FF0D4B04461B68187808F0B6FE36
:101E90000146204608F006FF09F0F0F8084B1870DC
:101EA00010BD00BF7C0D00207806002088060020B1
:101EB000C60D00203333534000F07F45740D0020E1
:101EC00014050020034B1B68DA79511CD9711344A7
:101ED000187A7047AC05002010B5FFF7F3FF0446F1
:101EE000FFF7F0FF04EB002080B210BD10B5FFF744
:101EF000F3FF0446FFF7F0FF04EB004010BD074B73
:101F0000197A814207D01A7D824203D0084202D159
:101F1000104001D00C335868704700BF2C000020DF
:101F2000F0B5137C012B29D80C255D43144C0133EB
:101F300005EB040C9CF8086030421DD02D5D1DB1EE
:101F4000022D14BF022501250E4C4E7B04EB051417
:101F500016B1277B3E420FD04F686668B7420BD35D
:101F60008F68A668B74207D815709460C2F804C09D
:101F7000D16013741046F0BDDBB2D3E70020F0BD92
:101F80002C00002044F9000810B5094A09491368DB
:101F90008C6812689342F8D1074A106811684FF4B0
:101FA0007A725043001BB0FBF1F002FB030010BD3E
:101FB0000817002010E000E07406002038B5104C2F
:101FC0000123054684F84030FFF7DEFFE36D41F260
:101FD0008832C31A9342236684BF002384F8643096
:101FE00094F86430EDB20F2BE065E55403D1054B56
:101FF00001221A7038BD024A013382F8643038BDBC
:102000007C0D0020F800002010B50446FFF7BCFF4F
:102010000D4B41F288319A6E9866821A8A42DA66CE
:1020200084BF002283F8702093F87030074A142B85
:10203000D45403D1064B01221A7010BD024A013359
:1020400082F8703010BD00BF7C0D0020AD01002073
:10205000AC01002010B50446FFF796FF164A536FF7
:102060005067C31AB3F57A6F84BF002382F87830C3
:1020700092F8783023B9A82C1CD110490B7006E0D7
:10208000022B02D10E490C7001E0242B01D80D491E
:10209000CC540133DBB282F87830094A127852000E
:1020A0000532934206D1044B002283F87820034B7B
:1020B00001221A7010BD00BF7C0D002044010020D9
:1020C0006A0100204501002038B50446FFF75CFF97
:1020D000114B40F6C411DA6FD867821A8A4284BF66
:1020E000002283F8802093F880200AB90F2C11D1A8
:1020F0000A480021017052B1094D182A154405F80B
:10210000014C04D1012283F88010027038BD0132E5
:1021100083F8802038BD00BF7C0D0020F90000202E
:10212000FA00002038B50446FFF72EFF0546FFF7FA
:102130002BFF401BA042FAD338BD10B504462CB18A
:102140004FF47A70FFF7EEFF013CF8E710BD08B5D9
:10215000014B1B68984708BDE01C00202DE9F041A9
:1021600006460F4690460025EBB2434518D20024A0
:10217000E3B2B3420FD20B4B0120DA68013482F094
:102180000802DA60FFF7E3FF3846FFF7D6FF0020CA
:10219000FFF7DDFFECE73C20FFF7CFFF0135E3E77A
:1021A000BDE8F081000C01400B490B7813F0010FE2
:1021B00003F004020AD072B9980707D443F004036D
:1021C0000B70064B1A88064B1A8070471AB902200A
:1021D000FF210122C2E77047DC1C0020F80200202A
:1021E0003015002040F2DB14604308B50A4B08228A
:1021F0001A61841E084B2046DA6882F00802DA6011
:10220000FFF79BFF0120FFF7A2FF1920FFF795FFC3
:102210000020FFF79CFFEDE7000C014008B50368C4
:102220005B69984708BD08B503681B69984708BDF6
:1022300008B50368DB68984708BD08B503689B6864
:10224000984708BD08B503685B68984708BD10B596
:10225000044C2068FFF7F6FF18B12068FFF7EDFF88
:10226000F6E710BD9405002008B503681B68984781
:1022700008BD064B10B5044621461868FFF7F4FF69
:10228000034B1B689A7954409C7110BDB005002027
:10229000AC05002038B5044624200D46FFF7E9FFC1
:1022A0004D20FFF7E6FF002C084C0CBF3E202120FC
:1022B000FFF7DFFF2368002228469A71FFF7D9FF56
:1022C000236893F84900BDE83840D2E7AC05002008
:1022D00001460020DEE7F8B50E4E0F4C0F4DC1B29F
:1022E0000746306884F88110FFF7BEFF2B6894F82A
:1022F00081109A7930684A409A71C7F3072184F8AF
:102300008110FFF7B1FF2B6894F881109A794A4049
:102310009A71F8BDB00500207C0D0020AC050020AE
:10232000F8B51B4D1B4C1C4F0646C1B2286884F8FB
:102330008210FFF799FF3B6894F882109A79286819
:102340004A409A71C6F3072184F88210FFF78CFF88
:102350003B6894F882109A7928684A409A71C6F3CB
:10236000074184F88210FFF77FFF3B6894F88210E2
:102370009A7928684A409A71310E84F88210FFF7E2
:1023800073FF3B6894F882109A794A409A71F8BDBD
:10239000B00500207C0D0020AC05002010B5441EC7
:1023A00014F8011F21B1034B1868FFF75DFFF7E731
:1023B00010BD00BFB8080020014B186854E700BFEB
:1023C0001812002038B5054C05465E212068FFF73D
:1023D0004BFF20682946BDE8384045E70805002046
:1023E000014B5E2118683FE70805002010B50A4C34
:1023F0005E280146206805D15D21FFF735FF206882
:102400003E2105E05D2903D1FFF72EFF20683D2125
:10241000BDE8104028E700BF0805002010B50446BD
:10242000C0B2FFF7E3FFC4F30720BDE81040FFF799
:10243000DDBF10B50024094BE0B21B7883420CD9F4
:10244000074B33F81010074B53F820301BB10B2803
:1024500001D89B6898470134EDE710BDB01C0020FF
:10246000B21C002088090020054B1B6803EBC0004C
:1024700090F9063019420CBF01204FF0FF30704731
:10248000A00400200A4B1A6802EBC002D379FF2B8C
:1024900007D008490978994203D9074A32F813004E
:1024A00004E00728D4BF908840F2DC5000B27047A7
:1024B000A0040020F3090020BA0400202DE9F04F09
:1024C0000C68836889B0D0F800A0D0F80480064674
:1024D000204603938B460BF037FB074620460BF054
:1024E000A7FBDBF80440814620460BF02DFB054698
:1024F00020460BF09DFBDBF80820044610460192B5
:102500000BF022FB019A834610460BF091FB3946F3
:102510000290584608F0C6FB39460490029808F02D
:10252000C1FB59460590484608F0BCFB029906904D
:10253000484608F0B7FB29460790584608F0B2FB1A
:102540000146504608F0AEFB21468346069808F047
:10255000A9FB0146059808F09DFA0146404608F09F
:10256000A1FB0146584608F095FA21468346049897
:1025700008F098FB0146079808F08AFA014603988C
:1025800008F090FB0146584608F084FA3060029942
:1025900005F1004008F086FB0146504608F082FB3A
:1025A00021468346079808F07DFB0146049808F011
:1025B0006FFA0146404608F075FB0146584608F0A0
:1025C00069FA21468346059808F06CFB0146069897
:1025D00008F060FA0146039808F064FB014658468B
:1025E00008F058FA21467060504608F05BFB294617
:1025F000044609F1004008F055FB0146404608F04A
:1026000051FB0146204608F045FA39460446284663
:1026100008F048FB0146039808F044FB01462046B9
:1026200008F038FAB06009B0BDE8F08F2DE9F84F36
:10263000374E0446376838460BF086FA054638466A
:102640000BF0F6FA7668804630460BF07DFA83464A
:1026500030460BF0EDFAD4F8049006462946484679
:1026600008F020FBA76882464146384608F01AFB6E
:102670000146504608F00CFA21688246584608F098
:1026800011FB41460446484608F00CFB314608F071
:1026900009FB0146204608F0FDF93146044638465C
:1026A00008F000FB294608F0FDFA0146204608F034
:1026B000F1F9014650460BF049FB164908F0F2FAD1
:1026C00007F00CFF10A3D3E9002308F085F8124BA4
:1026D000044618680D4607F001FF02460B462046E7
:1026E000294607F09DFD00220C4B08F075F808F014
:1026F0007BF90BF05FFA83B21A0444BF00F5B473A0
:102700009BB218B2BDE8F88F182D4454FB21094044
:10271000E00200200000E144B80600200000244050
:1027200080EAE073A3EBE0738B4206DB002801DD57
:10273000401A704702D00844704700207047074B8A
:102740001B7803F0040303F0FF001BB1044B18884F
:10275000C0F3C01000F00100704700BFDC1C002077
:1027600042030020034B1A78510744BF22F00402B1
:102770001A707047DC1C002070B5FFF795F838B36D
:10278000144C237A0BB9A38070BD134D2E78C6F379
:102790008000FFF79BF890B1104B46F002061A68D4
:1027A0000F4B51892E7019805189598052899A8016
:1027B0000C4A12685288DA80E3880133E380FFF71D
:1027C0005FF810B92B785B0702D4BDE87040C9E709
:1027D00070BD00BFDC090020DC1C0020D8090020EF
:1027E000BA040020C40F00202DE9F041027803460E
:1027F000202A00F10100F9D0092AF7D02D2A02D1B0
:102800000346414D04E02B2A08BF03464FF07E5596
:102810001E460024334616F8012BA2F13007F9B208
:1028200009290DD83949204608F03CFA04463846B3
:1028300008F0E4F90146204608F02CF90446E9E7DF
:102840002E2A17D1314F334616F8010B3038C2B259
:10285000092A0FD808F0D2F9394608F0D7FA01460C
:10286000204608F017F929490446384608F01AFAB4
:102870000746E8E71A7802F0DF02452A38D15A788D
:102880002D2A02D10233012604E02B2A14BF013382
:1028900002330026013B002713F8012F303AD1B252
:1028A000092903D80A2101FB0727F5E7B7F59A7F25
:1028B00028BF4FF49A77B8464FF07E51B8F1070F12
:1028C00007D90846124908F0EDF9A8F108080146B1
:1028D000F4E707F0070737B108460C4908F0E2F9BA
:1028E000013F0146F7E72EB1204608F08FFA04E0D9
:1028F0004FF07E51204608F0D5F90146284608F0F1
:10290000D1F9BDE8F08100BF000080BF0000204188
:1029100020BCBE4CF0B50124B0FBF4F58D4201D3D0
:102920004C43F9E70026DCB1B0FBF4F504FB1500DD
:10293000B4FBF1F41EB9002D01DC002CF3D1092DFC
:1029400003F101075FFA85FC04DD002A0CBF57255F
:10295000372500E0302565441D7001363B46E2E72F
:102960001C70F0BDF0B50124B0FBF4F58D4201D32D
:102970004C43F9E70026DCB1B0FBF4F504FB15008D
:10298000B4FBF1F41EB9002D01DC002CF3D1092DAC
:1029900003F101075FFA85FC04DD002A0CBF57250F
:1029A000372500E0302565441D7001363B46E2E7DF
:1029B0001C70F0BD70B50646B6FBF2F4084615462D
:1029C00014B12046FFF7F6FF05FB1464024B1B5DB4
:1029D00000F8013B70BD00BFF20901082DE9F0418C
:1029E000069C002B06460F460CBF4FF020084FF008
:1029F0003008234613F8011B09B9154603E0002AE5
:102A0000FBDD013AF6E7002D04DD30464146B847CC
:102A1000013DF8E714F8011B11B13046B847F9E75A
:102A2000BDE8F081024B9A6822EA00009860704786
:102A30000C17002030B50E4D0028B8BF40420D4C99
:102A400090FBF5F304FB03003C22424392FBF5F0BC
:102A500003EB830304FB002203EB830300EB8303FC
:102A60000B804FF47A7392FBF3F24A8030BD00BFC3
:102A700080969800806967FF094B1B7873B1094BFA
:102A80001B685B782BB1084BD87C003018BF012045
:102A90007047064B1878C0F38000704701207047DC
:102AA000640D0020040500202C030020DC1C002005
:102AB000094A0A48002310B5116803701A46CC1859
:102AC00064880CB9CC5C24B104330132802BD2B2BF
:102AD000F5D1027010BD00BFC80500204C060020D3
:102AE00010B50C4B0C4819780C4B93F883204B080D
:102AF0005C1E047001F0010109480B440370094990
:102B00005308581E087002F00102074913440B7065
:102B100010BD00BF610600205C0600207C0D002077
:102B20005E0600205F0600205D060020F0B5104A1A
:102B300010481678104A0023176880F883301A4628
:102B400019460546D0B2B0420CD217F82200013225
:102B500004099C4200F00F00A8BF631C8842A8BF74
:102B6000411CEFE785F88330044B1970F0BD00BFBE
:102B70004C0600207C0D0020C805002061060020C6
:102B8000F8B5101A0C461F4608F038F80546381BF1
:102B900008F034F8174B079E196808F083F82946A7
:102BA0000446284608F07EF821460746204608F0ED
:102BB00079F80146384607F06DFF0BF0C9F80E4969
:102BC00008F070F808F05AFA069B2146186005F1E3
:102BD00000400BF0BBF8094908F064F8084907F019
:102BE00059FF08F025FA0028BCBF00F50C40A030C2
:102BF0003060F8BD440000202C7D8E3FA00CB34512
:102C000000A00C4610B507F0F9FF0021044608F0BB
:102C100005FA08B1204601E004F10040054908F03A
:102C2000F5F8054908F03EF80AF08EFF034B1860EE
:102C300010BD00BF8096184B35FA8E3C4400002032
:102C400070B50446007907F0D5FF1E4908F0DEF89C
:102C50001D4D1E4E2860A07B07F0CCFF194908F0DF
:102C6000D5F8EE606860607907F0C4FF184908F095
:102C7000CDF8184D2860E07B07F0BCFF114908F043
:102C8000C5F86860607E07F0B5FF134908F0BEF82C
:102C9000EE60A860A07907F0ADFF0D4908F0B6F826
:102CA0000E4D2860207C07F0A5FF064908F0AEF81D
:102CB0006860A07E07F09EFF074908F0A7F8EE6065
:102CC000A86070BD0000C842800F00200000FA44D8
:102CD00000002041900F002000007A44B40F002033
:102CE00044F25063984203DDA0F50C40A0387047D1
:102CF000034B9842BCBF00F50C40A030704700BFAA
:102D0000B0B9FFFF10B50023094CDAB204EB82041E
:102D1000246A01338442F7D10023064CD8B234F838
:102D2000104001338C42F8D102EB8000C0B210BDDC
:102D300044F9000880FB0008044B53F820301BB115
:102D400007289CBF1B681980704700BFB809002086
:102D500010B5054C00202188FFF7EEFF61880120A7
:102D6000BDE81040E8E700BF5E0000202DE9F0411B
:102D70000F88002347FA03F2D2072BD58A7803F095
:102D8000070512F0100F18BF91F803C002F00F06EC
:102D900018BF46EA0C06AD004FF00F0C0CFA05FC0C
:102DA00006FA05F5DC0850F82480282A28EA0C0CDD
:102DB00045EA0C0540F8245005D101229A40C46828
:102DC00024EA020205E0482A04D101229A40C4689C
:102DD0002243C2600133102BCCD1BDE8F081034BFC
:102DE0001A88013292B21A80704700BFB4060020E0
:102DF0002DE9F04F974B91B01B68BBB9964C2378E7
:102E0000013B042B00F2F886DFE813F015061506E7
:102E10001506E606CC062068FFF70FFA8F4B04462E
:102E20001B681B784BB1012B00F0ED80894C2068AA
:102E3000FFF708FA0028EED1E0E72428884D0CD0EF
:102E400006D80A2800F08E800D2800F08B80C6E09E
:102E50002A2806D02C2804D0C1E02B706B70AB70F0
:102E6000CEE06A782E782A4400217D4BD170EEB9ED
:102E7000DA789E74472A19D11A79502A16D15A79CC
:102E8000472A07D19A79472A04D1DA79412A01D110
:102E900001229A746A79724B522A07D19A794D2A83
:102EA00004D1DA79432A04BF02229A74AB7C6C4FB6
:102EB000012B02D0022B36D049E0B31E072B46D897
:102EC000DFE803F0040810141C27452C03F0DCFA9B
:102ED00068613CE0EA78624B532A38D15A69524221
:102EE0005A6134E003F0D0FAA86130E0EA785C4B34
:102EF000572A2CD19A6952429A6128E0EB78302BFC
:102F0000584B1A788CBF42F0020222F002021A706B
:102F10001DE0002003F012FB287718E0002003F0EA
:102F20000DFBE88313E0072E06D0082E0FD10120F9
:102F300003F004FB78840AE0012003F0FFFA41F279
:102F4000184358434FF47A72B0FBF2F33B840136D6
:102F500000232A2C424A2E706B704CD1012182F83A
:102F600024104DE095F82430002B34D03C4BDB7816
:102F7000402B04D9A3F137021201D2B202E01B01A7
:102F800003F0F0022B79A978402B8CBF373B303B04
:102F9000DBB21344DBB29942314A1BD1937C012B43
:102FA00008D0022B16D1118C2F4B528C19802F4B2D
:102FB0001A800FE02B4909788E070CD52C495069EF
:102FC000086090694860107F2A490870D18B2A4AAE
:102FD000118000E00023002285F8242010E06B78A7
:102FE0001F4A0E2B03D8591C13445170DC7095F8FE
:102FF00024301B4A1BB991784C40947000E00023A8
:1030000003F001035BE1164B002193F82520082A09
:1030100000F25481DFE802F00B0514324353718D46
:103020009A00622801D1022207E083F82510B52C0E
:1030300040F0448193F82520013283F825203DE1BA
:10304000032283F8252083F8260083F8270083F8DD
:10305000280033E1300A0020100A00202C0A00204A
:10306000000E0020DE02002086050020E20F002076
:1030700020050020580500208A050020042283F83E
:10308000252093F8272093F828100244D2B283F821
:1030900027200A4483F8282083F829000EE105221E
:1030A00083F8252093F8272093F828100244D2B201
:1030B00083F827200A4483F828205885FEE006215B
:1030C00083F8251093F8271093F828002144C9B2FB
:1030D00083F82710014483F82810598D6A4A01EBC0
:1030E0000424A4B2B4F5007F89BF00215485518522
:1030F00082F8251000229A85E0E093F8272093F8C3
:1031000028100244D2B283F827200A4483F82820EA
:103110009A8DC72A03D85C49114481F830000132E6
:1031200092B29A855B8D934240F0C8800722564B3D
:1031300083E7082283F8252093F82730834200F0A4
:10314000BD80514A002382F82530B8E083F825106D
:1031500093F828104C4A814240F0B08092F8291030
:10316000062946D004D8022912D003292CD0A5E084
:10317000122957D0302940F0A18092F83410434AE8
:10318000102988BF1021117010784149002257E0A2
:103190004049506B4860906B0860116C4FF47A7036
:1031A00091FBF0F13C48018092F8F8103B4A19B1CC
:1031B000117841F0020102E0117821F00201117052
:1031C000012283F8F92050E092F8351011F0010146
:1031D00005D092F83420D41E6242624100E00A46D3
:1031E00083F8F820002A40D12C4A117821F00201FE
:1031F00016E092F83B1011F0010105D092F83A2048
:10320000D01E4242424100E00A4683F8F82022B92B
:10321000224A117821F00201117093F85F10204AC0
:10322000117022E0516C1F480180916C42F21070C5
:1032300091FBF0F11C480180012182F8FA1014E0A2
:10324000824201F10C0110DA11F8045C174C15559B
:1032500011F8035C164C155511F8015C154C155509
:103260000D78154C15550132EAE793F8F930064A06
:1032700023B392F8FA300BB3002382F8F93082F8C6
:10328000FA3001231BE000BF000E0020E40F0020F5
:10329000300E0020200500208A050020DE020020DC
:1032A0005805002086050020E20F0020E50F0020D1
:1032B000F50F002005100020151000200023002B22
:1032C0003FF4B4ADA54BA64E9A68DA6032689A60B6
:1032D000A44B1A6842F020021A60A34B1A78012A04
:1032E0000CBF002201221A70A04B1A7891077FF5BB
:1032F0009DAD9F49097804297FF698AD9D490978CD
:1033000001F0040101F0FF0011B922F001021A706E
:103310001B78964F13F0010F974C984D11D180B147
:103320009B070ED5964B28686A6818605A60FFF7AD
:1033300069FC944B1B88A4F8FC303B7843F00103F4
:103340003B7094F8FE304FF00509013393FBF9F917
:1033500009EB8909C9EB03098B4B8C481B7884F86E
:10336000FE900593831D03EB890907900023DFF886
:103370000CE2874A53F80E00864F985090FBF7FCFA
:1033800002F1080743F807C0834F03EB0E0107FB68
:103390000C0742F2107097FBF0F00691079980B28B
:1033A00021F8020F02F1100A03EB830B049007913E
:1033B00053F80A0059F80B1049F80B70C1EB0008DC
:1033C00008EB0700734F4FF0050843F80A0090FB25
:1033D000F8F007FB0C000599183201299850774640
:1033E00008D1DDF810E0AEF10202B2F5797F9CBFA2
:1033F000069908600433082BB9D1DFF87C81306866
:10340000D8F84C31C01A07F0F5FB644907F0FEFC10
:1034100033684FF07E51C8F84C31814607F0E0FD2B
:1034200010B94FF07E5000E048460CAAC4F8500195
:10343000534B00920DAA019297E803000CCBFFF7C3
:103440009FFB0C9B56496422B3FBF2F30D980B8053
:10345000544B90FBF2F21A80444A474E127812F015
:10346000010208BF1A8098F8543108BF0A80002B67
:103470003AD0D6F850114FF07E5007F0C7FCD6F87E
:10348000583181462868C01A07F0B8FB494607F052
:1034900009FC07F0CDFDD6F85C211FFA80FA6868B8
:1034A0000FFA8AFA801A07F0A9FB3F4B196807F058
:1034B000F9FB494607F0F6FB07F0BAFDB6F96231B1
:1034C00000B2C218B6F960310221534492FBF1F206
:1034D00093FBF1F392B29BB2A6F86621A6F8643191
:1034E000A6F86221A6F86031012388F854312F4BE9
:1034F00079681B88386803F030031F4D1F4EC8F8E9
:103500005C11C8F85801002B3FF490AC05F5B87376
:10351000009305F5BA730193D5F86821D5F86C319D
:10352000FFF72EFB7368D5F86C01C01A07F066FB35
:103530001D4B196807F0B6FB07F07AFDD5F8683126
:103540003268C5F87C019B1AC5F878310E4B1B78A0
:10355000012B2DD0022B00F0F98067E4100A002027
:103560000817002068020020E51C0020DE02002071
:1035700058050020DC1C0020000E00202005002043
:1035800054150020F802002068150020FE0E0020CF
:103590002C0F002080969800806967FF00007A4415
:1035A000880500208C0500204400002042030020F4
:1035B000D5F88071D5F89C410497D5F8907104F145
:1035C00000400597D5F89471D5F85061079707F03A
:1035D0002FFD8046204607F02BFD8F4BD5F89851E4
:1035E0001B688E4C0695089009930025DFF84CA2C5
:1035F0005AF81570AAF11403384635F8039007F00D
:10360000FDFA049907F04EFB07F012FDC9EB00002C
:1036100080B20AF1280A25F80A000FFA80FA50460B
:1036200007F0ECFA059907F03DFB07F001FD1FFAE2
:1036300080FB0AEB070007F0E1FA079907F032FB7D
:10364000314607F02FFB216807F024FA07F0F0FC61
:10365000404505DBDDF820E07045A8BF704600E07E
:10366000404607F0CBFA206007F0E2FC58441FFA0E
:1036700080FB606809F13109381A07F0BFFA31465A
:1036800007F0C4FB0999206184468878D4F808A023
:10369000CDF80CC007F0AEFA06F020FF5CA3D3E92A
:1036A000002306F06FFF02460B4600205C4907F03E
:1036B00093F807F099F9314607F0ECF901463046E6
:1036C00007F0A4FBDDF80CC00346514660460393A7
:1036D00007F0DEF9039B0146184607F0E3FA0146BE
:1036E000504607F0D7F91FFA89F9B9F1620F014680
:1036F00020616760A0600ED9069807F0D3FA07F042
:1037000097FC484BB0F5FA6FA8BF4FF4FA609842A7
:10371000B8BF184600E00020834440F6B8330FFAE3
:103720008BFB9B45A8BF9B463F4B0A229B45B8BFDE
:103730009B466A433D4B54F8141B25F803B03C4BA1
:103740000235042DD1503FF471AB4FE7324BD5F821
:1037500070B11F68B5F8A461B7F808904FEA5B0331
:10376000994528BF994633B2994502DC1FFA89F979
:103770000BE03049D5F8500107F094FA07F058FCF7
:1037800030441FFA80F9A5F8A491D8F87451D8F8FC
:10379000A861AE1B3046FFF7A3FA0028D8BF40420D
:1037A00041F293139842CCBF00200120002847D05B
:1037B000304607F023FA204907F074FA0AF038FA85
:1037C0000646584607F016FA0146304607F06AFAF0
:1037D00007F02EFC80B240F6B83203B29342A8BF85
:1037E0001346114AA8F8AC019342ACBFEB18AB18D2
:1037F00048F6A042934203DDA3F50C43A03B04E04E
:10380000002BBCBF03F50C43A033C8F8B03119E05E
:10381000182D4454FB211940C8030020BC1500207A
:103820000000F03F30F8FFFF48F4FFFFD003002016
:10383000E41500200000C842D3023739780F002079
:10384000C8F8B051D4F8B021C2F50C502830049219
:1038500007F0D4F9AE4907F025FA05460AF074F9E5
:103860000F9028460AF0E4F9D4F8C051D4F8B431E6
:10387000D4F8B8E10E9005F100400793CDF828E0A8
:1038800007F0D6FB0590284607F0D2FBD4F850810C
:10389000D4F8BC410B9009949E4C0025484607F093
:1038A000ADF90EAB53F8151007F0FCF9DFF8A0A244
:1038B00006463AF9050007F0A1F90146304607F03F
:1038C000E7F807F0B5FB944B06B2B6F57A7FA8BFD0
:1038D0004FF47A769E42B8BF1E46B0B20AF13C0A57
:1038E00025F80A0000B207F089F90799824607F027
:1038F000D9F907F09DFB80B208900A99504607F06D
:10390000D1F9414607F0CEF9216807F0C3F807F076
:103910008FFB0599884204DB0B9A9042A8BF1046A2
:1039200000E0059807F06AF9824620606068143468
:10393000301A07F063F9414607F068FA54F80C3C76
:1039400044F8040C8446B8780693CDF80CC007F010
:1039500051F906F0C3FD6CA3D3E9002306F012FE73
:1039600002460B4600206D4906F036FF07F03CF892
:10397000414607F08FF80146404607F047FADDF868
:103980000CC0034606996046039307F081F8039B39
:103990000146184607F086F90146069807F07AF8BE
:1039A00044F8106C014644F8040C44F80C0C0998D7
:1039B00007F078F907F03CFB089E0644504607F0F4
:1039C00037FB304440F6B83300B29842A8BF1846DF
:1039D000534B0A229842B8BF18466A43514BE852EB
:1039E000514B0235042D42F803A07FF457AF3B79C9
:1039F0002BB1049864224D4B90FBF2F21A803B8865
:103A00004B4C9B450ED9D4F8A831D4F87401C01A98
:103A1000FFF766F942F210730028B8BF404298429F
:103A20007FF704AA434B01221A70B4F8FC203F4BE5
:103A30001A80FFF7FBB9404A116890460F7817B11A
:103A4000012F0DD0ABE0012B00F2A98062783B4B37
:103A500003EB02133A4A59681068FEF7E9FB9BE052
:103A6000374E3068FEF7DFFBB146002800F0978044
:103A70002378344D022B29D0032B31D0012B40F079
:103A80008E80314B1F686B69FB1A632B40F2878075
:103A90002B69042B18D8DFF8A480306808EB0313D7
:103AA0005968FEF7C5FB6B78366808EB03139D6811
:103AB00015F8011B19B13046FEF7D6FBF8E723696C
:103AC0006761013323616AE0022066E06A781B4B7C
:103AD000306803EB02135968FEF7AAFB03205CE091
:103AE0002B7E03B92F76237E164D012B36D12B6901
:103AF0007B2B2FD8154AD9F80000D15CFEF7B4FB18
:103B00002B6901332B6129E0182D4454FB21194006
:103B1000D3023739E415002018FCFFFF0000F03F06
:103B200048F4FFFFD0030020BC15002050150020F2
:103B3000000E0020681500202C0A00201CF400084C
:103B4000300A0020100A00200817002074F900082D
:103B5000640F002000232B6102232B76237E284D47
:103B6000022B16D12B690F2B11D8D8F8002025492C
:103B70005278D9F8000002EB02120A44134493F879
:103B80007D10FEF771FB2B6901332B6101E00323EC
:103B90002B76237E022B02D9042001F07FFE002326
:103BA000636029E063680522013363606378012064
:103BB0000133DBB2B3FBF2F202EB82029B1A6370B9
:103BC000114B00221B68A360104B1A70104B1A781F
:103BD00022F002021A700DE00B4B1A68A368D21A89
:103BE00040F6C4139A4207D90A4B05201A6822F0FE
:103BF00020021A6001F052FE11B0BDE8F08F00BF44
:103C0000100A002074F90008081700205805002049
:103C1000DE020020680200202DE9F74F05F00EFCBF
:103C200010B90A20FEF7DEFA8C4C40F2A45220466E
:103C30008B4909F051FD94F8A0354FF49A72022B8C
:103C400084BF002384F8A03594F8A035854F02FB8B
:103C5000034303F501733B60A36842F201021A407B
:103C60003AB944F208021A401AB97C4A43F40053A4
:103C70009360A368DB0703D54FF40050FEF7D2FE34
:103C8000A3685E0409D50820FEF7CCFE4FF400506F
:103C9000FEF7C8FE0120FEF7C5FEA3681D0706D586
:103CA0004FF40050FEF7BEFE0120FEF7BBFEA368F6
:103CB00098040ED54FF40040FEF7B4FE4FF40060B8
:103CC000FEF7B0FE4FF48030FEF7ACFE4020FEF76A
:103CD000A9FEA368590603D54FF48030FEF7A2FE73
:103CE000614B624D1D6005F0D1FE614B05F11A027A
:103CF00001201A6005F066FC0146012005F04EFB2C
:103D0000002840D0022005F05DFC0146022005F0AD
:103D100045FB002837D0102005F054FC0146102048
:103D200005F03CFBA3681A0600D560B3082005F037
:103D300049FC0146082005F031FBA3681B0700D5AC
:103D400008B3042005F03EFC0146042005F026FBE4
:103D5000A3685E0503D400231A46194609E000282B
:103D6000F9D110E079B90121C00708D40C33182B20
:103D70000BD040481844007A8507F5D5F2E70132A8
:103D8000D2B2022AF2D905F096FA3868002390F8E8
:103D9000516090F8505003FB03F11939714301F65B
:103DA000C4115943694340F6C41291FBF2F1324AFF
:103DB00022F813100133072BEDD190F85230B4F8EC
:103DC000D0E0B4F8D22090F853C0CEEB0202C3F199
:103DD000640B03EB83085D4201925FFA8BFB4FEAB1
:103DE0004808CCF16409ADB20022AEB231B200296C
:103DF00004DC002E14BF1E46012600E05E4601FBD7
:103E000001FA76430AFB0CFA9AFBF6F64E4471432C
:103E10004FF00A0A91FBFAF108EB0106019936B25C
:103E20004E434FF47A7196FBF1F61449764456529C
:103E300002325544182AADB2D7D1114B114A136042
:103E4000114A4C3313600278104B012A03D0022A26
:103E500022D00F4A21E00F4A1FE000BF0C170020BC
:103E600000F80108F8010020F40000201A180020D2
:103E7000040800202C000020001500201815002048
:103E8000001800201402002004050020700000200B
:103E9000B16A00081D6900083F4A1A603F4B00F5EF
:103EA000947204301A60FEF7CBFE3D683C4E05F577
:103EB0008E7333603B4B00229A803B4B3B4A05F1AB
:103EC000DC0113603A4AB4F8F0001160394AA3F1FA
:103ED00022011160384AA3F128011160374A05F523
:103EE00092711160364A2C331360364B364A1A6091
:103EF000364B05F593721A6006F07CFEB060B4F89C
:103F0000F20006F077FE95F86030321D337195F8B7
:103F10007C30F060737194F82331B5F8D8003374B5
:103F20002B4B1A602B1D736105F16C03B361294B98
:103F300005F168021A6006F061FE0146264806F0A7
:103F400065FF06F0CBFA10A3D3E9002306F01AFBB5
:103F500006F04AFD214B1860686E06F0BFFA0CA30C
:103F6000D3E9002306F00EFB02460B4600201C4955
:103F700006F032FC06F038FD1A4B186003B0BDE8BD
:103F8000F08F00BFAFF300803B597E90A9E78140DE
:103F9000182D4454FB210940316D0008C80300204E
:103FA000C40F0020DC090020041800208402002037
:103FB000A0040020E0040020A4040020DC03002072
:103FC000A8040020AC0400201A180020B40400202B
:103FD000B80200201403002000006144C403002044
:103FE0000000E03F0403002070282DE9F84300F0B2
:103FF000858200F2D280692800F00F8200F2A4804E
:10400000662800F0668100F29480642800F0368112
:10401000652840F038840B20FEF75AF9CF4BB3F9EE
:104020000000FEF758F9CE4B988B00B2FEF753F91B
:10403000CC4B1B68C3F3C000C3F38002800040EA8E
:104040004200C3F340021043C3F3401240EAC200EF
:1040500003F010031843FEF73EF9C34B1A88C34B15
:1040600002F0080493F8069093F8078093F808C0CC
:1040700044EA891444EAC81444EA0C2493F80CC0B6
:1040800012F0010F44EA0C3493F80DC00CBF4FF04E
:10409000000E4FF0020E44EA4C3493F80FC012F0B9
:1040A000020F44EACC3493F810C00CBF0027042759
:1040B00044EA0C4493F811C012F0040F44EA4C4453
:1040C00093F812C00CBF0026102644EA8C4493F8E3
:1040D00013C01B7D44EACC4444EA0354A44B12F0C1
:1040E000400F1B780CBF00252025C3F380031C4321
:1040F00044EA0E043C4312F0100F44EA06040CBFDD
:1041000000204FF400702C4312F0200F0CBF002150
:104110004FF480610443974B12F4807F44EA01041A
:104120000CBF00224FF400620020197814430346AC
:10413000BAE0672800F00681682840F0A4831020C8
:10414000FEF7C6F8002460E16C2800F0798117D8EA
:104150006A2800F02A836B2840F095830520FEF73B
:10416000B7F8854BB3F90000FEF7B5F8834BB3F908
:104170000000FEF7B0F8824B187800F0010006E36B
:104180006E2800F06D8100F293810620FEF7A0F802
:104190000020FEF7C5F8002060E3772800F0BD821C
:1041A00045D8732800F0F68239D8712800F038829B
:1041B000722840F06883734C1620FEF789F80020BF
:1041C000FEF789F8B4F9D000FEF785F86E4DB4F922
:1041D000D200FEF780F8B4F9D400FEF77CF82B6823
:1041E000B3F91E01FEF777F80020FEF774F80020FF
:1041F000FEF796F82B68B3F95A000A2390FBF3F008
:10420000FEF769F894F80401FEF733F894F8060114
:10421000FEF72FF894F80501FEF72BF8B6E27528A3
:1042200000F0F28100F29482002701244DE2A028E0
:1042300000F017830AD8782800F0B8807B2840F077
:1042400022830820FEF744F80024D2E0F02800F092
:10425000F982FE2800F0EA82A42840F01483404D41
:10426000002495F820002E4680000130C0B2FEF7F1
:104270002FF895F82000FDF7FCFFBFE20720414C26
:10428000FEF726F8E620FDF7F4FF6079FDF7F1FF71
:104290000020FDF7EEFF94F824013C4B3C4A002837
:1042A0000CBF10461846E9E28B420CD2394A9D5C9D
:1042B000012202FA05F5254218BF9A4003F10103D5
:1042C00018BF1043F0E7FEF72BF82E4B93F8A0052C
:1042D0005DE21220FDF7FCFF2F4B304C1B88B3F53D
:1042E000806F22D90025605F082390FBF3F0023530
:1042F000FDF7F1FF062DF6D1294CB4F90000FDF7CA
:10430000EAFFB4F90200FDF7E6FFB4F90400254C1A
:10431000FDF7E1FFB4F90000FDF7DDFFB4F902009D
:10432000FDF7D9FFB4F9040098E2B4F90000FDF7F5
:10433000D2FFB4F90200FDF7CEFFB4F90400FDF797
:10434000CAFFD9E71020FDF7C3FF0024164B185D04
:104350000134FDF78EFF102CF8D191E224030020E8
:10436000C40F002068020020420300202C0300201C
:10437000DC1C00201D080020880500208C05002082
:10438000E51C00200C170020F80100203C000080F4
:10439000340000800808002000000020C80200202F
:1043A0001C030020660600205E0000203820FDF778
:1043B0008FFF0025B04E05F11B043368E400234451
:1043C000B3F90400FDF787FF336801352344B3F9DF
:1043D0000600FDF780FF33682344B3F90800FDF7BA
:1043E0007AFF33681C44A07AFDF743FF082DE1D122
:1043F00046E2A14B1B6803EBC40393F8E3000134CE
:10440000FDF737FF082CF4D13AE29C4B185D0134DC
:10441000FDF72FFF102CF8D132E2994D00242878B7
:10442000400000F0FE00FDF753FF2B789C4280F027
:104430002782944B33F91400FDF74DFF0134F4E764
:10444000914C0620FDF744FFB4F90000FDF743FF4F
:10445000B4F90200FDF73FFF8C4BB3F90000FDE11A
:104460000720FDF735FF8A4B4FF6FF741878FDF7EC
:1044700000FF884B1868A042A8BF204620EAE070E1
:1044800000B2FDF728FF844BB3F90000FDF723FFCE
:10449000824B93F80C21824B18680028B8BF404229
:1044A0000AB10A235843A042A8BF204600B2D5E172
:1044B000714C0720FDF70CFF236893F85000FDF7BF
:1044C000D8FE236893F85100FDF7D3FE236893F8D4
:1044D0005400FDF7CEFE236893F85500FDF7C9FEA2
:1044E000236893F85600FDF7C4FE236893F8520042
:1044F000FDF7BFFE236893F8530048E15E4D1E2090
:10450000FDF7E6FE2B6800241B78022B69D12B688F
:10451000644903EB8403586A06F0C4FB09F04AFBC4
:10452000FA28A8BFFA2020EAE070C0B2FDF7A1FE89
:104530002B685D4903EB8403186B06F0B3FB09F0AD
:1045400039FBFA28A8BFFA2020EAE070C0B2FDF7D4
:1045500090FE2B68554903EB8403D86B06F0A2FB51
:1045600009F028FB6428A8BF642020EAE070C0B2EC
:104570000134FDF77EFE032CC9D1072C2B681ED118
:10458000986C484906F08EFB09F014FBFA28A8BF86
:10459000FA2020EAE070C0B2FDF76BFE2B684149BB
:1045A000D86C06F07FFB09F005FBFA28A8BFFA20BB
:1045B00020EAE070C0B2FDF75CFE00200BE023446F
:1045C0001879FDF756FE2B682344987BFDF751FEC2
:1045D0002B682344187E0134FDF74BFE0A2CCCD106
:1045E0004EE12B6823441879FDF743FE2B682344E2
:1045F000987BFDF73EFE2B682344187E0134FDF7BF
:1046000038FE0A2CEDD13BE12F20FDF761FE284C4E
:1046100014F8010F002800F03381FDF72AFEF7E7B8
:10462000244D00242878800000F0FC00FDF750FEA7
:104630002B789C420CD2204A0F4BA25C1B68203284
:1046400053F822000134C0F30B00FDF744FEEFE7FE
:1046500000242B789C4280F01381074B164A1B687C
:10466000A25C013403EB8203B3F88200C0F30B00B9
:10467000FDF731FEEDE700BFF8010020B21C00207D
:10468000F3090020BA040020E8020020F80200200C
:10469000140500201C050020721500200C170020B6
:1046A00018050020000020410000C84200007A44A4
:1046B00047FA00081D08002008080020002C00F020
:1046C000DF80F8B2FDF704FE002400256F4B1B7855
:1046D0009D42F3DA6E4BE95C00236E4A03EB02085D
:1046E0009A5C8A4204D00C33B3F5847FF5D112E092
:1046F000D8F8040009F03AF881460CB9264601E0E2
:10470000074408E04E4506DAD8F80430985DFDF716
:10471000B0FD0136F6E70135D8E75C4D0024287876
:10472000FDF7D6FD2B789C4280F0AA80584BE05CC8
:104730000023584A99189A5C824204D00C33B3F58E
:10474000847FF6D102E0087AFDF793FD0134E9E7B2
:10475000FDF7B8FB06461220FDF7BAFD002E46D144
:104760004D4B1D685C683046FDF783FD2846FDF71C
:10477000D7FD2046FDF7D4FD484B1868FDF7D0FD66
:104780000020FDF7A8FD0020FDF7A5FD0020FDF7A6
:1047900070FD75E00820FDF79BFD0124E0B20134B7
:1047A000FDF767FD092CF9D16AE01020FDF790FDB7
:1047B0003B4B3C4C187800F00200FDF75AFD3A4B99
:1047C0001878FDF756FD2068FDF7AAFD6068FDF733
:1047D000A7FD364BB3F90000FDF77DFD344BB3F96F
:1047E0000000FDF778FD334BB3F91E0036E0102EC4
:1047F00001D1314BB5E700242546B4E796F82030C7
:104800009C423DD22D4D285DFDF733FD05F110038F
:10481000185DFDF72EFD05F12003185D3035FDF71D
:1048200028FD285DFDF725FD0134E7E70820FDF7A9
:104830004FFD0024224B185F0234FDF74CFD082C7D
:10484000F8D11DE01F4C0420FDF742FD2368B3F9A9
:104850005E00FDF740FD2368B3F95C00FDF73BFD0A
:104860000EE00C20FDF734FD174B1868FDF758FDDE
:10487000164B1868FDF754FD154B1868FDF750FDF1
:104880000120BDE8F8830020BDE8F8831D08002062
:104890000808002078FA0008541500205C15002054
:1048A000DE02002020050020580500208A05002097
:1048B00086050020C40F002060150020E50F0020B1
:1048C00026100020F8010020E8F7FF1FECF7FF1F7B
:1048D000F0F7FF1FAFF300809248F0B50368924AEB
:1048E0009C8AA4B2E1B211F0010F2ED0198821F4F4
:1048F00000610904090C1980198889B241F48061AA
:10490000198000211170517899B1917811B9D1783D
:10491000FF290ED1012191701179022904D1198842
:1049200089B241F400611980517941F00101198285
:10493000E2E0517901F0FE011982D378FF2B00F0FB
:10494000DB80794BFF211970D6E08E073AD5BFF393
:104950005F8F1479E4B2012C13D1517889B1917829
:1049600079B1198821F480610904090C1980BFF319
:104970005F8F198B1988947189B241F40071198085
:104980001BE0198BBFF35F8F14796749022C0AD1A2
:104990004C7844B1897831B1198821F480610904D7
:1049A000090C1980A2E014795F49032C05D14C78D9
:1049B0001CB18978002940F09980998889B241F426
:1049C000806198E04D0756D50121917151780029F9
:1049D00037D09178002934D01179147802291988B8
:1049E0001DD921F480610904090C19801E8A91687F
:1049F000E5B2F6B264B20E551C88A4B244F4007459
:104A00001C80AB1C1370036801351C8A6DB2E4B2C4
:104A10004C55998889B241F48061998026E089B229
:104A200041F4007119801E8A9568E1B2F6B264B251
:104A30002E551B8A4C1C64B2DBB203312B5511700E
:104A400014E0947838490CB90C7B44B1198889B2C8
:104A500041F40071198013780133137006E01C884B
:104A6000A4B244F480741C8001238B7001680B880D
:104A7000DB05FCD440E001F0400101F0FF05D9B1B5
:104A800011781F8A9668CCB2651C49B2FFB2EDB2AC
:104A90007754157016796DB2E91C8E4205D199884C
:104AA00021F480610904090C99801379AB4223D168
:104AB0001D4B02341C701FE027061DD511784CB227
:104AC000661C0BD0156901312C5DC9B2E4B21C82A1
:104AD0001479117049B28C420ED107E0D17815706B
:104AE000C9B21982517809B9117929B9998821F483
:104AF00080610904090C9980147992F90010621CF4
:104B00009142094B0DD100229A709B7933B1026812
:104B1000938823F440731B041B0C9380034B0022E7
:104B20001A70F0BDD810002030100020DE100020D8
:104B30004B8810B5DC0607D52C4B14791B6853F84D
:104B400024402B4B43F820404B889B0607D5274B2E
:104B500054791B6853F82440254B43F820404B8878
:104B60001C070DD5234B0C781B78B3EB141F07DB08
:104B70001E4BD4781B6853F824401D4B43F820404B
:104B80004B889B070DD51C4B0C781B78B3EB141F7F
:104B900007DC164B54781B6853F82440144B43F839
:104BA00020404B88DC070ED5144B0C781B7804F0A2
:104BB0000F049C4207DC0D4B14781B6853F824400B
:104BC0000B4B43F820404B885B070ED50C4B097804
:104BD0001B7801F00F01994207DB044B92781B68A8
:104BE00053F82220024B43F8202010BD600D002016
:104BF000CC0500205F0600205D0600205C0600203A
:104C00005E0600202DE9F74F9F4F9B463B7D0C46EB
:104C100091465A1C05463A750068224649460C26BC
:104C20005E4301F0DDFBAB686868ADF80430182323
:104C30008DF8063001A902238DF80730FEF796F8AB
:104C40002B7B183707EB060A2C680C2B00F2F2803E
:104C5000DFE813F00D00F000F000F0004D00F00070
:104C6000F000F0008200F000F000F000B600238CAD
:104C7000864823F001031B041B0C2384218CA2888B
:104C8000238B844223F073034FEA03434FEA134319
:104C900089B292B243F0700314D000F500608442F0
:104CA00010D000F5406084420CD000F58060844252
:104CB00008D000F58060844204D021F0020141F068
:104CC000030107E021F00E0122F4407241F00301DC
:104CD00042F48072A2802383A4F834B02184238B11
:104CE00023F008031B041B0C43F0080332E0238C61
:104CF000664823F010031B041B0C2384218CA2881C
:104D0000238B844223F4E6434FEA03434FEA1343E1
:104D100089B292B243F4E04308D000F500608442C7
:104D200004D021F0200141F0300107E021F0E00142
:104D300022F4406241F0300142F48062A280238379
:104D4000A4F838B02184238B23F400631B041B0CCC
:104D500043F4006323836DE0238C4C4823F4807379
:104D60001B041B0C2384218CA288A38B844223F078
:104D700073034FEA03434FEA134389B292B243F0FD
:104D8000700308D000F50060844204D021F4007163
:104D900041F4407107E021F4606122F4405241F493
:104DA000407142F48052A280A383A4F83CB02184D5
:104DB000A38B23F008031B041B0C43F0080338E00B
:104DC000B4F820C0314A2CF4805C4FEA0C4C4FEA16
:104DD0001C4CA4F820C0B4F820C0A388B4F81C80F0
:104DE0002CF4005C28F4E6484FEA08484FEA0C4CE3
:104DF0004FEA18484FEA1C4C94429BB248F4E048F2
:104E00004CF4405C03D002F50062944203D123F4D9
:104E1000804343F48043A380A4F81C80A4F840B0EE
:104E2000A4F820C0A38B23F400631B041B0C43F4E1
:104E30000063A383AB7B43B1B4F844306FEA4343D0
:104E40006FEA53439BB2A4F8443023889BB243F0EB
:104E5000010323802B7B0C2B10D8DFE803F0070F16
:104E60000F0F090F0F0F0B0F0F0F0D00343404E05D
:104E7000383402E03C3400E04034BC515046AAF8DB
:104E8000049003B0BDE8F08F30100020002C0140EA
:104E9000F8B50121044604F089FE01283B4F01D0FA
:104EA000002616E04FF6FE732382A68D0025B6B2CB
:104EB0002046795DFDF726FF354B142202FB0030BA
:104EC000C36813B1007C314698470235082DEFD1F5
:104ED000E6E7BD5D95B92046022104F067FE012892
:104EE00050D14FF6FD73238229462046FDF70AFF75
:104EF000274B142202FB0030A18E3EE0042D12D17C
:104F00002046294604F052FE01283BD14FF6FB73A0
:104F1000238229462046FDF7F5FE1D4B142202FB95
:104F20000030218F29E0082D12D12046294604F0B7
:104F30003DFE012826D14FF6F773238229462046ED
:104F4000FDF7E0FE124B142202FB0030A18F14E0AB
:104F50000C2D17D12046102104F028FE012811D174
:104F60004FF6EF73238229462046FDF7CBFE084B10
:104F7000142202FB0030B4F84010836889B20BB1F0
:104F8000007C98470236082EA3D1F8BD80FB0008AC
:104F9000C40600202DE9F041067B04460F46006858
:104FA000314690461D46FDF7ADFE0F2808D8194B37
:104FB000142202FB0030C0F80880C5600671077437
:104FC000237B22680C2B1CD8DFE803F0071B1B1B7C
:104FD0000C1B1B1B111B1B1B160093899BB243F060
:104FE00002030DE093899BB243F0040308E0938928
:104FF0009BB243F0080303E093899BB243F0100394
:10500000938125B193899BB243F001039381BDE85D
:10501000F08100BFC4060020234B70B519684FF41F
:105020007A73B1FBF3F1214B21481A78214B224DC1
:105030001B7804F075FC214B21481968214B2E6820
:10504000B1FBF3F104F06CFC00241F4BE2B253F807
:10505000221049B1012303FA02F2324202D01B4866
:1050600004F05EFC0134F0E72A6892070DD5184A77
:105070001848127803EB8203196A04F051FC164BAE
:10508000197A11B1154804F04BFC1548FDF786F963
:10509000BDE87040134B14481A88144B92B219881B
:1050A00040F2A45304F03CBC081700201405002073
:1050B000C90A01087400002068020020780000205E
:1050C000070B010840420F0088FB0008250B010870
:1050D000DD1C0020290B01086C020020330B0108A5
:1050E0000E0D0108E00F0020370B010824030020FB
:1050F00008B540F2E9330D4A1189890709D5908135
:1051000040F2E933094A1189C9070AD59089C0B22A
:1051100008BD013B9BB2002BEDD1FDF760FEFF20E7
:1051200008BD013B9BB2002BECD1F6E700300140FB
:105130002DE9F04F964D89B02B689A8A92B202926F
:10514000029A12F4706F1CBF01222A71029A12F4A3
:10515000E06F00F011811A8B9A8822F480621204A9
:10516000120C9A80029A960500F106811A8894051D
:1051700000F102811A88D00540F1F3801A88D10528
:10518000FCD41A8892B242F400721A801A889205EE
:10519000FCD495F805807F4B1421B8F1010F28BF8E
:1051A0004FF0010801FB08327B4F906DFC69B2F8AB
:1051B0005060B2F852A0D2F848B02043D46C4AEA0A
:1051C00006090222C5F800B085F80580F861C4F828
:1051D000109020468DF80E1003A98DF80F20ADF821
:1051E0000C900093FDF7C2FD08220192A2681642BE
:1051F00003D10A20FCF796FFF8E70A206661FCF766
:1052000091FF26610A20FCF78DFF019B013B019372
:10521000ECD10A20C4F814A0FCF784FF0A206661D0
:10522000FCF780FF0A202661FCF77CFF0222C4F80D
:1052300010A020468DF80F2003A91C228DF80E2007
:10524000ADF80C90FDF792FD544A93453A6905D1AB
:1052500042F400123A614FF4001004E042F480027C
:105260003A614FF4800004F07FFEBBF8042003A8ED
:1052700022F440721204120CABF80420BBF8002098
:10528000142792B242F00102ABF80020BBF80440B0
:1052900004F0BAFD24F03F04059841492404B0FB12
:1052A000F1F1240C0C43A4B2ABF80440BBF800208D
:1052B000002422F001021204120CABF80020394A3B
:1052C0000126B0FBF2F24FF49670414392B24FF4D4
:1052D0007A70002A91FBF0F108BF0122013142F4FB
:1052E000004289B2ABF82010ABF81C20BBF80020BC
:1052F00003A892B242F00102ABF80020BBF80020F4
:1053000022F4816222F002021204120CABF8002097
:105310004FF48042ABF808201E4A8DF80D4007FB81
:10532000082898F855308DF80E408DF80C308DF81F
:105330000F60FCF78FFC98F854309DF80F208DF823
:105340000C308DF80D401AB103A8FCF783FC13E074
:10535000590903F01F039E40134A203142F821608F
:105360000AE01A8892B242F400721A809A8822F4F3
:1053700040721204120C9A802A68938A23F4706394
:105380001B041B0C93820023AB7109B0BDE8F08FA6
:10539000D810002088FB0008001002400054004094
:1053A00040420F00804F120000E100E03F4A2DE92B
:1053B000F84F916840F201130B4040F201118B420B
:1053C00093460AD13A4BDA7993F808901A72B9EBFE
:1053D000020918BF4FF0010901E04FF001094FF039
:1053E0000008344B5FFA88F41B78A3425CD9324B37
:1053F000324E1B68324F23B93B685B8926F8143064
:105400004FE03A68072C94BF12F804A0A24629483E
:1054100051469847DBF808300546DB0509D5B9F158
:10542000000F06D0274B50461B6829461B68DB69D6
:105430009847A5F2EE2240F2DC5392B29A4288BF1E
:105440003B68DBF8082088BF5D8942F20103134006
:105450002BB31D4B1978164B01F0030202EB8402AB
:1054600093F86A0003EB420255811A4620B90329DA
:1054700015D9012183F86A1002EBC40399895D896B
:1054800002EB44020D44D9891B8A0D441D44ADB280
:10549000A2F86C5004232DB295FBF3F5ADB226F8BB
:1054A000145008F101089CE7BDE8F88F0C170020A4
:1054B000D8100020F3090020FC090020BA040020C5
:1054C000F4000020E801002070150020094B30B5E1
:1054D0009D68094B05F480551868084B1C6800232B
:1054E0000DB1828800E0A28805495A520233182B78
:1054F000F6D130BD0C170020E0040020A4040020E9
:10550000E404002010B5144B07229B894FF47A73F2
:10551000013A1FD010490C89A40706D5FF248C81BD
:105520000D490C89E4070FD507E0591E89B213B95C
:10553000FDF755FC0EE00B46ECE7898989B200289F
:10554000E6D001700130E3E7591E89B2002BEFD09D
:105550000B46E5E7012010BD0030014013B50122E4
:1055600004464FF6FF71006800F03AFF236801A877
:105570001A8892B242F001021A80637B8DF80430DF
:1055800001238DF805308DF806308DF80730FCF7D3
:1055900061FB02B010BD2DE9F04F684CD4F88430A7
:1055A0006749581C0A78894602F0FF0C0AB1034685
:1055B000F6E794F88C7094F88D6094F88E50D4F8D7
:1055C0009010C4F88430E0461FFA88F213B21F2B03
:1055D00000F393805B4901EB8300C278807831F857
:1055E0002310C0F1FF0080B2002861D0C0F1FF009D
:1055F00050433C23B1FBF3FA0012BAF1050F5AD81D
:10560000DFE80AF0030B1A283846161A4E43C5B2D3
:10561000B6FBF3F62E44F6B248E0B1FBF3F703FB1A
:105620001717BFB2C5B2C7F13C07101A4743B7FB03
:10563000F3F72F44164629E0B1FBF3F503FB1515EC
:10564000C7B2ADB2101A4543B5FBF3F53D44EDB218
:10565000164630E0B1FBF3F603FB1616B6B2C7B23E
:10566000C6F13C06101A4643B6FBF3F63E44154617
:10567000F6B220E0B1FBF3F703FB1717C6B2BFB2D7
:10568000101A4743B7FBF3F737441546FFB212E051
:10569000B1FBF3F503FB1515ADB2C6B2C5F13C0580
:1056A000101A4543B5FBF3F53544EDB2174602E059
:1056B0001546164617464FEA072A4AEA064A4AEAB4
:1056C000050A1723012199400CF1170211EA0A0F6C
:1056D000C3EB02021C490CBF0920112092B213F146
:1056E000FF338854EED20CF1180C08F101081FFAB0
:1056F0008CFC1FFA88F8154966E7012389F8003009
:10570000134BA4F88A2040F22A3284F88C7084F873
:105710008D6084F88E50C4F89010A4F888C05A6048
:105720000C4A00219184118889B241F00101118055
:105730001A6842F001021A60BDE8F08FD81000200C
:10574000DA1C0020CC050020340A0020641100205F
:105750006C00024000040040826A8169436B11447E
:10576000D960416A914203D98A1A5A60816204E081
:1057700001698A1A5A6000228262002280F844205D
:105780001A6842F001021A60704738B5134B144D85
:105790001A78144C2968A2B1D4F89420024491429A
:1057A0001BD300201870FCF7D2FC2B68C4F894308F
:1057B0000D4B1A780AB1013A1A70012384F8983017
:1057C00038BDD4F89420C832914206D30120187015
:1057D000FCF7BDFC2B68C4F8943038BD4B15002095
:1057E00008170020D8100020AE02002037B5264D43
:1057F0008DF8073095F899308DF8062002AA8DF8BB
:1058000004008DF805101A4412F8042C443AD2B260
:105810000F2A32D81D49022B01EB4202B2F8704028
:1058200003D814B12046FFF7B0FF95F89930164A17
:10583000022B0BD9164B1968D2F89430091B8B42F6
:1058400004D2002382F89930124A137095F89830E8
:10585000012B00D0B4B995F89930022B03D80A4A2D
:10586000013382F899300C4B002085F898001870AD
:1058700003B0BDE83040FCF76ABC022B4FF0C8040F
:10588000D0D9D2E703B030BDD810002088FB000883
:1058900008170020AE0200204B1500200449054BDC
:1058A0000968002218701A6159611A76704700BFA2
:1058B00008170020100A0020024B03481968034A09
:1058C00004F02EB87C000020C50B0108EF0B010886
:1058D00038B5054607F04AFFC0B270B90446134B0D
:1058E00004F120021B682146114853F8222001349C
:1058F00004F016F8152CF2D138BD284607F08BFFBE
:10590000142804460BDC2021284607F022FF07F06C
:1059100082FF064B20341B6843F8240038BD05483D
:105920001521BDE8384003F0FBBF00BFF80100209F
:10593000F70B0108030C01080EB40FB5074906ABBD
:105940000190074A01A8039303F024FF019B002262
:105950001A7004B05DF804EB03B070471D1900081D
:10596000290C01082DE9F0438DB0054607F0FEFE35
:10597000C0B2002858D104467F4B00211E68142273
:1059800007A807F0B2FEA500002303A905A803930A
:10599000059377190B7183801A46DFF8F0E1B7F8A9
:1059A00002C03EF8138018EA0C0F0CD00EF10A0E5C
:1059B0000DF1300813F80EE002F1010C424402F838
:1059C00024EC5FFA8CF20133052BE6D100231A4652
:1059D000DFF8C0E1B7F802C013F80E8018EA0C0F28
:1059E0000CD00EF1060E0DF1300813F80EE002F1A6
:1059F000010C424402F81CEC5FFA8CF20133062BD6
:105A0000E6D1735D8DE803001A0907A85B4903F02E
:105A10000F03FFF791FF2146594807AA013403F00D
:105A20007FFF202CA8D1A3E0284607F0F4FE1F2812
:105A3000044600F3918028462021E4B207F089FE55
:105A40001F2C01D94F4888E04B4B471C1B68002195
:105A500003EB84042046042207F047FE00254A4B4E
:105A600007AE304600210A2215F803905FFA85F848
:105A700007F03BFE0023FA5CF91832B10A2B04D080
:105A80004A4502D0F2540133F5E74A4501F10107D6
:105A900067D1B8F1020F0DD0B8F1030F0CD0B8F1F7
:105AA000010F0BD0304607F0B6FE2378C0B243EAB0
:105AB00000100AE0002219E0002226E0304607F03C
:105AC000AAFE237800F00F001843207038E001335D
:105AD000062B0AD02D4800F115069E5D8E42F6D1A8
:105AE0000344D97B63880B43638001320CA9D3B292
:105AF0000B4413F8141C19B30023EBE7412B1DD002
:105B0000542B08BF04230ED00132D3B20DF130085C
:105B1000434413F8143C9BB1492B01D1002302E00C
:105B2000572B07D10123194931F8131063880B4310
:105B30006380E9E7462BE1D10223F4E70323F2E790
:105B40000135042D8BD10124FCF7B2FFFCF7EEFFE9
:105B5000FCF7C6FF64B975E70D48202103F0E0FEAD
:105B600006E020460021042207F0BFFD0024EBE7F9
:105B70000DB0BDE8F08300BFC8050020290C010866
:105B8000350C0108410C010833FC000818FC000822
:105B90004F0C010827FC000810B50748FCF7FEFB76
:105BA0000024064B0648E218E15852680C3403F012
:105BB000B7FEE42CF5D110BD710C01088CFC000877
:105BC000870C0108F8B5074607F0D0FD044638B940
:105BD0001A4B1B485A791B4B013A53F8221028E004
:105BE00038461949224607F0C9FD60B91748FCF745
:105BF000D5FB174C54F8041F19B1164803F090FE5A
:105C0000F8E7154805E000250E4B53F8256026B946
:105C10001248BDE8F840FCF7C1BB38463146224681
:105C200007F0ACFD01350028EED1044B0C485D7146
:105C30003146BDE8F84003F073BE00BF0C170020EA
:105C40008F0C010870FD00088F110108A30C0108DA
:105C50006CFD0008250B01080E0D0108B60C0108AB
:105C6000CB0C010837B502790D461106044683684E
:105C700006D526494FF49A7091F8A01500FB013320
:105C800002F03F02042A12D006D8012A0DD0022ABF
:105C90002FD193F900102DE0102A0AD0202A0AD023
:105CA000082A26D1B3F9001024E0197822E01988D7
:105CB00020E019681EE06946186803F00DFF0146F0
:105CC000134803F02DFEF5B1E06804F097FF694634
:105CD00003F002FF01460F4803F022FE206904F0A2
:105CE0008DFF694603F0F8FE01460A4803F018FEEE
:105CF00009E00021084803F013FE25B10748E168D8
:105D0000226903F00DFE03B030BD00BF0C17002068
:105D1000300B01082F0B0108E10C0108DD0C010814
:105D20002DE9F041002407462546114B3946E65837
:105D300004EB0308304607F055FD58B10D483146D5
:105D400003F0EEFD40460021FFF78CFF0A4803F008
:105D5000E7FD0135143440F63C239C42E5D125B9DA
:105D60000648BDE8F041FCF719BBBDE8F08100BF73
:105D700018FE0008570F01080E0D0108E40C010879
:105D80002DE9F74F044607F0F1FC054620B1012844
:105D900019D123782A2B16D15248FCF7FFFA002498
:105DA000514B5248E618E15803F0BAFD30462946F7
:105DB000FFF758FF4E48FCF7F1FA143440F63C2345
:105DC0009C42EDD18AE020463D2107F0C2FC00282C
:105DD0007FD0034613F8012C202A01D1013BF9E7BB
:105DE000451C2846C4EB030A07F015FD83462846E8
:105DF000FCF7FAFC0026054614237343DFF8E8900D
:105E000053F8097003EB0908384607F0AFFC034666
:105E10001A4620463946019307F0B0FC019B002842
:105E20004ED15FFA8AF29A424AD1D8F80C0004F0B7
:105E3000E5FE0146284605F0E7F800283ED0D8F8F0
:105E4000100004F0DBFE0146284605F0D3F80028D8
:105E500034D098F804309C064FF0140303FB0696E8
:105E6000327958BF5D4610062946B36806D52148E9
:105E70004FF49A7490F8A00504FB003302F03F023F
:105E8000042A0BD004D8013A012A0CD819700AE070
:105E9000102A05D0202A05D0082A04D1198002E052
:105EA000196000E01D603946134803F039FD3046A3
:105EB000002103B0BDE8F04FFFF7D4BE0F4803E068
:105EC0000136832E98D10E4803B0BDE8F04FFCF7A1
:105ED00065BA204603B0BDE8F04F21E703B0BDE846
:105EE000F08F00BFFC0C010818FE0008570F0108D6
:105EF0000E0D01080C170020110D01081C0D0108E2
:105F0000E40C01082DE9F04389B0044607F02EFCAB
:105F1000C6B2002E6CD18B48FCF740FA8A4C20693F
:105F2000002105F053F840BB01368848314603F0A4
:105F3000F7FC206904A903F0CFFD0146844803F073
:105F4000EFFC606904A903F0C7FD0146804803F037
:105F5000E7FCA06904A903F0BFFD01467C4803F0FB
:105F6000DFFCE06904A903F0B7FD0146794803F0BE
:105F7000D7FC0C2E04F11004D1D10025764C2F460D
:105F80002B464FF00008B04504F1100415DA18460E
:105F900054F8101C04F07EFD54F80C1C8146284671
:105FA00004F078FD54F8081C0546384604F072FDEC
:105FB00008F101084B460746E5E76848019302955A
:105FC0000397FCF7EBF9002401ABE058644920F09B
:105FD000004005F023F8634B634A0434002814BFE3
:105FE00010461846FCF7DAF90C2CEDD15F4891E029
:105FF00020465F49052207F0C1FB38B9524B002209
:1060000003441030C0281A61F8D197E0204659495E
:10601000042207F0B3FB06462046002E40D1202183
:1060200007F097FB002800F08980451C284607F000
:106030009DFB34468046504B53F824600EB94F48C0
:1060400068E0284631465FFA88F207F097FB671C44
:1060500020BB3D4B0021C2181030C02811619C4666
:10606000F7D1474B002403EBC702D2F804E098466F
:10607000BEF1000F04D14348314603F051FC55E016
:1060800018F837309C42F6DA23010CEB0305103583
:1060900073440FCB013485E80F00F1E73C46CAE7B3
:1060A00007F0B9FB461E0B2E074643DC2046202195
:1060B00007F04FFB054640B1451C2846FCF794FB12
:1060C000214B3F01D851012400E0044628462021FD
:1060D00007F03FFB054640B1451C2846FCF784FB12
:1060E000194B013403EB061358612846202107F0B1
:1060F00030FB054640B1451C2846FCF775FB124BAA
:10610000013403EB061398612846202107F021FB98
:1061100018B91D48FCF742F910E00130FCF764FBA8
:10612000094B032C03EB0616F061F2D11748FFF779
:10613000E9FE03E016480C2103F0F2FB09B0BDE8CC
:10614000F08300BF440D01080C1700206F0D0108FB
:10615000750D01088A0C010820170020790D01082F
:106160000AD7233C400D01083C0D01080E0D010823
:10617000880D01088E0D010870FD0008B60C01089D
:10618000CCF20008930D0108A30D0108F60F0108D9
:10619000DD0D01087FB5044607F0E8FA082824D190
:1061A00000231F49E25C09681144497801F00301AA
:1061B000022908BF203AE2540133082BF1D100250F
:1061C000665D1848314607F0C4FA28B101356019F8
:1061D000314607F0BEFA18B11348FCF7DFF81CE0AF
:1061E000082DEDD1204603F039FC1048FCF7D6F815
:1061F00000230F4A04A91A4492F80E210A440949BF
:10620000595C0133082B02F80C1CF2D10023094819
:1062100001A98DF80C3003F083FB04B070BD00BF02
:106220008000002049140108050E0108250E010810
:106230000C1700208A0C01082DE9F047054607F0ED
:1062400095FA304B0446D3F808809A4690B92E4808
:10625000FCF7A4F82D4B53F8241049B10123A340B7
:1062600013EA080F02D02A4803F05AFB0134F1E781
:10627000284821E028462849224607F07FFA58B9E5
:106280002648FCF78BF8264C54F8041F0029EFD061
:106290001F4803F045FBF7E72B7800262D2B03BFA3
:1062A000013504F1FF344FF001094FF00009174B9D
:1062B00053F8267027B91B48BDE8F047FCF76EB8C5
:1062C00028463946224607F059FAC8B90120B0409D
:1062D000830501D51448EFE7B9F1000F03D0FCF7AF
:1062E000A1FB124804E040EA0800CAF80800104880
:1062F000FCF754F839460F48BDE8F04703F010BBEF
:106300000136D4E70C1700203A0E0108CCFD000836
:10631000250B01080E0D01088F1101084D0E010813
:10632000C8FD0008620E0108790E01088D0E0108F3
:10633000970E01088A0C010870B5044607F016FA9A
:1063400008B9204830E020461F4907F089FA0024A8
:106350002646254678B12CB1012C06D107F05BFA10
:10636000064602E007F057FA0546174900200134B7
:1063700007F076FAEEE70B2D05D9BDE8704013481B
:106380000C2103F0CDBA012C08DC114B294633F95E
:1063900015201048BDE8704003F0C2BAA6F57A7324
:1063A000B3F57A7F04D90C48BDE8704003F0B8BA61
:1063B0000A482946324603F0B3FA054B23F8156024
:1063C00070BD00BFA00E0108C50F0108DA0E01085C
:1063D000E4040020000F0108180F01083A0F01081B
:1063E000254B10B55343254A254C12680139B2FBA1
:1063F000F3F20388013AA04289B292B29BB212D062
:1064000004F50064A0420ED0B0F1804F0BD0A4F58B
:106410009834A04207D004F58064A04203D004F56C
:106420008064A04202D123F070039BB2154CA042BD
:1064300006D004F58064A0421CBF23F440739BB2D5
:1064400003800F4B8185984202850FD003F50063CE
:1064500098420BD003F54063984207D003F5806360
:10646000984203D003F58063984201D1002303864C
:106470000123838210BD00BF40420F00780000203E
:10648000002C014000100040284BF0B51D68002290
:106490002748165C1418AB19597801F0040101F073
:1064A000FF0371B10132102AF2D10020F0BD1BB1FF
:1064B00003EB83035B00DBB210F8012B303A13448B
:1064C000DBB2221A022AF2DC002184420AD919B175
:1064D00001EB81014900C9B210F8012B303A114497
:1064E000C9B2F2E72E2E14D1601C002204240678D3
:1064F00002EB8202AF197F7852007F0792B203D578
:10650000303A3244013092B2013C14F0FF04EED133
:1065100000E00022074806244143642000FB0212E9
:106520000548B2FBF4F200FB0320F0BD8000002020
:10653000030E002040420F008096980030B50022E4
:1065400013460D495C5C9CB12E2C04D1013378B10B
:106550001C1800250D550A246243C95CA1F13004C2
:10656000092C9CBF303A52180E2B03D80133E8E7B0
:10657000104630BD002030BD030E002070B5064629
:1065800000240B4BE5182A7916420AD0E158094835
:1065900003F0C6F928460021FFF764FB0648FBF725
:1065A000FDFE143440F63C239C42EAD170BD00BF8E
:1065B00018FE0008530F01080E0D0108A14B2DE92C
:1065C000F04F1B7885B0013B012B00F237819E4BC9
:1065D0001D78854240F032819C4B1B78022B00F0E5
:1065E0002D819B4E002333809A4B13F805B09A4BB4
:1065F00083F800B0994B1A7803921AB1984B33F98B
:10660000150008E0974B1A6802F100421A60944A9C
:1066100032F91500404204F0F1FA934904F0F6FB18
:106620009149044604F03EFB04F002FD8D4F8E4973
:10663000D7F800A01FFA80F85046A6F8028004F0B0
:1066400031FB04F0F5FCDFF84092B080D9F800206F
:1066500000211046029204F0B9FC0027834B029AF5
:10666000002857D01A68204611460292019304F080
:10667000D5FC029A019B38B11C607D4BC3F800A089
:10668000734BA3F80680BFE01046394604F0C6FC01
:10669000002800F0B980774B1A789846002A31D14B
:1066A0002046514604F0F4F94FF07E5104F098FC76
:1066B000714C28B16068714904F0F4FA60600FE031
:1066C0006F49606804F0EEFADFF8D09182464946DF
:1066D00004F086FC10B9C4F804A001E0C4F80490EA
:1066E000012388F80030674B00221B685B449A72D4
:1066F000039A82F00103594A1370634B1F605B4B8E
:106700001F6081E0614BC9F800401A68584BFA32AB
:106710005A6079E020461146019304F061FC019B28
:1067200020B1594A14604A4AA2F80680D3F8008082
:10673000554B4046D3F80090494604F0A9F9534B15
:10674000824619684A4B5A688A1A002A0BDA4FF0B7
:106750007E5104F063FC002856D02046494604F0E0
:106760005DFC002850D0424A4046116804F056FCB7
:10677000414C48B1012320684149338004F092FA2A
:106780003E492060A06809E0022350464FF0804156
:10679000338004F043FC28B1A068394904F082FA40
:1067A000A06004E02068354904F07CFA2060354B95
:1067B0002D492068D3F8008004F074FA04F05EFCE0
:1067C00008F80B00A06804F059FC039AD84482F042
:1067D0000103224A88F8140013702B4B1F60234BCF
:1067E0001F60244B1A780132D2B2032A01D01A70EA
:1067F0000AE000221A70204B2549586804F052FA2A
:1068000004F03CFC88F80A0015B9338864333380FF
:10681000124A13780BB11F4B00E01F4B114A136053
:106820000F4B33F9150004F0E9F90F4904F0EEFAC3
:106830000C4A0146106804F02BF900E0084605B048
:10684000BDE8F08F4403002098030020A803002037
:106850002610002020F20008A90300209903002040
:10686000E80200204803002000002041A00300208F
:10687000741100209A030020AC0300200AD7833F44
:10688000EC51783FA40300209C030020081700204F
:1068900000007A440000A0410000A0C16F12833ABA
:1068A00010B50848FBF77AFD074B1C682046FBF73C
:1068B000BAFC18B90A20FBF740FCF7E7034A044B7F
:1068C000DA6010BD620F0108B80800200400FA0564
:1068D00000ED00E008B50448FBF760FD02F0D2FDD2
:1068E000BDE80840FFF7DCBF6E0F010810B5044695
:1068F0000748FBF753FD074A002313729363064AC8
:106900001370FEF7E3FD2046BDE81040E2E700BF4C
:10691000750F010874110020DB1C00202DE9F04FD9
:10692000002485B007460191924602938046254691
:10693000022DDFF878914FEA450607D1019AB9F99F
:10694000040053791B3343435B1148E04C4B39F946
:10695000151033F9153003EB4101CAF100039942D8
:1069600003DB5145B4BF0B4653464649029A31F901
:1069700006B0915FCBEB030303EB010BFBF7DFFEEC
:1069800098B1414B58465B5D009304F037F93F499D
:1069900004F03CFA009B01461846FFF70FFE3B4906
:1069A00004F080F904F044FB8346394B1988C8078A
:1069B00011D4019A39F9060013798A0703F11B03F0
:1069C00000FB03F34FEA231309D57A7C02FB0BFB90
:1069D00003EB2B2303E0FB7903FB0BF31B112D4A85
:1069E00098F80AB0905F042290FBF2F0181A7B5DD1
:1069F000294A43430393294BA158B3F800C00135FA
:106A00000CFB00F3DB120BFB03132549B3F5001F4E
:106A1000A8BF4FF400138B42B8BF0B462149A350C7
:106A200062584FEA1C1C6050821A4FF6FF70B0FB90
:106A3000FCFC0CFB02F201F10C0C183154F80CB008
:106A4000605892115844104444F80C2098F81420CF
:106A5000032D02FB00F0039A4FEA202000EBE21026
:106A6000114A00EB633344F801B0935308F1010875
:106A700004F104047FF45CAF05B0BDE8F08F00BF03
:106A8000D01C0020E802002038FC00080000204153
:106A9000420300201C0300200C16002024030020C9
:106AA0000000E0FFB0110020D4030020BA03002052
:106AB0002DE9F04F87B005938E4B0492B3F9022075
:106AC000B3F90030002AB8BF5242002BB8BF5B4276
:106AD00000249A42B8BF1A46019003922646A14666
:106AE00027460294A0462546DFF83CA2BAF80030BB
:106AF00099075AD0022D58D07E4BDDF810C0F25EB7
:106B00007D4BF35E03EB4202CCF100039A4203DBC0
:106B100063469A42B8BF1346784ADDF814C036F986
:106B200002B03CF90620CBEB030303EB020BFBF7AF
:106B300006FE90B1724B584615F8038004F05EF8DB
:106B4000704904F063F901464046FFF737FD6D498F
:106B500004F0A8F804F06CFA834601996423CA791A
:106B600002FB0BF292FBF3F2CB7E6FF0040101FB10
:106B700003F8424505DB03EB83039A42B4BF90461A
:106B80009846614A42F21071A3585B448B42A8BFF9
:106B90000B465E498B42B8BF0B46A350019A92F850
:106BA00011B00BFB03F31B130293BAF8003003F090
:106BB0000302012A01D1022D3DD101994D4A11F85C
:106BC00005C05349B75E895F524A81EAE170A0EB84
:106BD000E170B0F5206F54F802901DDC022D15D045
:106BE0005020784390FBFCFC042091FBF0F1C1EBBA
:106BF0000C0CE1444848B9F57A5FA8BF4FF47A59C4
:106C00008145ACBF42F80490105107E087EAE77075
:106C1000A0EBE7706428E3DD002111513D4AA15843
:106C20007D2291FBF2F9019A2A44927A02FB09F93A
:106C3000402299FBF2F99A0716D5022D14D0039A37
:106C4000DDF80CC0C2F5FA730CFB09F07A43DDF8ED
:106C500008C003FB082203FB0C034FF4FA7192FBFC
:106C6000F1F293FBF1F308E0DB0701D5022D02D12D
:106C70004B463A4601E0029B42462549DFF8ACB05C
:106C8000715A04200FFA81FC15F80BB09CFBF0FA46
:106C90000BFB0AFB6FF04F0A9BFBFAFB93441F4A66
:106CA00036F902A0B152CAEB0C0C9CFBF0F002F1D9
:106CB000080102F1140A54F801C054F80A20605087
:106CC00017496244695C02444A43202192FBF1F275
:106CD0009A1A144801359344032D44F80AC026F843
:106CE00000B004F1040406F102067FF4FDAE07B023
:106CF000BDE8F08FBA030020D01C0020E80200207D
:106D000038FC0008000020418C150020F0D8FFFF5F
:106D10001C0300200C16002080C1FFFFD4110020AE
:106D200014150020D4030020420300200E1500207B
:106D30002DE9F04F89B007937A4B8146188804916A
:106D4000059203F057FF784903F0ACFF002403904D
:106D50004F4625462646022EDFF80CA20BD1049999
:106D6000BAF904004B790A33584303F047FF6F49DF
:106D700004F04CF844E06E4B3AF90520EB5E0599BF
:106D80001A444B429A4203DB0B469A42B8BF134661
:106D9000684AAA5E9B1A079A505F184403F02EFFB8
:106DA000654904F033F88046FBF7C9FC28B1634B12
:106DB0004146985DFFF702FC8046614B1A88D10777
:106DC00005D54046D9F8441003F06CFF18E004994B
:106DD0003AF905000B7901921433584303F00EFF82
:106DE000524904F013F8019A8346930709D5D9F85C
:106DF0004810404603F056FF0146584603F04AFE4D
:106E00008346504A505F03F0F9FE4F4AD16803F0C1
:106E100049FF82465146584603F03AFE396A804699
:106E200003F040FFDFF844B106900399404603F0B9
:106E300039FFF96A03F036FF54F80B1003F02AFE0D
:106E40004249804604F0CCF838B94046404904F045
:106E5000E5F820B1DFF8F88001E0DFF8F0804BF8CA
:106E60000480DFF80CB1504654F80B1003F010FE0C
:106E700044F80BA0034603994FF07E50029303F0B1
:106E8000C5FF029B0146184603F00CFF0BF10C03F3
:106E9000E2580BF1180B54F80B1082461046019281
:106EA000029303F0F7FD514603F0F4FD019A029BB3
:106EB00044F80B2044F803A0264903F0A7FFB96B60
:106EC00003F0F0FE2449824604F08AF838B95046AF
:106ED000224904F0A3F820B1DFF880A001E0DFF838
:106EE00078A00698414603F0D5FD514603F0D0FD49
:106EF00006F060FE1A4BB0F57A7FA8BF4FF47A70A7
:106F00009842B8BF18460136164B032EE85204F1DA
:106F1000040405F1020507F104077FF41CAF09B072
:106F2000BDE8F08F24030020BD37863500004842BD
:106F3000D01C0020E80200200000204138FC00089E
:106F4000420300201C030020FC01002000007AC343
:106F500000007A4300004040000096C300009643C2
:106F600018FCFFFFD4030020BA03002018160020ED
:106F7000F41100202DE9F047704B86B01A7899463D
:106F8000DFF8C88192B90123D8F80000022189F8FE
:106F9000003002F045FAD8F80030694A6948C2F872
:106FA000A430FBF7FBF96848FBF7F8F9D8F80000C4
:106FB000FBF748F9002800F0BE80644B604C18686D
:106FC000FBF73BF90928014601D03F284FD14FF08C
:106FD000000AA56B5E4F56462DB15E4839682A46B9
:106FE00006F0CCFB10B9BA4606B93E465A4B0C37F0
:106FF0009F42F1D3CEB13768DAF800E02B46F85C57
:107000001EF80310814201D0A3630EE05A1C41B95F
:107010002D2B06D8A263234420202244187211721B
:1070200003E04C4958541346E9E7A36B0BB15645AE
:1070300012D04A48FBF7B2F9564509D856F80C0B5E
:10704000FBF7ACF9D8F800000921FBF70DF9F3E7DD
:107050003D48FBF7A3F90025A36B9D42A6D23D4B0B
:10706000D8F80000595DFBF7FFF80135F4E7A36B92
:1070700033B904283BD104F10800FFF737FC5AE08C
:107080000C2801D136488CE70A2901D00D2949D1B5
:107090003448FBF783F9A36BE21800231372227ABA
:1070A000232A17D00493304B2A4E009303A8284973
:1070B00013220C23039606F0B2FB054638B1006894
:1070C00006F054FB0130AB683044984702E0274893
:1070D000FBF764F91F480021302206F006FB00236D
:1070E000A36399F80030002B7FF45DAF23E00C28F8
:1070F000C8D07F2903D159E72F2B3FF657AFA1F115
:107100002002D2B25E2A3FF651AF13B920293FF4D4
:107110004DAF5A1CA263D8F800001C442172FBF743
:10712000A3F843E77F29E7D1013BA363002223446F
:107130001A720F4838E706B0BDE8F087DB1C002064
:10714000741100208A0F0108C20F0108B80800203E
:107150008CFC00087C11002070FD0008C70F01089E
:10716000CC0F01080E0D0108E71A0008D70F01081F
:10717000F30F01082DE9F74FBF4AC04C1068516862
:107180006B4603C3DFF82C83002140F2A452204653
:1071900006F0ABFA04F50173C8F800304F232370F2
:1071A0000323637140F24C420223A360A4F81A2126
:1071B0004FF4167340F26C72A4F8F030A4F81C215E
:1071C000FA231922A4F8F23084F823212A2340F26A
:1071D0007E42A4F8EE30A4F8D0204FF4FA7340F2C7
:1071E0003A72A4F8F630A4F8D22020234FF47A7231
:1071F00084F8F430A4F8D4206E2340F27E5284F850
:107200000431A4F8D6202B2340F2EA524FF0320981
:1072100084F80531A4F8D820212340F2B452012685
:1072200084F8063140F2DC5B4FF4C873A4F8DA202E
:10723000A4F8DC9084F8EC60A4F8083184F82261AA
:1072400084F82561A4F8DE30A4F818B1A4F8E09021
:1072500002F031F840F6AC53A381D8F80030002595
:107260001E21A573D97399730B211972142117224A
:107270005972197550211A765A76997755226421D8
:107280009A71D9772D22082078211A74D8745A77E8
:107290005973DA75DFF820E2794A7A490E202827F7
:1072A00098724FF00A0A5A20D87283F82160C3F806
:1072B00024E01D701F715F719D7683F807905D74E7
:1072C000DD769D741D7783F815A01F731A63D9634B
:1072D00019644FF08241D9624FF07C5199636A4939
:1072E0005A631A67694A59646949C3F828E083F800
:1072F0005000DFF8C8E141205A67664A996483F874
:10730000510059660420152183F860009A6783F8BC
:107310007C60C3F84CE083F8545083F8555083F8F0
:107320005650A3F858B083F8529083F85350A3F8FE
:107330005C50A3F85E50A3F85A5083F8687083F845
:10734000697083F86C10544802F088FBD8F800305C
:107350004FF44872A3F8D820C82283F81D214FF4B7
:107360009662A3F81E2140F2D932A3F8202140F6FC
:10737000430283F8D760A3F8222183F8D45083F81E
:10738000D55083F8D67083F8DA5083F81CA11A46DA
:1073900046464FF47F71A2F8DC104FF4FA61A2F870
:1073A000DE1040F2DC51A2F8E0101DF805100135A6
:1073B00082F8E210082D4FF0FF0182F8E31002F18D
:1073C0000802E6D1012283F8242183F8252183F8DD
:1073D0002621C82183F82C216422A3F82811A3F8C0
:1073E0002E2114214FF4967283F82A11A3F830212C
:1073F0001E21282283F82B11A3F832210023E21842
:1074000010330021C02B1161F9D124480021402202
:1074100006F06BF900232249E21859580433086832
:10742000382BC2F8C401F6D11E480021802206F094
:107430005CF91D4B1B4C03F1300518685968224656
:1074400003C20833AB421446F7D1FBF731FBFBF71D
:107450006DFBFBF745FB34684FF49A7221461348E5
:1074600006F03AF9124821464FF49A7203B0BDE88B
:10747000F04F06F031B900BF3AFC00080C170020AD
:107480009A99193F8FC2753DCDCC4C3DF6287C3F73
:107490000000A0403D0A773FF70F0108D0180020F8
:1074A00078F200085018002042FC0008441A00201E
:1074B000781B0020F8010020000020400000404020
:1074C00008B50548FAF76AFFFFF754FE01F0DAFF46
:1074D000BDE80840FFF7E4B9001001082DE9F041CC
:1074E0008CB01E469DF848308846012B17469A4BB3
:1074F00006D198425CD10422A3F530531A6101E011
:10750000984255D19548964B87600360954BB507D7
:10751000436103F5807383614FF48073C36003613B
:107520008D4B036503F104038364C36403F548438F
:1075300003F154030363A3F11403D3F8D42F43637B
:1075400042F48042C3F8D42FD3F8D02F42F0010286
:10755000C3F8D02F4FF002038DF803304FF40073BF
:10756000ADF800304FF018038DF8023003D57E4897
:107570006946FBF7FBFB4FF48063ADF80030F4077E
:107580004FF048038DF8023003D577486946FBF782
:10759000EDFB0E238DF8043001A801238DF8053092
:1075A0008DF806308DF807306C4CFAF753FB4EE03F
:1075B0006E4B984240F0CB806D4C694BA7602360C6
:1075C0006C4B206563618033A3618023E3604023BB
:1075D0002361694BB007A364E36403F5E33303F568
:1075E000FE73DA6942F48022DA619A6942F0080295
:1075F0009A614FF002038DF803304FF48063ADF8C9
:1076000000304FF018038DF8023003D55B4869460F
:10761000FBF7ACFB4FF40063ADF80030F1074FF01F
:1076200048038DF8023003D554486946FBF79EFBAA
:1076300027238DF804300222012301A88DF805309C
:107640008DF806208DF80730FAF704FB484C00252A
:10765000012384F844302562E561A5626562C4F8BF
:107660002C806671A760A571204602F017FCE36CC0
:10767000F20701934FF480530A934FF08003029571
:107680000395049505950795089509950B9506931F
:1076900024D5206BD0B1E368049320230993636958
:1076A0000293FAF75FFA01A9206BFAF73DFA236B10
:1076B0001A6842F001021A60226D918A89B241F083
:1076C000400191825B689BB2236407E0236D4FF613
:1076D000DF721A80DA6842F02002DA60A36C0025BB
:1076E00001934FF480530A9380230693B3070295C6
:1076F0000395049505950795089509950B951ED555
:10770000606BB8B12369049310230393FAF72AFA44
:10771000606B01A9FAF708FA636B1A6842F002027B
:107720001A605D605D60236D9A8A92B242F08002B9
:107730009A8204E0236DDA6842F08002DA60236DF9
:1077400020469A8992B242F400529A8100E00020C9
:107750000CB0BDE8F08100BF00380140B416002035
:1077600074FC00081C120020000801400048004082
:10777000601600201C14002004480040000C01404A
:107780002DE9F04F87B09A468046894616469DF807
:10779000405001F017FF02AF0446034600F1100EFF
:1077A000186859683A4603C2083373451746F7D13B
:1077B000237B0BB903960496404602A901F0EEFD27
:1077C000044640B14368586830B1404602A9224699
:1077D000FAF7A6FBF4E71EE0A36894F800B01F7860
:1077E00017B900950D4803E0022F14D10C480095FD
:1077F000494632465346FFF771FE054650B1094BE4
:10780000077103EB8B03C3F8C002636841465860FD
:1078100001F006FE284607B0BDE8F08F00380140B1
:10782000004800401C1200202DE9F743FBF724F923
:107830007D4E05463378834200F0F2807B4C23680E
:107840001B78002800F0A38063BB0420FAF757FBE5
:10785000774F01463860DFF8E48190B143794FF407
:10786000165188F8C8328368C8F8CC32FAF7E0FCC1
:1078700038680221FAF7D2FC3868042101F0D0FD03
:1078800010E06C4B04201B684FF416529B78009359
:107890000223FFF775FF4379386088F8C8328368A0
:1078A000C8F8CC32236893F80090B9F1010F29D1C0
:1078B0000420FAF724FB604F01463860DFF87C8132
:1078C00090B143794FF4964188F8D0328368C8F874
:1078D000D432FAF7ADFC38684946FAF79FFC3868AD
:1078E000042101F09DFD0DE000904B4604204FF473
:1078F0009642FFF745FF4379386088F8D0328368B5
:10790000C8F8D43223681F78022F7AD10420FAF7FE
:10791000F6FA4A4C0146C4F8D802A0B143794FF4B4
:10792000964184F8DC328368C4F8E032FAF780FCD0
:10793000D4F8D8023946FAF771FCD4F8D8020421F9
:1079400001F06EFD0EE000903B4604204FF496429D
:10795000FFF716FF4379C4F8D80284F8DC32836855
:10796000C4F8E032D4F8D872354C94F84A20022A90
:1079700049D1344B1C60002C43D0204600214C22BE
:1079800005F0B3FE0223276084F84A3039E07BB962
:10799000274FDFF8A880386898F8C812FAF73EFC3D
:1079A0003868D8F8CC12FAF743FC386802F048F887
:1079B00023681B78012B0FD11F4FDFF880803868B8
:1079C00098F8D012FAF72AFC3868D8F8D412FAF7E7
:1079D0002FFC386802F034F823681B78022B10D192
:1079E000164CD4F8D80294F8DC12FAF717FCD4F845
:1079F000D802D4F8E012FAF71BFCD4F8D80202F04F
:107A00001FF835700CE094F89630022B01D14C34FD
:107A1000AFE7002AADD04C34002B18BF0024A8E7F4
:107A200003B0BDE8F08300BF01050020040500207D
:107A300008050020680D0020940500201C1200207D
:107A400020080020A8050020F7B5254B1B78042B43
:107A50003FD12020FAF753FA044670B12046FAF7D6
:107A6000E2FB18B90A20FAF768FBF7E71D4B20463E
:107A70001B681969FAF7DCFB0AE01A4B21461B6800
:107A800000901A6920200323FFF77AFE044600B312
:107A9000154B08221A61154D2868FAF7D3FB50B12F
:107AA000114E082777612868FAF7C7FB0146204680
:107AB000FAF7DAFB37612046FAF7C4FB0028EAD070
:107AC00020462D68FAF7B9FB01462846FAF7CCFBA9
:107AD000E1E7074803B0BDE8F040FAF75FBC00BF3C
:107AE000100A00200C0A0020000C0140300A00207F
:107AF0001610010873B5264C264DE369284643F459
:107B00008043E361236901A943F48043236118237F
:107B10008DF806304FF42043ADF8043003238DF880
:107B20000730FBF723F904234FF480460DEB0301E4
:107B300028468DF80630ADF80460FBF717F94FF4CE
:107B40008053ADF804302846102301A98DF8063083
:107B5000FBF70CF9236930463343236102F004FA42
:107B60000D4B1A8802F4415242F4457242F003026E
:107B70001A809A8B22F400621204120C9A83072254
:107B80001A821A8892B242F040021A8002B070BD86
:107B900000100240000C01400038004000000000CE
:107BA00060492DE9F04F604B0A68B3F90640B2F81E
:107BB000583085B09C420FDBB4F5FA6F92F85660EE
:107BC00007DAE11A4E43A3F5FA6396FBF3F664363F
:107BD00003E0C6F1640600E06426544B0020B3F8CD
:107BE00018B193F9EC3015465B429BB20393014602
:107BF0004D4B40F2E637C35E0293CBEB030303F237
:107C0000F31EBE4503D8002BB8BF5B4201E04FF422
:107C1000FA730229DFF820C12ED092F8D47027B170
:107C2000BB42CCBFC7EB030300236427DFF80491FA
:107C300093FBF7FE6FF0630A39F81E800AFB0E3AD9
:107C40000EF1010E39F91E900FFA88FECEEB090EE7
:107C50000EFB0AFE9EFBF7FEC6442CF800E092F8ED
:107C600054E003FB0EFE324B9EFBF3F33B449BB20E
:107C7000734393FBF7F717E092F8D57027B1BB4237
:107C8000CCBFC7EB03030023DDF80CE003FB0EF7CA
:107C9000ACF8047092F85570002BB8BF5B427B4380
:107CA000234F93FBF7F76437531893F804C0DFF8BA
:107CB0008CE007FB0CFC64239CFBF3FC01F80EC07A
:107CC00095F80E800EF1030C07FB08F898FBF3F80B
:107CD00001F80C8095F818C00EF1060E07FB0CF7A2
:107CE00097FBF3F301F80E30029BDFF84CE05B45A5
:107CF00004DA3EF800305B422EF8003001310329EF
:107D000000F1020005F101057FF472AF074FB7F8EB
:107D10001A319C4214DBB4F5FA6FA8BF4FF4FA6431
:107D20000FE000BFF8010020BA0400200C1700206B
:107D30000CFEFFFF00150020BA0300200E150020E6
:107D40001C46E41A4FF47A725443C3F5FA63B4FB49
:107D5000F3F36420A44C93FBF0F204EB42016FF0C8
:107D6000630606FB0233098B04EB4202B2F91A6088
:107D70000AB2B21A534393FBF0F09C4B01441A88A9
:107D80009B4D5606AEF806103ED59A4B1888238EAA
:107D9000C01A00B202F090FB91A3D3E9002302F0D5
:107DA000F1FB02F021FE064605F0CEFE804630468D
:107DB00005F03EFF0646B5F9020002F01FFF8146BE
:107DC000B5F9000002F01AFF4146824602F06AFF50
:107DD00031468346484602F065FF0146584602F0A8
:107DE00057FE03F025F941462880484602F05AFF25
:107DF00031468046504602F055FF0146404602F0AB
:107E000049FE03F015F96880BA6840F60203134092
:107E1000002B53D0784B06211D88636B1D4494F8CA
:107E2000383065630133DBB2B3FBF1F084F83830EE
:107E300001FB103313F0FF0F40D1900706D5F9F77F
:107E4000FDFFF9F7E5FF684B83F83900BB681905BA
:107E500032D56A4BE16B5A7B694B33F81200082329
:107E600091FBF3F280B28A1A0244E26392FBF3F2CE
:107E700092B240F6E4435A43624B40F6FF71B2FBC4
:107E8000F1F219684FF47A73C8888988121A5A4334
:107E900092FBF1F255435C4995FBF3F30A60D4E998
:107EA0001001C01841EBE371C4E910010023574AE7
:107EB00003F004F9564B186000236363554E4A4B98
:107EC000327B94F8398002B1012283F84820BB68E4
:107ED000514D13F4807F2CD0DFF850912878D9F8D9
:107EE0000030C0F380001B685B68984760B10123D5
:107EF00084F84930D9F800301B68DB68984718B11E
:107F0000394B022283F84920D9F800301B689B685E
:107F1000984728B12B785A075CBF022384F8493070
:107F2000D9F800301B689B69984710B1002384F88A
:107F300049303A4B1A6893060DD5737A13B9354B0D
:107F40009B7A2BB1364B1B78980701D4012300E0B4
:107F5000002384F84A3094F84920234B022A02D1A6
:107F60004C204E211EE0012A06D153204D214C22E7
:107F70000B46FDF73BFC2CE093F84A20012A03D185
:107F8000532001464E2206E093F84820012A04D1EE
:107F90005320014602464D23EBE7B8F1000F04D011
:107FA00053204D210A464423E3E710490A8811066D
:107FB00003D553204D210246DAE71A4A12781AB146
:107FC0003220FDF7E2FB04E0404683F84B80FAF7ED
:107FD000BEF82B785A072BD5134B08225A617BE049
:107FE000399D52A246DF913F001500204203002038
:107FF000BA030020F80200202403002078060020A5
:1080000088060020740D002018050020407E050021
:108010001C0500202C030020DC1C0020680200202E
:10802000DE020020AE020020000C0140EC0900201E
:1080300032781AB99C4A43F0010313709B4B1B889A
:108040001BB19B4A13689B0705D49A4B1B880033CE
:1080500018BF012300E0012343B1974BDA6882F097
:108060000802DA602B7823F001032B70934B1B7806
:10807000180703D42B7823F001032B70337D1BB139
:108080002B7823F001032B702B788D4A13F0010F0E
:1080900005D00023E364884B082119610BE0E16CF3
:1080A000136841B9874903F5F42303F59073CB6452
:1080B000814B08215961E36C12686BB1D21A002A16
:1080C0000ADB7D4A03F5F423D16803F5907381F050
:1080D0000801D1607B4AD3647B4B1B780BB1FFF75F
:1080E000A3FB7A4B1B7813B1FEF744FF13E3DFF8D1
:1080F0000C8298F84A30012B05D0754B08F14C08DA
:108100009845F6D107E3734BD8F800207249C3F8BD
:1081100000800A609946704E3068FAF793F800289C
:10812000EBD03068FAF789F8D9F8003093F8482096
:10813000DAB9B0F124014A424A4183F84820002AC2
:10814000E9D12B785B07E6D4232802D1FEF712FF92
:10815000E1E7624B1B681B7D8342DCD1604A614BC7
:108160001A60614A614BDA60D5E7012A04D14D28D3
:1081700014BF00220222CBE2022A04D13C2814BF01
:1081800000220322C4E2032A0AD140284FF0000251
:1081900000F2BE821A71DA71587198710422B7E246
:1081A000042A06D19A7983F8490050409871052233
:1081B000AEE2052AAFD159791A799142997906D957
:1081C00041409971511C197113441872A3E78142FF
:1081D00040F09B8293F84900FBF706FF002840F02F
:1081E0008F82D9F8003093F84930C83B322B00F227
:1081F000AC82DFE813F04D002902920033004D01FC
:1082000002020A027801F7014D0235004800B1016F
:10821000E901A801AA02AA02AA02AA02AA02AA02C3
:10822000AA02AA02AA02AA02AA02AA02AA02AA02EE
:10823000AA02AA02AA02AA02AA02AA02AA02AA02DE
:10824000AA02AA028500AA02AA02AA02AA02AA02F5
:10825000AA02AA02AA02AA02AA0212020026E8E0C0
:108260002B7803F0040303F0FF06002B40F0458257
:10827000F9F728FE022887F8A00540F2B9811C4BC7
:1082800083F8A065B4E1F9F727FEA4F8500034E2C2
:108290000026F9F721FE174B98530236102EF8D11D
:1082A0000122154BF2E100BFDC1C002080020020FF
:1082B00068020020D81C0020000C0140DE020020D3
:1082C000CC1C00200015002000050020DB1C002035
:1082D000B8080020AC050020B005002004080020EC
:1082E000EFBEADDEF04F00200400FA0500ED00E027
:1082F0000C170020BA040020E40100202008002010
:10830000C84ED6F800A0F9F7E7FDAAF85E00366877
:10831000F9F7E2FDA6F85C00EFE1C24E33681B7886
:10832000022B69D10026DFF8FCA2DAF800B0F9F7D9
:10833000C9FD06F108020BEB820B02F05BFCBA49A7
:1083400002F064FDCBF80400DAF800B0F9F7BAFDEA
:1083500006F10A020BEB820B02F04CFCB34902F06F
:1083600055FDCBF80800DAF800B0F9F7ABFD06F1DF
:108370000E020BEB820B02F03DFCAD4902F046FD14
:108380000136032ECBF80400CDD1072E1BD1DFF828
:1083900094B2DBF800200092F9F794FD02F02AFC79
:1083A000A14902F033FD009ADBF800B09064F9F7C0
:1083B00089FD02F01FFC9C4902F028FDCBF84C001F
:1083C000F9F780FD14E0DAF800B0F9F77BFD0BEB6C
:1083D00006031871DAF800B0F9F774FD0BEB060329
:1083E0009873DAF800B0F9F76DFD0BEB0603187619
:1083F00001360A2EC9D180E14FF0000AD6F800B04C
:10840000F9F760FD0BEB0A031871D6F800B0F9F725
:1084100059FD0BEB0A039873D6F800B0F9F752FD3B
:108420000BEB0A030AF1010ABAF10A0F1876E5D13B
:1084300063E1804B1A789A4696420FD2794BD3F873
:1084400000A07D4B16F803B0F9F746FD0BF12003B1
:10845000C0F30B004AF823000136EAE700269AF839
:1084600000309E4280F04981734BF25C6D4B0136C7
:108470001B6803EB820BDBF880300193F9F72CFDCE
:10848000019BC0F30B0043EA0043CBF88030E6E7E2
:1084900064490E68F9F716FD624A86F850001668BE
:1084A000F9F710FD5F4B86F851001E68F9F70AFDD9
:1084B0005C4986F854000E68F9F704FD594A86F8BD
:1084C00055001668F9F7FEFC564B86F856001E68F4
:1084D000F9F7F8FC534986F852000E68F9F7F2FCF8
:1084E00086F8530009E1F9F7F7FCF9F7F5FCA7F86E
:1084F000D000F9F7F1FCA7F8D200F9F7EDFC494AF2
:10850000A7F8D4001668F9F7E7FCA6F81E01F9F7FA
:10851000E3FCF9F7EBFC434B1E68F9F7DDFC00EBDD
:1085200080004000A6F85A00F9F7CCFC87F8040157
:10853000F9F7C8FC87F80601F9F7C4FC87F80501CC
:10854000F9F7C0FCD9E00026F9F7C6FC3B4B98537D
:108550000236102EF8D1D0E00026DFF8C8A0DAF8F5
:1085600000200092F9F7B8FC009A06F11B034FEACD
:10857000C30B5A449080DAF800200092F9F7ACFC63
:10858000009A5A44D080F9F7A7FC072804D8DAF8F3
:10859000002002EB0B03D872A0F57A739BB2B3F5FF
:1085A0007A7F05D8DAF8003003EBC603A3F8E000C1
:1085B000DAF800A0F9F786FC0AEBC6030136082EAC
:1085C00083F8E200C9D198E00026164BD3F800A04A
:1085D000F9F778FC0AEBC6030136082E83F8E300AE
:1085E000F3D18AE02B785E0700F18780FEF7C2FDA9
:1085F00000F048FFFBF710FB7FE02B7858077CD496
:108600000F4B4FF4C8721A8077E02B78590774D457
:108610000C4B1A7842F0040238E02B785A07E7D561
:1086200093E000BFF8010020000020410000C84294
:1086300000007A441D08002008080020E4040020FF
:1086400080020020DE020020F9F73CFC434B1A7840
:1086500010B142F0020201E022F002021A70F9F7B2
:1086600031FC3F4B3F4E1870F9F740FC3060F9F792
:108670003DFC7060F9F730FC3B4B1880F9F72CFC9F
:108680003A4B18803A4B1A7842F002021A7034E0E2
:10869000F9F718FC0090F9F729FC0190F9F726FC8E
:1086A0008246F9F723FC0646F9F716FCF9F714FCA5
:1086B000F9F708FC9DE80C0082B92E4963650B8828
:1086C000C4F858A023F010030B80244B1A7842F012
:1086D00001021A708EB1284BDE650EE0102A0CD113
:1086E0002366C4F864A00EB1234BDE652348022341
:1086F000011D84F8683000F00BFE0020F9F7E8FD5A
:10870000D9F800309879F9F7B4FDD9F80030002293
:1087100083F84820FFE41A4A13689B060FD5194BCB
:10872000E26E1B689A1A002A09DB0D4A1278042AA5
:1087300005D903F51233104A03F5F873D366124BCB
:108740009B683BB11148984704E001200021F9F7EC
:10875000A1FDD5E705B0BDE8F08F00BFDE02002027
:1087600058050020200500208A05002086050020ED
:10877000E51C0020420300200015002060150020A9
:1087800068020020CC1C0020FC0100201205002003
:1087900010B50446204604F0E9FF10F0FF0F07D1A2
:1087A0000B4B0C4893F8A015BDE8104001F0B8B889
:1087B000204605F030F8022808D8054B064C83F80F
:1087C000A00500F05FFEFBF727FAE3E710BD00BF4E
:1087D0000C17002016120108F60F01082DE9F04FC2
:1087E000754985B0044604F089FF74490028204685
:1087F0000CBF0126032604F081FF002808BF0226D3
:10880000F20740F1BE806E4801F08AF80020FDF7C3
:1088100053F86C4F6C4801F083F86C4801F080F815
:108820007A796B4B013A6B4853F8221001F078F8D3
:108830003869002102F0CAFB00285CD13C4605469D
:10884000D4F810800021404602F0C0FB00284ED131
:10885000013561482946D4F814B0D4F818A0D4F8EA
:108860001C9001F05DF84046002102F0B9FB10B108
:108870005A4801F055F86946404601F02DF9014685
:10888000574801F04DF85846002102F0A9FB10B1FD
:10889000524801F045F86946584601F01DF9014675
:1088A0004F4801F03DF85046002102F099FB10B10D
:1088B0004A4801F035F86946504601F00DF9014685
:1088C000474801F02DF84846002102F089FB10B11D
:1088D000424801F025F86946484601F0FDF8014696
:1088E000404801F01DF80C2D04F11004A8D13E48B9
:1088F000691C01F015F83D4801F012F83C4CD7F81E
:10890000088054F8041F19B13A4801F009F8F8E753
:108910000C46394B53F8245055B10123A34013EAB8
:10892000080F03D03548294600F0FAFF0134F0E77C
:10893000334800F0F5FF29467B1893F80E3104AA5E
:108940001344304A8A5C0131082903F8102CF3D112
:10895000002369462C488DF8083000F0E1FF2B48D1
:1089600000F0DEFF2A48FCF7FDFF2A4800F0D8FFA0
:10897000274800F0F3FF284800F0D2FF4020FDF721
:10898000FDFDB30714D5254800F0CAFF244800F0C8
:10899000C7FF1F48FFF7FCFE224800F0C1FF1C483C
:1089A000FCF796FF1C4800F0BBFF8020FDF7E6FDBA
:1089B00005B0BDE8F08F00BF23120108B511010812
:1089C0002A1201080C170020381201084A12010867
:1089D00070FD00085612010861120108C50F010858
:1089E000300B01088A0C0108691201087B1201088A
:1089F000C8FD00088B120108CCFD0008991201087F
:108A0000A612010849140108B2120108BB1201089C
:108A1000F60F0108C71201080E0D0108D512010852
:108A2000E8120108F61201082DE9F74F9E4A9F4906
:108A300013689F4D03F59C4320330B60AB681746CA
:108A400013F4807F04D09B4B1B681B681B699847FD
:108A5000AB6842F201041C405CB9974E337873B1A5
:108A6000944B1B681B681B689847FCF79FFC34708D
:108A700005E0924B1A7801321A70FCF797FCAB684C
:108A8000D80404D58E4B1B780BB9F9F76BFE8D4BD0
:108A90003C681B681E7CCEB18B4A013E32F9160041
:108AA000A0F57A70B0F57A7FA8BF4FF47A7020EA0B
:108AB000E07002F0A3F8854902F0A8F9844902F0B9
:108AC000F1F802F0DBFA7D4B58803EE0AB68190408
:108AD0003BD57A4A5368E31A002B36DB04F59C43F6
:108AE000203353607B4B59797B4B33F81100137A59
:108AF00080B2013303F00F031372D71802F07EF82F
:108B0000764902F083F902F0B9FA334678723046BA
:108B10006A4E06F109029A5C01331044102B80B2B0
:108B2000F6D100B290FBF3F000B26428A8BF642035
:108B300020EAE07002F062F8694902F067F96449DE
:108B400002F0B0F802F09AFA7080AB68DA0510D53E
:108B5000644B9C42644C08D923681B681B6A984785
:108B600018B923681B685B6A984723681B685B69B0
:108B70009847AA68544E12F4805F4D4BB5F8DC104C
:108B8000B6F9062007D0B3F81831581A824207DD2B
:108B900019448A4202E0B3F81A319A42C0F2C48200
:108BA0000122524F0021D7F8009095F8218195F8C5
:108BB00022C1B5F81A41B5F81CA10B46705E9B089E
:108BC000A042C4BF63F07F03DBB202315045B8BF9F
:108BD00043F040030829F1D1384C617E994204D119
:108BE000A17EF92903D8013100E00021A176637646
:108BF000D9F88030B3B1324B1B783BB192B93C4BC2
:108C00001B78DB070ED5F9F7CFFA0BE0384B1B7852
:108C1000580707D5BCF1000F02D0F9F7A3FD01E01A
:108C2000002AFAD0A37E254A142B40F09380304BC3
:108C300018F100081B7818BF4FF0010803F0040377
:108C400003F0FF00A3B1D9F8803023B9537E5F2B26
:108C500001D1F9F787FDB8F1000F7BD0D9F880304A
:108C6000002B77D1637E7D2B74D1F9F77BFD71E00A
:108C7000537E572B0BD11F4B4FF47A721A801E4B29
:108C80001B6813F0080365D11C4A138062E0A968D1
:108C9000490743D55A2B41D1194B1978A1B3187004
:108CA0000122184B4AE000BFCC1C0020EC01002040
:108CB0000C170020E8010020F000002070150020B3
:108CC0002C030020F4000020BA04002000007A44A5
:108CD00000C07F447806002088060020CDCC2342C7
:108CE0000000C842404B4C00E8090020F801002079
:108CF000DC1C0020D81C002068020020F8020020A4
:108D0000AD020020AF020020D17E964B81F0010120
:108D1000D17609B1022211E003220FE05D2B00F0B1
:108D2000D3815B2B00F0D2815E2B09D1D0E1A72B40
:108D300040F0B1818C4B1A7842F004021A7009E0BD
:108D4000D9F88020002A40F09E816F2B40F0958159
:108D5000F9F72AFAD5F808C01CF0040F2FD0E27EEC
:108D6000824B8AB1824A127852070DD5814AB6F9F0
:108D70000610B2F81A21914206DD1A7822B97E490E
:108D8000322008807D49CA761B7C53B17C4B1A780F
:108D90002AB97C4A127812B9774A3221118001220D
:108DA0000CE0784B1A7852B1714A127802F0040242
:108DB00002F0FF011AB91970734B01221A70734B3C
:108DC0003F68002293F80180803710461146134611
:108DD000434501DB00233BE0082BFBD02BB19C0774
:108DE00003D1043A1030D2B2C0B2694C40F2A46947
:108DF00004EB4304268954B21C44A6F2155A04EB32
:108E0000440436B2BAF5C77FE4B204F1010B8CBF5B
:108E10004FF0000A4FF0010A4E450AFA0BFAD4BF90
:108E20004FF000094FF0010904F1020B09FA0BF9A8
:108E30004AEA090940F2135A5645CCBF00260126DA
:108E400006FA04F449EA0404844001332143BFE7ED
:108E500057F82320454E11420CBF002201229A559B
:108E60000133152BF4D173784A4F4B4C1BB13B683F
:108E700098070BD416E01CF4807F13D0474B1B6877
:108E80001B689B6898470028F1D10BE0228812F0FC
:108E900001030DD1394942F00102CB610B623E4919
:108EA0000A8006E0238823F001032380012300E0E9
:108EB0000023B2788AB183B1238823F0010203F042
:108EC000020392B29BB222805BB92C4942F00202AB
:108ED000CB610B62304B1A8003E0238823F002033E
:108EE00023803B68990640F1B4801F490B789A07AC
:108EF00040F1A8802A4A1278042A40F2A380727AAC
:108F0000A2B103F0100303F0FF02002B40F0A18098
:108F10002388244823F0200343F010032380224BAE
:108F2000011D1A7000F0F4F9022290E023F0100302
:108F30000B700E4B9B7A002B56D01C4B1B6859892B
:108F40001B4BB3F900000028B8BF4042884231DA19
:108F5000B3F90230002BB8BF5B428B42ACBF002399
:108F6000012328E0AE020020DE0200202C030020B6
:108F7000DC1C00200C17002094020020701500203B
:108F8000AC020020AD020020AF020020F309002057
:108F9000BA0400206802002042030020E8090020F3
:108FA000580500205415002048000020C803002068
:108FB000BA0300201346DB0716D5228802F02003EF
:108FC0009BB2002B45D1634942F020020A80624ADD
:108FD00062481370624B011D1A685B68026043604F
:108FE00000F096F9012232E023885B4A23F0200347
:108FF000238013786BBB012111701A465949002058
:1090000050525949594F5052594907EB030C50528D
:109010000021D9510232CCF80400CCF8081007F135
:10902000280C503743F80C10D9519C441F44042A93
:10903000CCF80400CCF808107860B96003F1140390
:10904000DCD106E02388002223F030032380494B43
:109050001A70F37A1BB1238843F4807302E02388EB
:1090600023F4807323806B79082B01D00E2B6DD1F4
:10907000238823F04003238068E0B8F1000F02D07A
:109080007E2B3FF465AE972B7FF451AE3A4B4FF4F5
:10909000C8721A805EE60022BB2B019201D1022326
:1090A00003E0B72B04D14FF6FE73ADF8063020E095
:1090B000BE2B01D1022304E0BD2B7FF44BAE4FF653
:1090C000FE73ADF8043014E0012202E0022200E059
:1090D00003225FFA82F808F1FF3385F8A03500F02B
:1090E000D1F9FAF799FD022028214246F9F736F81E
:1090F00030E63B68BDF80410B3F85C200A44A3F8DE
:109100005C20BDF80610B3F85E200A44A3F85E2088
:1091100000F0B8F9FAF780FD0F2014210122F9F7C9
:109120001DF80023A37615E6144B00220021DA6116
:109130001A62C3F89C20C3F8A020C3F8A420C3F887
:10914000A810C3F8AC10C3F8B0102AE503B0BDE80E
:10915000F08F00BF4203002048000020601500206F
:1091600020050020D01C0020CC03002094150020F6
:10917000D003002068150020800200207015002018
:1091800008B500F07FF9FAF747FDBDE808400F2069
:1091900014210122F8F7E2BF1A4B73B51A881A4D51
:1091A00022F040021204120C1A801A88102622F0B3
:1091B00038021204120C1A801A88044692B242F045
:1091C00040021A80BB206E61FBF792FF6846FCF7F5
:1091D00099F92E619DF800209DF8013043EA0223A1
:1091E00023809DF802209DF8033043EA0223638028
:1091F0009DF804209DF8053043EA0223A38002B0C5
:1092000070BD00BF00300140000801401A4B73B52B
:109210001A881A4D22F040021204120C1A801A8881
:10922000102622F038021204120C1A801A88044602
:1092300092B242F040021A80C3206E61FBF758FFE1
:109240006846FCF75FF92E619DF800209DF801301B
:1092500043EA022323809DF802209DF8033043EA6D
:10926000022363809DF804209DF8053043EA022321
:10927000A38002B070BD00BF003001400008014073
:10928000426A10B58469A154416A02690131B1FB97
:10929000F2F402FB14124262426B32B11368DB0734
:1092A00008D4BDE81040FCF757BA036DDA6842F005
:1092B0008002DA6010BD10B500231349DAB2585CA1
:1092C0002728084603D00133092BF6D11A460F4B45
:1092D00083F828210022845CD1B2102C03D0013203
:1092E000092AF8D111464FF4E132C3F82C21C3F812
:1092F0003021C3F83421C3F83821522283F82911D0
:1093000083F83C2110BD00BF521401080C17002047
:10931000F7B50368174C184D23600B68174E636050
:109320000068F9F76FFC95E80300154B0196009370
:1093300094E80C00F9F724FC3668124B60681E6054
:109340006B68114FC01A01F059FC104B196801F0FD
:10935000A9FC01F06DFE22682B687860D31A3B608F
:109360000B4B1E600B4B1B68DA880B4B1A8003B04B
:10937000F0BD00BF680F002020050020740F002002
:10938000700F0020B00F0020780F00204400002054
:10939000A80F0020C8030020A40F00202DE9FF41E2
:1093A00080460F461C480021142204F09EF9002636
:1093B00073B2002B28DC0C225A43184C02F10C0328
:1093C0002244127A23440025E8B20135CAB91D7A35
:1093D000D1B2013295B9401A002801DC0136E7E725
:1093E00001AD94E8070085E8070093E8070084E8EA
:1093F000070095E8070083E80700EFE7691E0D40C6
:10940000E6E7511E0A40DFE7034A4046394604B00A
:10941000BDE8F041F8F784BD241600202C000020A0
:10942000054B5A68824204D01A690C33824218BF35
:1094300000235972704700BF2C0000200F4B1A7890
:109440004F2A17D1598840F2A452914212D11A7969
:10945000BE2A0FD193F8A1250020EF2A0CD113F8D2
:10946000012B5040064A9342F9D1D0F1010038BF98
:109470000020704700207047704700BF00F80108C7
:10948000A4FD01084A4B4F222DE9F3411A7040F226
:10949000A4525A80BE221A71EF2283F8A12500221D
:1094A00083F8A22511461E46B35C0132594040F2B2
:1094B000A4539A42F8D13E4B3E4A83F8A2153E4B44
:1094C00004275A6002F188325A600020013F17F0E9
:1094D000FF075DD0384B3422384CDA60C4F30903FF
:1094E0007BB1331903F17843A3F5FC33D3F8008043
:1094F0004FF400500023019300F03EFD0428E5D115
:109500001BE04FF4302000F037FD0428DED12A4D57
:109510004FF430202B6943F002032B616C612B69FF
:1095200043F040032B6100F027FD2A6941F6FD73EB
:10953000134004282B61D4D0C8E71F4D4FF40050CE
:109540002B6943F001032B611FFA88F3238000F09D
:1095500013FD042812D1A31C0193019B4FEA184864
:10956000A3F800804FF4005000F006FD2B6941F68F
:10957000FE721A4004282A6106D0A7E72B6941F63B
:10958000FE721A402A61A1E70D4B04349C42A5D11A
:10959000094B04281A6942F080021A6102D1FFF7D0
:1095A0004DFF10B90A20F8F71DFE02B0BDE8F081AA
:1095B0000C170020230167450020024000F8010835
:1095C000A4FD010870B50022064630491001431879
:1095D000415CB14204D00132062AF6D1002070BDB0
:1095E0002B4D042E05F114040FCB84E80F002B46FD
:1095F00018D007D8012E0CD0022E44D1254B1B6861
:109600009B680DE0102E38D0202E06D0082E3AD1BF
:109610001CE0204B1B685B6832E01E4B1B681B691B
:10962000AB612DE01C4A126812783AB1012A08D0C9
:10963000022A0CBF4FF49642002204E04FF4165267
:1096400001E04FF496429A61DA611CE0134A126815
:10965000127A042A17D8DFE802F008080308080085
:109660000F4AAA61EA61032204E04FF4E132AA61E1
:10967000EA61012283F8212005E0064B1B68DB68C4
:10968000EB61204670BD074870BD00BF84F3000841
:10969000241600200408002004050020F400002007
:1096A000A08601003816002038B5374B374D1A8890
:1096B000102422F040021204120C1A801A886B2027
:1096C00022F038021204120C42F030021A801A887A
:1096D00092B242F040021A806C61FBF709FD8020D3
:1096E000FBF706FD96202C61F8F727FD6C616820DA
:1096F000FBF7FEFC0320FBF7FBFC96202C61F8F740
:109700001CFD6C616B20FBF7F3FC0320FBF7F0FC06
:1097100001202C61F8F706FD6C616A20FBF7E8FC7C
:109720002046FBF7E5FC01202C61F8F7FBFC6C619F
:109730006C20FBF7DDFC0020FBF7DAFC01202C613C
:10974000F8F7F0FC6C611920FBF7D2FC0020FBF766
:10975000CFFC01202C61F8F7E5FC6C611C20FBF7C5
:10976000C7FC2046FBF7C4FC01202C61F8F7DAFCAB
:109770006C611B20FBF7BCFC1820FBF7B9FC044B09
:1097800001222C611A7038BD0030014000080140F0
:10979000B60600202DE9F04F064689B00F46154663
:1097A0009B462978002900F0B880252902D0013590
:1097B0003046B0E06C78302C03D002354FF0000911
:1097C00003E0AC784FF001090335A4F13003092B15
:1097D0004FF000081AD8A4F13003DAB2092A07D8EA
:1097E0000A2B13DC0A2202FB083815F8014BF2E7BA
:1097F000A4F16103052B02D8A4F15703F0E7A4F10B
:109800004103052B02D8A4F13703E9E76C2C03BF11
:109810002C78012201350022632C66D006D8252C35
:1098200077D0582C3FD0002C77D0BAE7732C63D078
:1098300002D8642C11D0B4E7752C02D0782C32D029
:10984000AFE70BF1040A05ACDBF800000A2112B106
:109850000022234613E0234620E00BF1040A05AC66
:10986000DBF8000072B1002806DA2D238DF81430E1
:1098700040420DF1150300E023460A210022F9F7CA
:1098800071F80DE0002806DA2D238DF814304042DF
:109890000DF1150300E023460A210022F9F73AF8FA
:1098A000D34600941AE00BF1040303930DF1140A5C
:1098B000DBF80000102132B1583C6242624153464D
:1098C000F9F750F806E0B4F158035A425A415346AA
:1098D000F9F720F8DDF80CB0CDF800A03046394695
:1098E00042464B46F9F77AF85BE730469BF80010A2
:1098F0000BF10404B8470AE0DBF80030304600936F
:109900003946424600230BF10404F9F767F8A346F1
:1099100047E730462146B84743E709B0BDE8F08F36
:109920000FB407B50A4904AB08680A4953F8042B79
:1099300009680193FFF72EFF074B1868F8F773FCCF
:109940000028F9D003B05DF804EB04B0704700BF05
:10995000700600206C060020181200202DE9F74345
:10996000044603F003FFC0B290B9304C054694F8AA
:10997000C711B4F8C42194F8C6312D480091294686
:109980000135FFF7CDFF102D04F10404EFD14AE0BB
:10999000204603F040FF0F28054636DC20462021F4
:1099A00003F0D7FE234FEDB2D7F80090441CAD0072
:1099B0000026204603F02FFF5FFA86F8B8F1010F6A
:1099C00083B208D0B8F1020F0BD0B3F5B47F1ED22A
:1099D0003A6853530AE0FF2B19D83B682B44987020
:1099E00004E0FF2B13D83B682B44D87020462C2171
:1099F00003F0AFFE044608B1441C02E0B8F1020FC8
:109A000005D10136032ED4D10DE00B4806E009EB59
:109A100005000021042203F068FE0848102103B06D
:109A2000BDE8F0437CE703B0BDE8F0830C170020ED
:109A30005B140108600D00206F140108410C01083F
:109A4000054B5A68824204D01A690C33824218BF0F
:109A5000002300225A7270472C00002070B5054682
:109A6000441E14F8011F61B1064E304603F071FE2A
:109A70000028F6D0861B0448631B304480F80E3162
:109A8000EFE770BD491401080C1700200F4970B5AD
:109A900000230C781A46D8B2844205D00D7B85424B
:109AA00008BF01200CD100E000200C2505FB0010B0
:109AB000074D084E154495F828510132755D057221
:109AC0000133052B01D0012AE5D970BD2C000020FF
:109AD0000C1700205214010830B587B005460C461B
:109AE00003A800210C2203F000FE2846002101F00B
:109AF00095FA20B128462A4900F0CCFF03E0284619
:109B0000274900F0C5FF274901F0CCF801F090FA91
:109B1000054685EAE570A0EBE57069460A22F8F78C
:109B200049FF00239D420370ACBF20232D236846CC
:109B30008DF80C3003F01AFE012807D130238DF880
:109B40000D308DF80E308DF80F300CE0022805D165
:109B500030238DF80D308DF80E3004E0032804BF5B
:109B600030238DF80D30694603A803F0E5FD03A806
:109B700003F0FCFD0338C5B22A4603A9204603F0D2
:109B80001FFE002363552046074903F0D5FD03A9B6
:109B90002046294403F0D0FD204607B030BD00BF69
:109BA0006F12033A00007A4493140108038A8289F1
:109BB00011EA030092B203D011420CBF0020012031
:109BC00070477C4B70B51B78012B0CBF032500251B
:109BD00099BB048C24F001042404240C0484038B1A
:109BE000048C9BB223F0F30343F0010343EA051511
:109BF000714BA4B2984215D003F50063984211D07E
:109C0000B0F1804F0ED0A3F5983398420AD003F5F7
:109C10008063984206D003F58063984218BF24F011
:109C20000A0401D124F0020444F001042243058314
:109C30000284038B23F00C033AE004293FD1048C07
:109C40005D4B24F010042404240C0484018B048C48
:109C500021F440710905090D41F480719842A4B2C4
:109C600041EA053512D003F5006398420ED0B0F1F9
:109C7000804F0BD0A3F59833984207D003F580634B
:109C8000984203D003F58063984207D124F0200462
:109C900044F0100444EA021292B204E024F0A0045A
:109CA00044F01004224305830284038B23F44063B1
:109CB0001B041B0C0383038B9BB2038370BD082919
:109CC000018C37D121F480710904090C0184838B44
:109CD000048C9BB223F0F30343F0010343EA051520
:109CE000354BA4B2984212D003F5006398420ED0CF
:109CF000B0F1804F0BD0A3F59833984207D003F50D
:109D00008063984203D003F58063984207D124F41E
:109D1000007444F4807444EA022292B204E024F411
:109D2000206444F48074224385830284838B23F06F
:109D30000C0338E021F480510904090C0184838B61
:109D4000068C23F440731B051B0D43F4807343EA18
:109D50000535194BB6B2984212D003F5006398420C
:109D60000ED0B0F1804F0BD0A3F59833984207D0B6
:109D700003F58063984203D003F58063984207D1CE
:109D800026F4005646F4805646EA023292B205E0C6
:109D900047F6FF54344044F48054224385830284C0
:109DA000838B23F440631B041B0C8383838B9BB244
:109DB000838370BDBC080020002C014038B5104CD6
:109DC00004EB0014A278E36842B90122A270A180DA
:109DD0001868197B0222BDE83840F2E6A288E180CB
:109DE0006078891A074A89B2002522F81010A570F8
:109DF00021811868197B2A46FFF7E3FEA57238BD5A
:109E000008090020481600201F4B10B55A6802F0C0
:109E10000C02042A03D0082A04D01C4A14E01C4A6D
:109E2000126811E05A685968C2F38342C90302F10B
:109E3000020201D4174906E0596811F4003F1449A1
:109E4000096818BF49084A4302605968124AC1F3B9
:109E50000311545C0168E14041605C68C4F3022472
:109E6000145D21FA04F484605C68C4F3C224145DB8
:109E7000E140C1605B68C3F381331A44137CB1FBDA
:109E8000F3F1016110BD00BF0010024000127A0022
:109E90001400002000093D004900002070B54479FD
:109EA00086B004F00403866803F0FF0523B14FF485
:109EB00080654FF4005300E02B4614F0010F14BFEF
:109EC00004220022A107046D48BF42F00802218A43
:109ED00048BF92B289B221F440510B432382A38937
:109EE00001A89BB223F4B05323F00C031D432A4373
:109EF000A281A38A23F440731B041B0CA382FFF7E7
:109F000083FF1649049A039B8C4208BF1346A2891B
:109F10001921594312B2002AB4BF7600B600B1FB32
:109F2000F6F16423B1FBF3F21201100903FB1011E7
:109F3000A08900B2002806DAC9003231B1FBF3F380
:109F400003F0070305E009013231B1FBF3F303F03D
:109F50000F031A4392B2228106B070BD003801404F
:109F600041719BE7816099E7024B1A6922EA000080
:109F7000186170470010024010B50446F7F7C0FDA5
:109F8000012806D11CB1F7F7BBFD013CF8E705201D
:109F900010BD002C08BF052010BD00BF0148FAF716
:109FA00077BF00BF000800400148FAF771BF00BF4B
:109FB000000400404FF08040FAF76ABF0148FAF70A
:109FC00067BF00BF002C014038B5194C236D1D88B8
:109FD000ADB2AA0612D5E26A1AB1988880B290474B
:109FE0000CE09B88E2696169DBB28B54E269E3684B
:109FF0000132B2FBF3F103FB1123E3612B0616D50B
:10A00000A26A616A0A4B8A420CD09869196D805C19
:10A010000132C0B288801969B2FBF1F001FB102255
:10A020009A6238BD1B6DDA6822F08002DA6038BDB2
:10A03000601600200D4BD3F8A4201188090613D513
:10A04000D96F986F81420BD0D86E405C0131C0B29D
:10A0500090805A6EB1FBF2F002FB1011D967704785
:10A06000D36823F08003D360704700BF60160020E0
:10A070000B480C4B4FF400525A60D0F888204FF632
:10A08000FE7311680B401360826FC36F9A4202D057
:10A090005430FBF761BB012380F89830704700BF54
:10A0A0006016002000000240084A13689B020BD58E
:10A0B000074B0021197007494FF6FE7308680340EB
:10A0C0000B604FF400135360704700BF0000024064
:10A0D000DA1C00206C000240FBF72AB8FBF728B816
:10A0E000FAF7FABBFAF7F8BB37B5254C254DA3694B
:10A0F000284643F48053A361E36801A943F48053E5
:10A10000E36018238DF80630A023ADF80430032354
:10A110008DF80730F8F72AFE4023ADF80430042309
:10A120000DEB030128468DF80630F8F71FFE1023CB
:10A13000284601A9ADF804308DF80630F8F716FE70
:10A14000E36843F48053E360E36823F48053E360FF
:10A150000D4B1A8802F4415242F4457242F0030258
:10A160001A809A8B22F400621204120C9A8307223E
:10A170001A821A8892B242F040021A8003B030BDAF
:10A180000010024000080140003001400F4B1A68E7
:10A1900042F001021A6059680D4A0A405A601A6872
:10A1A00022F0847222F480321A601A6822F480222B
:10A1B0001A605A6822F4FE025A604FF41F029A6035
:10A1C000044B4FF000629A60704700BF00100240DD
:10A1D0000000FFF800ED00E0024B1A6801321A603F
:10A1E000704700BF0817002008B5084BB3F8D80027
:10A1F00093F8A8250023D9B2914204D2044921F84A
:10A2000013000133F7E7F8F714F9FEE70817002009
:10A21000B21C002081F0004102E000BF83F0004347
:10A2200030B54FEA41044FEA430594EA050F08BFF1
:10A2300090EA020F1FBF54EA000C55EA020C7FEAB5
:10A24000645C7FEA655C00F0E2804FEA5454D4EB32
:10A250005555B8BF6D420CDD2C4480EA020281EAFC
:10A26000030382EA000083EA010180EA020281EA34
:10A270000303362D88BF30BD11F0004F4FEA013186
:10A280004FF4801C4CEA113102D0404261EB410195
:10A2900013F0004F4FEA03334CEA133302D052421B
:10A2A00063EB430394EA050F00F0A780A4F10104D7
:10A2B000D5F1200E0DDB02FA0EFC22FA05F2801811
:10A2C00041F1000103FA0EF2801843FA05F35941F7
:10A2D0000EE0A5F120050EF1200E012A03FA0EFC76
:10A2E00028BF4CF0020C43FA05F3C01851EBE371A0
:10A2F00001F0004507D54FF0000EDCF1000C7EEBBD
:10A3000000006EEB0101B1F5801F1BD3B1F5001FFA
:10A310000CD349085FEA30004FEA3C0C04F1010419
:10A320004FEA445212F5800F80F09A80BCF1004F42
:10A3300008BF5FEA500C50F1000041EB045141EAC4
:10A34000050130BD5FEA4C0C404141EB010111F4C5
:10A35000801FA4F10104E9D191F0000F04BF014670
:10A360000020B1FA81F308BF2033A3F10B03B3F14E
:10A3700020020CDA0C3208DD02F1140CC2F10C02DE
:10A3800001FA0CF021FA02F10CE002F11402D8BF3C
:10A39000C2F1200C01FA02F120FA0CFCDCBF41EA08
:10A3A0000C019040E41AA2BF01EB0451294330BDD7
:10A3B0006FEA04041F3C1CDA0C340EDC04F11404B4
:10A3C000C4F1200220FA04F001FA02F340EA03008B
:10A3D00021FA04F345EA030130BDC4F10C04C4F1D1
:10A3E000200220FA02F001FA04F340EA03002946B1
:10A3F00030BD21FA04F0294630BD94F0000F83F4FB
:10A40000801306BF81F480110134013D4EE77FEADD
:10A41000645C18BF7FEA655C29D094EA050F08BF29
:10A4200090EA020F05D054EA000C04BF194610460A
:10A4300030BD91EA030F1EBF0021002030BD5FEA4E
:10A44000545C05D14000494128BF41F0004130BD76
:10A4500014F580043CBF01F5801130BD01F00045CA
:10A4600045F0FE4141F470014FF0000030BD7FEA3D
:10A47000645C1ABF194610467FEA655C1CBF0B4638
:10A48000024650EA013406BF52EA033591EA030F4F
:10A4900041F4002130BD00BF90F0000F04BF002147
:10A4A000704730B54FF4806404F132044FF000057A
:10A4B0004FF0000150E700BF90F0000F04BF0021F3
:10A4C000704730B54FF4806404F1320410F0004559
:10A4D00048BF40424FF000013EE700BF42004FEA54
:10A4E000E2014FEA31014FEA02701FBF12F07F43D1
:10A4F00093F07F4F81F06051704792F0000F14BFCE
:10A5000093F07F4F704730B54FF4607401F0004511
:10A5100021F0004120E700BF50EA010208BF704768
:10A5200030B54FF000050AE050EA010208BF70475D
:10A5300030B511F0004502D5404261EB41014FF4C6
:10A54000806404F132045FEA915C3FF4DCAE4FF0CA
:10A5500003025FEADC0C18BF03325FEADC0C18BFB1
:10A56000033202EBDC02C2F1200300FA03FC20FA02
:10A5700002F001FA03FE40EA0E0021FA02F114444F
:10A58000C1E600BF70B54FF0FF0C4CF4E06C1CEA64
:10A5900011541DBF1CEA135594EA0C0F95EA0C0FD9
:10A5A00000F0DEF82C4481EA030621EA4C5123EA4C
:10A5B0004C5350EA013518BF52EA033541F480117B
:10A5C00043F4801338D0A0FB02CE4FF00005E1FB2E
:10A5D00002E506F00042E0FB03E54FF00006E1FB78
:10A5E00003569CF0000F18BF4EF0010EA4F1FF04BB
:10A5F000B6F5007F64F5407404D25FEA4E0E6D41FB
:10A6000046EB060642EAC62141EA55514FEAC5200B
:10A6100040EA5E504FEACE2EB4F1FD0C88BFBCF587
:10A62000E06F1ED8BEF1004F08BF5FEA500E50F138
:10A63000000041EB045170BD06F0004646EA0101FE
:10A6400040EA020081EA0301B4EB5C04C2BFD4EB30
:10A650000C0541EA045170BD41F480114FF0000E29
:10A66000013C00F3AB8014F1360FDEBF002001F097
:10A67000004170BDC4F10004203C35DA0C341BDC11
:10A6800004F11404C4F1200500FA05F320FA04F0E3
:10A6900001FA05F240EA020001F0004221F0004117
:10A6A00010EBD37021FA04F642EB06015EEA430E8A
:10A6B00008BF20EAD37070BDC4F10C04C4F12005BA
:10A6C00000FA04F320FA05F001FA04F240EA02006D
:10A6D00001F0004110EBD37041F100015EEA430E3E
:10A6E00008BF20EAD37070BDC4F1200500FA05F25E
:10A6F0004EEA020E20FA04F301FA05F243EA0203DD
:10A7000021FA04F001F0004121FA04F220EA0200EB
:10A7100000EBD3705EEA430E08BF20EAD37070BD31
:10A7200094F0000F0FD101F00046400041EB010111
:10A7300011F4801F08BF013CF7D041EA060195F0F3
:10A74000000F18BF704703F00046520043EB0303AD
:10A7500013F4801F08BF013DF7D043EA060370479A
:10A7600094EA0C0F0CEA135518BF95EA0C0F0CD0A5
:10A7700050EA410618BF52EA4306D1D181EA0301EB
:10A7800001F000414FF0000070BD50EA410606BFE5
:10A790001046194652EA430619D094EA0C0F02D12A
:10A7A00050EA013613D195EA0C0F05D152EA03366F
:10A7B0001CBF104619460AD181EA030101F000418D
:10A7C00041F0FE4141F470014FF0000070BD41F0D6
:10A7D000FE4141F4780170BD70B54FF0FF0C4CF4B0
:10A7E000E06C1CEA11541DBF1CEA135594EA0C0FCF
:10A7F00095EA0C0F00F0A7F8A4EB050481EA030E1C
:10A8000052EA03354FEA013100F088804FEA033302
:10A810004FF0805545EA131343EA12634FEA0222D0
:10A8200045EA111545EA10654FEA00260EF0004191
:10A830009D4208BF964244F1FD0404F5407402D2E3
:10A840005B084FEA3202B61A65EB03055B084FEA74
:10A8500032024FF480104FF4002CB6EB020E75EB71
:10A86000030E22BFB61A754640EA0C005B084FEA99
:10A870003202B6EB020E75EB030E22BFB61A754616
:10A8800040EA5C005B084FEA3202B6EB020E75EB61
:10A89000030E22BFB61A754640EA9C005B084FEAD9
:10A8A0003202B6EB020E75EB030E22BFB61A7546E6
:10A8B00040EADC0055EA060E18D04FEA051545EAD5
:10A8C00016754FEA06164FEAC30343EA52734FEA7E
:10A8D000C2025FEA1C1CC0D111F4801F0BD141EAF7
:10A8E00000014FF000004FF0004CB6E711F4801F5C
:10A8F00004BF01430020B4F1FD0C88BFBCF5E06F3C
:10A900003FF6AFAEB5EB030C04BFB6EB020C5FEA4B
:10A91000500C50F1000041EB045170BD0EF0004EA0
:10A920004EEA113114EB5C04C2BFD4EB0C0541EAD2
:10A93000045170BD41F480114FF0000E013C90E6CF
:10A9400045EA060E8DE60CEA135594EA0C0F08BF93
:10A9500095EA0C0F3FF43BAF94EA0C0F0AD150EA92
:10A9600001347FF434AF95EA0C0F7FF425AF104625
:10A9700019462CE795EA0C0F06D152EA03353FF44D
:10A98000FDAE1046194622E750EA410618BF52EACA
:10A9900043067FF4C5AE50EA41047FF40DAF52EA9E
:10A9A00043057FF4EBAE12E74A0011D212F5001214
:10A9B00011D20DD56FF47873B3EB62520ED44FEA17
:10A9C000C12343F0004343EA505323FA02F0704797
:10A9D0004FF00000704750EA013002D14FF0FF30D5
:10A9E00070474FF0000070474FEA4102B2F1E04378
:10A9F00024BFB3F5001CDCF1FE5C0DD901F0004C66
:10AA00004FEAC0024CEA5070B2F1004F40EB8300B5
:10AA100008BF20F00100704711F0804F21D113F1E1
:10AA20003872BCBF01F00040704741F480114FEA1A
:10AA30005252C2F11802C2F1200C10FA0CF320FAA3
:10AA400002F018BF40F001004FEAC1234FEAD323C0
:10AA500003FA0CFC40EA0C0023FA02F34FEA43032A
:10AA6000CCE77FEA625307D150EA01331EBF4FF0B3
:10AA7000FE4040F44000704701F0004040F0FE40CE
:10AA800040F40000704700BF80F0004002E000BFCB
:10AA900081F0004142001FBF5FEA410392EA030FC9
:10AAA0007FEA226C7FEA236C6AD04FEA1262D2EB13
:10AAB0001363C1BFD218414048404140B8BF5B4218
:10AAC000192B88BF704710F0004F40F4000020F0B1
:10AAD0007F4018BF404211F0004F41F4000121F0C7
:10AAE0007F4118BF494292EA030F3FD0A2F1010211
:10AAF00041FA03FC10EB0C00C3F1200301FA03F14F
:10AB000000F0004302D5494260EB4000B0F5000F71
:10AB100013D3B0F1807F06D340084FEA310102F130
:10AB20000102FE2A51D2B1F1004F40EBC25008BFE2
:10AB300020F0010040EA03007047490040EB0000AC
:10AB400010F4000FA2F10102EDD1B0FA80FCACF1DB
:10AB5000080CB2EB0C0200FA0CF0AABF00EBC250DA
:10AB600052421843BCBFD0401843704792F0000FC8
:10AB700081F4000106BF80F400000132013BB5E71B
:10AB80004FEA41037FEA226C18BF7FEA236C21D091
:10AB900092EA030F04D092F0000F08BF08467047F6
:10ABA00090EA010F1CBF0020704712F07F4F04D1C4
:10ABB000400028BF40F00040704712F100723CBFD7
:10ABC00000F50000704700F0004343F0FE4040F401
:10ABD000000070477FEA226216BF08467FEA2363BF
:10ABE0000146420206BF5FEA412390EA010F40F4AA
:10ABF000800070474FF0000304E000BF10F00043F6
:10AC000048BF40425FEA000C08BF704743F09643DC
:10AC100001464FF000001CE050EA010208BF7047F7
:10AC20004FF000030AE000BF50EA010208BF70477E
:10AC300011F0004302D5404261EB41015FEA010C93
:10AC400002BF84460146002043F0B64308BFA3F18B
:10AC50008053A3F50003BCFA8CF2083AA3EBC2536D
:10AC600010DB01FA02FC634400FA02FCC2F120028C
:10AC7000BCF1004F20FA02F243EB020008BF20F0C3
:10AC80000100704702F1200201FA02FCC2F1200229
:10AC900050EA4C0021FA02F243EB020008BF20EA1E
:10ACA000DC7070474FF0FF0C1CEAD0521EBF1CEA4C
:10ACB000D15392EA0C0F93EA0C0F6FD01A4480EA3A
:10ACC000010C400218BF5FEA41211ED04FF0006323
:10ACD00043EA501043EA5111A0FB01310CF000404F
:10ACE000B1F5000F3EBF490041EAD3715B0040EA75
:10ACF000010062F17F02FD2A1DD8B3F1004F40EB45
:10AD0000C25008BF20F00100704790F0000F0CF017
:10AD1000004C08BF49024CEA502040EA51207F3ADB
:10AD2000C2BFD2F1FF0340EAC250704740F40000B6
:10AD30004FF00003013A5DDC12F1190FDCBF00F0A7
:10AD400000407047C2F10002410021FA02F1C2F155
:10AD5000200200FA02FC5FEA310040F1000053EAF1
:10AD60004C0308BF20EADC70704792F0000F00F03F
:10AD7000004C02BF400010F4000F013AF9D040EA45
:10AD80000C0093F0000F01F0004C02BF490011F4D9
:10AD9000000F013BF9D041EA0C018FE70CEAD153D7
:10ADA00092EA0C0F18BF93EA0C0F0AD030F0004C57
:10ADB00018BF31F0004CD8D180EA010000F000400B
:10ADC000704790F0000F17BF90F0004F084691F0C9
:10ADD000000F91F0004F14D092EA0C0F01D1420203
:10ADE0000FD193EA0C0F03D14B0218BF084608D1CC
:10ADF00080EA010000F0004040F0FE4040F4000016
:10AE0000704740F0FE4040F4400070474FF0FF0CA8
:10AE10001CEAD0521EBF1CEAD15392EA0C0F93EAEF
:10AE20000C0F69D0A2EB030280EA010C49024FEA41
:10AE3000402037D04FF0805343EA111143EA1013FA
:10AE40000CF000408B4238BF5B0042F17D024FF4B2
:10AE5000000C8B4224BF5B1A40EA0C00B3EB510F8D
:10AE600024BFA3EB510340EA5C00B3EB910F24BF76
:10AE7000A3EB910340EA9C00B3EBD10F24BFA3EBFB
:10AE8000D10340EADC001B0118BF5FEA1C1CE0D1C3
:10AE9000FD2A3FF650AF8B4240EBC25008BF20F076
:10AEA000010070470CF0004C4CEA50207F32C2BFCA
:10AEB000D2F1FF0340EAC250704740F400004FF067
:10AEC0000003013A37E792F0000F00F0004C02BF98
:10AED000400010F4000F013AF9D040EA0C0093F062
:10AEE000000F01F0004C02BF490011F4000F013BBC
:10AEF000F9D041EA0C0195E70CEAD15392EA0C0F24
:10AF000008D142027FF47DAF93EA0C0F7FF470AF5B
:10AF1000084676E793EA0C0F04D14B023FF44CAF9E
:10AF200008466EE730F0004C18BF31F0004CCAD133
:10AF300030F000427FF45CAF31F000437FF43CAF6F
:10AF40005FE700BF4FF0FF3C06E000BF4FF0010C91
:10AF500002E000BF4FF0010C4DF804CD4FEA400273
:10AF60004FEA41037FEA226C18BF7FEA236C11D0BD
:10AF700001B052EA530C18BF90EA010F58BFB2EB70
:10AF8000030088BFC81738BF6FEAE17018BF40F0F0
:10AF9000010070477FEA226C02D15FEA402C05D1A4
:10AFA0007FEA236CE4D15FEA412CE1D05DF8040B29
:10AFB000704700BF844608466146FFE70FB5FFF7BC
:10AFC000C9FF002848BF10F1000F0FBD4DF808ED74
:10AFD000FFF7F4FF0CBF012000205DF808FB00BF65
:10AFE0004DF808EDFFF7EAFF34BF012000205DF8BF
:10AFF00008FB00BF4DF808EDFFF7E0FF94BF01200C
:10B0000000205DF808FB00BF4DF808EDFFF7D2FF08
:10B0100094BF012000205DF808FB00BF4DF808ED4B
:10B02000FFF7C8FF34BF012000205DF808FB00BF18
:10B030004FEA4002B2F1FE4F0FD34FF09E03B3EB45
:10B0400012620DD94FEA002343F0004310F0004F85
:10B0500023FA02F018BF404270474FF000007047DB
:10B0600012F1610F01D1420205D110F0004008BF7A
:10B070006FF0004070474FF00000704742000ED262
:10B08000B2F1FE4F0BD34FF09E03B3EB126209D423
:10B090004FEA002343F0004323FA02F070474FF0D9
:10B0A0000000704712F1610F01D1420202D14FF04E
:10B0B000FF3070474FF00000704700BF73B96AB9A6
:10B0C000002908BF0028BCBF00204FF00041C4BFCA
:10B0D0006FF000414FF0FF3000F03CB882B0EC461A
:10B0E0002DE9005000F006F8DDF804E002B00CBCD9
:10B0F000704700BF2DE9704F089E14461D468046DC
:10B10000894600F029F804FB01F3A4FB00AB00FB27
:10B1100005329344B8EB0A0869EB0B09C6E90089CC
:10B12000BDE8708F2DE9704F089E14461D4680467D
:10B13000894600F061F900FB05F5A0FB04AB04FBB8
:10B140000154A344B8EB0A0869EB0B09C6E900896E
:10B15000BDE8708F704700BF00292DE9F00FC0F2E5
:10B16000A1800024002BC0F29880154606460F46A9
:10B17000002B3FD18A4258D9B2FA82F34BB1C3F1C6
:10B18000200201FA03F720FA02F29D4000FA03F6CA
:10B190001743290CB7FBF1F201FB1277A8B200FBB1
:10B1A00002F34FEA164C4CEA0747BB4209D97F1914
:10B1B00002F1FF3C80F00581BB4240F20281023A7D
:10B1C0002F44FF1AB7FBF1F301FB137100FB03F0EF
:10B1D000B6B246EA0141884208D9491903F1FF375E
:10B1E00080F0F180884240F2EE80023B43EA024266
:10B1F000002303E08B420AD900231A461046194661
:10B2000014B1404261EB4101BDE8F00F7047B3FA61
:10B2100083F8B8F1000F40F088808B4202D382425D
:10B2200000F2E28000230122E8E712B90123B3FB18
:10B23000F2F5B5FA85F2002A3AD17F1B280C1FFAE5
:10B2400085FC0123B7FBF0F100FB11770CFB01F249
:10B250004FEA164848EA0747BA4207D97F1901F171
:10B26000FF3802D2BA4200F2C4804146BF1AB7FB8F
:10B27000F0F200FB12700CFB02FCB6B246EA004092
:10B28000844507D9401902F1FF3702D2844500F204
:10B29000AE803A4642EA0142B0E7E443524263EBF1
:10B2A000430362E7404261EB41014FF0FF3459E74D
:10B2B0009540C2F1200927FA09F126FA09F99740C9
:10B2C000280CB1FBF0F800FB18111FFA85FC0CFBF1
:10B2D00008F349EA07094FEA194747EA01418B4257
:10B2E00006FA02F608D9491908F1FF327AD28B42E0
:10B2F00078D9A8F102082944C91AB1FBF0F300FB80
:10B3000013170CFB03F21FFA89F949EA0747BA42FF
:10B3100007D97F1903F1FF3160D2BA425ED9023BEF
:10B320002F44BF1A43EA08438CE7C8F1200225FAEC
:10B3300002F103FA08FC27FA02F320FA02F207FAF4
:10B3400008F741EA0C0C4FEA1C49B3FBF9F109FB81
:10B3500011331FFA8CFA0AFB01FB17433A0C42EA3D
:10B3600003439B4505FA08F008D913EB0C0301F1E0
:10B37000FF3235D29B4533D902396344CBEB03030B
:10B38000B3FBF9F209FB12330AFB02FABFB247EA38
:10B390000347BA4508D917EB0C0702F1FF331BD25C
:10B3A000BA4519D9023A674442EA0145A5FB0001B2
:10B3B000CAEB07078F424FF000030AD305D02A4695
:10B3C0001CE76246FDE63B4610E706FA08F68642B1
:10B3D000F5D26A1E002311E71A46E5E70B46A0E7FF
:10B3E0001146CBE7904687E74346424606E7023AD6
:10B3F00050E702392F4439E72DE9F00F144605468E
:10B400000E46002B43D18A4253D9B2FA82F757B184
:10B41000C7F1200620FA06F601FA07F302FA07F44C
:10B4200000FA07F51E43210CB6FBF1F201FB126690
:10B43000A0B200FB02F32F0C47EA0646B34209D93B
:10B44000361902F1FF3780F0FD80B34240F2FA80F6
:10B45000023A2644F61AB6FBF1F301FB136100FB36
:10B4600003F0ADB245EA0141884208D9091903F158
:10B47000FF3680F0E980884240F2E680023B43EAF2
:10B480000242002310461946BDE8F00F70478B4278
:10B490004CD8B3FA83F6002E4FD18B4202D38242AE
:10B4A00000F2DD80BDE8F00F0023012210461946AE
:10B4B000704712B90124B4FBF2F4B4FA84F2002A02
:10B4C00040F08280091B260CA7B20123B1FBF6F0E5
:10B4D00006FB101107FB00F24FEA154C4CEA014144
:10B4E0008A4207D9091900F1FF3C02D28A4200F2D0
:10B4F000C8806046891AB1FBF6F206FB121107FB01
:10B5000002F7ADB245EA0145AF4208D92C1902F164
:10B51000FF3180F09B80A74240F29880023A42EAD5
:10B52000004210461946BDE8F00F704700231A4646
:10B5300010461946BDE8F00F7047C6F1200522FA03
:10B5400005F703FA06F421FA05F301FA06FB20FADF
:10B5500005F53C434FEA1448B3FBF8FC08FB1C33E9
:10B560001FFA84F909FB0CFA45EA0B0B4FEA1B455D
:10B5700045EA03439A4502FA06F204D91B190CF175
:10B58000FF356FD3AC46CAEB0303B3FBF8F508FBFA
:10B59000153309FB05F91FFA8BFB4BEA0347B94545
:10B5A00004D93F1905F1FF3362D31D4645EA0C4C1F
:10B5B000ACFB0223C9EB07079F424FF000054AD3BB
:10B5C00046D062462B465DE79440C2F1200921FA3D
:10B5D00009FC914020FA09F9260CBCFBF6F806FBA1
:10B5E00018CCA7B207FB08F349EA01094FEA194151
:10B5F00041EA0C4C634500FA02F509D91CEB040C36
:10B6000008F1FF323BD2634539D9A8F10208A444BE
:10B61000C3EB0C0CBCFBF6F306FB13C107FB03F2F8
:10B620001FFA89F949EA01418A4207D9091903F148
:10B63000FF3022D28A4220D9023B2144891A43EAB0
:10B64000084343E73A4605E7334618E70A4666E704
:10B65000B0409042B5D20CF1FF32002312E73346DE
:10B6600032460FE79A458DD9ACF1020C23448AE7A4
:10B67000B9459AD9023D274498E70346DEE790464C
:10B68000C6E70238214435E71C481D4902680060BE
:10B690008A4200F01D80002100F004B8194B5B586D
:10B6A000435004311848194B42189A42FFF4F6AF40
:10B6B000174A00F003B8002342F8043B154B9A42A6
:10B6C000FFF4F9AFFEF762FD00F036F8FFF7FEBFBA
:10B6D000114E124830601248016821F0706101601B
:10B6E000410201600F4C182020600F490F4808608C
:10B6F0000F48D0F800D0406800470000F04F00200D
:10B70000EFBEADDE6420010800000020EC00002048
:10B71000F0000020F81C0020181002400900000072
:10B7200004000140140C0140000C01404434434427
:10B7300000F0FF1FFFF7FEBF2DE9804893B0F4F73C
:10B74000E7FCDFF8E492B04CD9F8086000232370DE
:10B75000330740F1CA8063681B7A042B00F2C38070
:10B76000DFE803F00303056D9400237ABCE0627AFE
:10B77000A54B002A00F0B78000225A7293F82020CF
:10B78000170700F1B080D97A9A7A01F0070042EAEF
:10B7900000225A621A7B02F03F00400140EAD101C8
:10B7A0009962597B890041EA92119A7B02F001006B
:10B7B00041EA8021D962D97B01F00F00C00140EA43
:10B7C00052021A631A7C02F07F00000140EA111154
:10B7D0005963597C490041EAD212997C01F0030077
:10B7E00042EA40229A63DA7C02F01F00800140EABC
:10B7F0009101D963197DC90041EA5212997D1A64F9
:10B800005A7D01F0070042EA00225A64DA7D02F014
:10B810003F00400140EAD1019964197E890041EA64
:10B8200092115A7E02F0010041EA8021D964997E8A
:10B8300001F00F01C90141EA52021A6551E094F882
:10B840005420714B002A4ED0002283F8542093F8E4
:10B850005620012A47D193F87A20102A84BF10225B
:10B8600083F87A2094F87A10684A0023D8B2884284
:10B8700002F1020235D212F8010C12F8025C40EA21
:10B880000525634840F823500133EFE794F8BC20C6
:10B890005D4B42B3002283F8BC2093F8BD20A82A58
:10B8A00021D193F8D050F5B9574901EB450393F8EE
:10B8B000C00093F8C13003EB0020FEF7EDFD4EA36E
:10B8C000D3E90023FEF788FF4DA3D3E90023FEF759
:10B8D000A5FCFFF769F84F4B43F825000135082D0B
:10B8E000E2D1012300E000232370750408D594F809
:10B8F000F43023B1444B002283F8F4200123237059
:10B9000023783BB1F00505D53F4BD3F8F8301B68E1
:10B910001B689847404D23782A6833B93A4BD3F8CF
:10B92000FC30D31ADB43DB0F00E0012313B1FDF73A
:10B930007BF813E0D4F800315A1CC4F800212BB96D
:10B94000D9F80830190601D5F7F752FAD4F80031C2
:10B95000012B03DD2C4B0022C3F80021F6F714FB6A
:10B96000B9F80C3028602BB1D4F80421821A002ACF
:10B97000C1F29A81244D184499F80570D4F8103119
:10B98000C4F8040105F58E70D4F80861059798474E
:10B9900005F58E70014694F82221F6F781F91F4BC8
:10B9A0001B88002B00F0B380D5F824314FF000083D
:10B9B0001B7805F5947504934746184BB3F800A01F
:10B9C000174BBAF57A7F03D1002243F808202A6189
:10B9D000144AD05F53F80820024443F80820FFF7C8
:10B9E0000DF92A690132012A2A611FD100236860FA
:10B9F0002860AB6045E000BF9A99999999991940E0
:10BA00000000000000707740F00000204801002096
:10BA10006C010020C4010020CC1C0020D81C002098
:10BA2000540200200C0200200C170020D5F800C0A2
:10BA300001926146CDF808C00390FFF729F8019AFA
:10BA400083461046FFF7DAF801465846FFF7DEF95D
:10BA5000DDF808C001466046FFF71CF8039B02466C
:10BA60001146686018460192FFF712F801465846E1
:10BA7000FFF718F9A968FFF70DF8019AE8602A6046
:10BA8000A860674A002302F1540BBAF1010FBB52C0
:10BA900027F80B30DFF898A12CD12869012807DDA1
:10BAA0000138FFF7ABF80146E868FFF7AFF900E0AF
:10BAB000002002F04DF90346049858B10393FFF7B4
:10BAC0009DF8039B01461846FFF7A8FA10B14FF402
:10BAD0007A731AE0534B4FF47A7258F803300A2005
:10BAE00003F5FA7393FBF2F32BF807300F210122D1
:10BAF000F6F734FB0237062F08F1040805F11405A8
:10BB00007FF45BAFBAF80030013BAAF800300023A5
:10BB1000454D05F58E7205F5B871985A595A411A76
:10BB200099520233062BF3D1D5F8783113F0020382
:10BB300000F00083D5F8803105F5C470984705F50D
:10BB4000C470014695F88E21F6F7AAF8B5F8903141
:10BB500005F5C477002B44D00022D5F89401134694
:10BB6000314D37F902C0B5F8901105F5CC7EB1F52D
:10BB7000C87F04BF00214EF803105EF803102A4D61
:10BB800061444EF80310043300210C2BB95281524A
:10BB900002F10202E4D1B5F89031012B1CD1D5F8A5
:10BBA00098314FF4C872C83393FBF2F30380D5F891
:10BBB0009C31C83393FBF2F34380D5F8A031C833EE
:10BBC00093FBF2F2194B1B88D21A8280A6F85C1004
:10BBD000A6F85E10FDF7D4FAB4F89031013BA4F852
:10BBE0009031D9F808305A0740F18780B4F8A42181
:10BBF0000D4B322A1ED1D3F894211188A3F8A61137
:10BC000051889288A3F8A811A3F8AA21B6F85C205D
:10BC1000A3F8AC21B6F85E20A3F8AE210CE000BF7B
:10BC20000C02002054020020F00000200000002040
:10BC3000D81C0020002A3ED00021D4F894510A4696
:10BC4000904837F901C0B0F8A43100F5D87E322B06
:10BC500004BF00234EF802305EF80200894B6044B6
:10BC60004EF80200043200200C2A7852685201F18A
:10BC70000201E5D1B3F8A421012A17D183F8BD212F
:10BC8000022283F8BE21B3F8A62183F8BC012A80E2
:10BC9000B3F8A8216A80B3F8AA21AA80B3F8AC212E
:10BCA000B3F8AE31A6F85C20A6F85E30B4F8A43143
:10BCB000013BA4F8A43194F8BF21724BEAB1D3F848
:10BCC000B001D3F894113225002290FBF5F083F8EF
:10BCD000BF210880D3F8B40190FBF5F04880D3F879
:10BCE000B83193FBF5F5684B1B88ED1A8D80A6F8EB
:10BCF0005C20A6F85E20FDF743FAD4F89431B4F83E
:10BD000088111A8800268A1AA4F88821B4F88A11A2
:10BD10005A88B3468A1AA4F88A219B88B4F88C21E1
:10BD2000D31AA4F88C31F6F72FF9D4F8C0310546B0
:10BD3000C31A18460493FEF75DFFD4F8C4110690A9
:10BD4000FEF7B0FFD4F8C881C4F8C05198F800904D
:10BD5000079035464D4F785FFEF750FF0799FEF785
:10BD6000A1FF09A98851B9F1000F2BD04846FEF771
:10BD700045FF01464FF07E50FFF748F8034619464D
:10BD800007F1B00A4FF07E500393FEF781FE56F89C
:10BD90000A10FEF787FF07F16C010246485F019227
:10BDA000FEF72CFF039BBC371946FEF77BFF019A79
:10BDB00001461046FEF76EFE4AF80600FFF738F916
:10BDC000785304E007F1BC036C37EA5BEA52304F6A
:10BDD0000436EB5F0235062D03FB03BBBAD12A4DB7
:10BDE000642303FB0BFB2B8807F108005B439BFBE1
:10BDF000F3FBABF1490B09A91FFA8BFBF6F75EFBCE
:10BE0000BBF13B0FD8F8046011D9B4F9EC01FEF78F
:10BE1000F5FED4F8E86101463046FFF7FFF8194F08
:10BE200094F8EE31002837D043F0080336E04FF0A5
:10BE30007E513046FEF72EFE01464FF07E50FEF753
:10BE4000E5FF4FF0000A8146DFF848B030465BF866
:10BE50001A10FEF727FF034637F90A000393FEF78F
:10BE6000CDFE039B01461846FEF714FE4946FEF739
:10BE700019FF4BF81A000AF1020ABAF1060FE3D1D2
:10BE8000C3E700BFF0000020000000200C020020EB
:10BE9000C8020020D002002023F008033146D4F865
:10BEA000E40187F8EE3101F051FF0746C4F8F001D4
:10BEB000D4F8E001D4F8E8A100F10046D4F8E40198
:10BEC0000146FEF7EFFE514681465046FEF7EAFE78
:10BED00001464846FEF7DEFD01F03AFF01463046D6
:10BEE00001F034FF0646C4F8F4013846FEF7F6FACE
:10BEF000C3A3D3E90023FEF745FBFEF775FD01F070
:10BF000059FEA4F8F8013046FEF7E8FABCA3D3E9DD
:10BF10000023FEF737FBFEF767FD01F04BFED4F878
:10BF20007831A4F8FA011B0725D5B94809A9F6F715
:10BF3000C5FAD8F808504FF07E512846FEF7AAFD02
:10BF400001464FF07E50FEF761FFDFF8E4A2814624
:10BF50000AF10C0BDAF804102846FEF7A3FE0021C4
:10BF6000FEF798FD4946FEF79DFE4AF8040FDA45B4
:10BF7000F0D1A7483CE0DFF8AC9209A909F1040030
:10BF8000F6F79CFA6868D5F808A00146FEF78AFE25
:10BF9000514683465046FEF785FE01465846FEF759
:10BFA00079FDED68824629462846FEF77BFE01466C
:10BFB0005046FEF76FFD01F0CBFE00210546FFF76E
:10BFC00005F8A0B9D9F804002946FEF71FFF294655
:10BFD000C9F80400D9F80800FEF718FF2946C9F887
:10BFE0000800D9F80C00FEF711FFC9F80C008948C9
:10BFF000F6F71CFB8849A4F808020698FEF752FEE3
:10C0000006F10046054607F10047B4F908020D960F
:10C010000C97FEF7F3FD00F10040FEF75FFA7AA3FC
:10C02000D3E90023FEF7AEFAFEF7DEFC0E90B4F97A
:10C03000D801FEF7E3FD0F90B4F9DA01FEF7DEFD5B
:10C040001090B4F9DC01FEF7D9FD0CA911900FA8EE
:10C05000F6F734FA98F80130704E012B18D1704B76
:10C060001B785F070ED4D6F80C32402093FBF0F01B
:10C07000181AFEF7C3FD1199FEF70CFDFEF7D8FF65
:10C08000C6F80C02D4F80C32402093FBF0F001E02B
:10C09000644B1888FEF7B2FD01461198FEF7F8FCD4
:10C0A000D4F8141211902846FEF7F4FC01462846F5
:10C0B000FEF7ACFED4F81062054631461198FEF743
:10C0C000E7FC01462846FEF7EDFD01463046FEF747
:10C0D000E1FC0646C4F810020F98D4F8187201F07B
:10C0E00069FDD4F824522978F6F71AFB3844C4F8CD
:10C0F00018021098D4F81C7201F05CFD2978F6F74C
:10C100000FFB3844C4F81C023046D4F8207201F00A
:10C1100051FD6978F6F704FB434B049D1A683844D7
:10C120002A441A60D4F82832C4F820020133C4F833
:10C13000283205E0A5F88831A5F88A31A5F88C31B8
:10C14000B4F81C21059EA4F82C22B4F81E21012E5F
:10C15000324BA4F82E220ED1B3F93212B3F92021BA
:10C1600002EB4102032192FBF1F292B2A3F83022DA
:10C17000A3F8322203E0B3F82021A3F83022F5F728
:10C1800003FF2A4B254D1860D4F83832C4F8380222
:10C19000C31AA4F83432FBF703FD94F85032002B95
:10C1A00000F0A980B5F852321E0600F1EC801C4B5D
:10C1B0001B78580740F18C8095F85422194B12B126
:10C1C00095F855223AB10022C4F8582201221A7477
:10C1D000002284F855221B7CD4F80851032B95F8D3
:10C1E00000800E4E05F1040784F8543222D13846FF
:10C1F00006F517714C2201F06FFA5FE0AFF3008093
:10C200003B597E90A9E78140399D52A246DF913F7C
:10C21000EC02002004000020BD378635F00000202D
:10C22000DC1C002000000020D41C0020CC1C0020BE
:10C23000E8020020012B07D106F5177039464C2281
:10C2400001F04AFA002302E0022B02D1012386F812
:10C25000A832012384F8A93284F8AA320023C4F852
:10C26000AC32C4F8B032A64A94F8A832C4F8B4721A
:10C27000D35CA44A1D4484F8B932C4F85822287902
:10C2800084F8B882FEF7BAFC9F49FEF7BFFDC4F8F8
:10C29000BC02A87BFEF7B2FC9C49FEF7B7FDC4F8D0
:10C2A000C002287EFEF7AAFC9949FEF7FBFCC4F801
:10C2B000C402FEF7E3FE00232876AB73B4F85232D3
:10C2C00043F08003A4F85232012384F8C8325AE0C4
:10C2D0000026D5F858023146FEF778FE07460028BA
:10C2E00051D1FCF74DFF8B4B0122C5F8586285F800
:10C2F00054721A7447E0B5F8529219F0800F37D093
:10C3000095F85422834F511E012924D87F49D5F82E
:10C31000C002FEF7C7FCFEF7B1FED5F8B46295F88F
:10C32000B9827D49B04488F80A00D5F8C402FEF706
:10C33000B9FCFEF7A3FE88F814003078FEF75EFC27
:10C340000146FEF7A7FBFEF799FEB37AB070337390
:10C35000337DB37505E0032A03D185F854320123F8
:10C3600001E03B7C013329F080093B74A4F8529230
:10C370006A4B1B78590706D494F8C8321BB1684B36
:10C38000012283F85522D4F80861654D96F8DA80C9
:10C39000B8F1000F53D0B5F852329A074FD0D5F804
:10C3A000E001D5F8E4B10146FEF77CFC594682462F
:10C3B0005846FEF777FC01465046FEF76BFBD5F872
:10C3C000E871824639463846FEF76CFC0146504615
:10C3D000FEF760FBB5F8D09201F0BAFC0146384692
:10C3E000FEF714FD4F490746FEF704FE18BB38461A
:10C3F00001F05CFCD5F8D412FEF754FC01F0DAFB36
:10C40000B0F5617FA8BF4FF46170FEF755F83AA30D
:10C41000D3E90023FEF7E0F9FEF7E6FA01F008FCA5
:10C4200005464046FEF7EAFB2946FEF73BFC01F0D5
:10C43000C1FB80B200E000204844A4F8D002D4F848
:10C440007831374D9B0640F1A180B5F8523203F0A8
:10C450003003002B00F09A8095F8EE31DF0740F1B1
:10C460009580B5F90802FEF7C9FB2F49FEF71AFCC3
:10C47000074601F0DDFB8146384601F065FBD5F843
:10C48000D832804693F803A0B5F9E202274FBAF1FB
:10C49000000F4DD0B5F8DE32CAF100051FFA83FB5C
:10C4A0001BB2C01AF6F71CFCA84203DB5045A8BF1C
:10C4B000504600E02846B4F8DC328344B4F9E00288
:10C4C0009AB21BB21FFA8BFBC01AA4F8DEB201921B
:10C4D000F6F706FCA842019A03DB5045B4BF0546B7
:10C4E00055461544ADB2A4F8DC520FFA8BF0FEF7B6
:10C4F00085FB824628B220E0A2EB0FE5DD169640D0
:10C5000020F200080000A0410000204100007A4411
:10C510005555553F000000209A99993FDC1C00209A
:10C52000F00000208FC2753C35FA8E3CD01C0020F4
:10C53000FEF764FB8246B5F9E002FEF75FFB414679
:10C5400005465046FEF7AEFB494683462846FEF7B1
:10C55000A9FB01465846FEF79BFABC49FEF756FC7C
:10C56000FEF766FD494638805046FEF79BFB414684
:10C5700081462846FEF796FB01464846FEF78AFAB2
:10C58000B249FEF743FCFEF753FD7880B04BB14F44
:10C590001D68301D06F15C0306F15001B7F8F62066
:10C5A000A847AD4B93F800A0BAF1030F13D9B4F923
:10C5B000CE02B4F9E8120028B8BF40426FF063021F
:10C5C000121A914204DB00F164028A42A8BF0A46B3
:10C5D000A4F8E82220E0BAF1010F1DD894F8EA325D
:10C5E0009E4D013B142B00F2FE81DFE813F09B000F
:10C5F000FC01FC016D00A900FC01FC015A01FC01D9
:10C60000FC01FC01FC01FC01C600FC01FC01FC0179
:10C61000FC01FC01B901D101D4F8EC32B4F8D0220C
:10C62000B4F8E682B4F8E492B4F9E8B28C4D04931D
:10C630000026564505F11005D0D210B20192FEF742
:10C64000DDFA55F8101CFEF72DFB84460FFA88F032
:10C65000CDF808C0FEF7D2FA55F8081CFEF722FB09
:10C66000DDF808C001466046FEF714FA84460FFA6A
:10C6700089F0CDF808C0FEF7C1FA55F80C1CFEF79A
:10C6800011FBDDF808C001466046FEF703FA049B83
:10C69000844693F90000CDF808C040420BFB00F03F
:10C6A000FEF7ACFA55F8041CFEF7FCFADDF808C0FA
:10C6B00001466046FEF7EEF9FEF7BAFC6949019AB9
:10C6C00021F816000136B4E702210420F5F7CCFE6C
:10C6D000B4F8E882012100FB08F01FFA80F9042079
:10C6E000F5F7C2FEB4F8E66200FB06901FFA80F987
:10C6F0000420F5F7C7FE4844288102210520F5F7FC
:10C70000B3FE00FB08F001211FFA80F80520F5F7C1
:10C71000ABFE00FB06801FFA80F80520F5F7B2FE9D
:10C7200040440BE005200121F5F79EFEB4F8E862D5
:10C73000704386B20520F5F7A5FE3044688152E1CA
:10C740000020F5F79FFED4F8B063B4F9FA2196F90A
:10C7500006304FF03208534393FBF8F31844288017
:10C760000120F5F78FFE96F90E30B4F9F821534306
:10C7700093FBF8F84044688035E13B4B1B78580741
:10C7800003D4D4F8B4339B880BE0D4F8B413B4F9D1
:10C79000D0220B8849889A4203DB9142B4BF0B46F2
:10C7A0001346EB81EA892F4B1A80D4F8B8331E78F0
:10C7B00066B30220F5F766FE2C4BD3F8B033B3F91D
:10C7C0001020598A904203DB0AB29042B8BF024659
:10C7D000D4F8BC1325484989C2EB010EB4F8C02334
:10C7E0000FFA8EFE0FFA82FCF44501DA164401E0DE
:10C7F00002DD961BA0F8C063B4F9C02393F916308C
:10C800005343642293FBF2F31944A980B4F85222F3
:10C81000164BD1050FD5B3F8CA22EA802A81B3F8A6
:10C82000CE22B3F8CC326A81AB81D4F8B0A3DFF862
:10C830002C8003261CE0B3F8E422EA802A81B3F8B6
:10C84000E822B3F8E6326A81EEE700BF000020413B
:10C85000700000200C170020B01C00205E0000209B
:10C86000E0030020B21C0020DC1C0020F0000020AF
:10C870000AEBC60393F90630B8F90690304609FB77
:10C8800003F9642399FBF3F9A8F80690F5F7FAFD8C
:10C8900001364844072EA8F8060008F10208E7D13F
:10C8A000A1E0BC4B1B785A0703D4D4F8B4339B885F
:10C8B0000BE0D4F8B413B4F9D0220B8849889A421B
:10C8C00003DB9142B4BF0B461346EB81EA89B24BBE
:10C8D000B24E1A80B4F85232DFF8C482DB054FF052
:10C8E00003004FF001010ED5F5F7BEFDB8F8CC926C
:10C8F000022100FB09F01FFA80FA0320F5F7B4FDCE
:10C90000B8F8CA820DE0F5F7AFFDB8F8E69202215B
:10C9100000FB09F01FFA80FA0320F5F7A5FDB8F82F
:10C92000E48200FB08A00121F0800420F5F79CFDC3
:10C9300000FB09F002211FFA80F90420F5F794FDAD
:10C9400000FB089030810320F5F79CFDEB8818442C
:10C95000E8800420F5F796FD2B891844288142E0F1
:10C9600001210420F5F780FDB4F8E662704386B239
:10C9700004202E81F5F786FD304428810121052011
:10C98000F5F772FDB4F8E462704386B26E81D1E6C9
:10C99000B4F8E892032630460221F5F765FD00FB66
:10C9A00009F001211FFA80F83046F5F75DFDC6F168
:10C9B00006037B4923F001030B44B3F8E43200FB88
:10C9C00003801FFA80F825F816803046F5F75AFDE7
:10C9D000404425F816000136072EDCD1704BB3F821
:10C9E000D0226D4B1A80BB68990632D50020F5F72E
:10C9F00049FD288080460120F5F744FD94F8432244
:10CA0000664E6880664B22B3D3F8C423B3F9FAE1CB
:10CA1000127812F0020FB3F9F8211ED0D3F8B03318
:10CA200093F90E1093F906304A435B420EFB03FE66
:10CA3000322192FBF1F26FF0310392B29EFBF3F3DD
:10CA400013449EFBF1FE98447244A6F80080104403
:10CA50007080D4F8B013002316E0D3F8B01391F926
:10CA600006300EFB03FE32239EFBF3FEF044A6F8D5
:10CA7000008091F90E104A4392FBF3F31844E7E764
:10CA8000EA520233102B0CD0E85E31F9232001EB7F
:10CA9000830690427688F3DB32B28242A8BF024618
:10CAA000EEE7D4F8C4331B785A0705D43D4B3A4A15
:10CAB00018781188012321E0394B002693F8C883A8
:10CAC0000423A8F104085FFA88F85FFA88F94FFA9E
:10CAD00089F2D6420ED4324A03F1010A08EB06006D
:10CAE00002EB4303B3F8CA135FFA8AFAC0B2F6F74F
:10CAF00023F953460136042EE9D1D7E7834208D201
:10CB000032F9136009B28E42A8BF314689B20133AF
:10CB1000F4E7BB68D4F8B42303F4805B03F010039C
:10CB200005931C4BB4F9D0631B78D4F8BC7303F0A5
:10CB30000403DBB2D4F8F0E304934FEA4009002386
:10CB40004B4556D0B2F8028008B24045124806DD87
:10CB500030F803C0C1EB0808C44420F803C0BBF19F
:10CB6000000F21D0B7F80AC030F903806645CBBF6B
:10CB7000BEF802009088B2F802A0BEF800A080457E
:10CB8000DFF814C003DBD045B4BF404650462CF854
:10CB9000030024E0DC1C0020B21C00205E0000200A
:10CBA000F0000020B01C002030F903C01088B2F85B
:10CBB0000280844503DBC445B4BF60464046DFF8CD
:10CBC000C88023F80800B88903EB080C864206DA0F
:10CBD000059808B9108800E09088ACF80000049827
:10CBE00028B9284833F800C0274823F800C002338A
:10CBF000A6E7D4F80C34002B54D0244B93F8EA3237
:10CC0000013B142B48D8DFE803F00B4747264B477E
:10CC1000471F47474747472D4747474747262D0068
:10CC2000D4F8EC325B782BB1194B00205989F6F718
:10CC300083F837E0174B1B7803F0040303F0FF0081
:10CC4000002BF1D10146F2E70020E988F6F774F8ED
:10CC500001202989EBE700202989F6F76DF80120EA
:10CC60006989E4E70020E988F6F766F80120298958
:10CC7000F6F762F802206989F6F75EF80320A989C1
:10CC8000D5E700BFE4040020B21C0020F000002023
:10CC90005E000020DC1C0020CB4B9B689B0601D56E
:10CCA000F6F756F8F5F7C5FBC84B1B78002B40F09C
:10CCB0009B82DFF81483D8F808305F0540F1948236
:10CCC00094F81034C24D002B00F08E82F5F7D4FE9C
:10CCD000002800F0898295F81134002B00F084823E
:10CCE000D5F814341B78002B40F04181D5F8180496
:10CCF000F5F7A8FA002840F03A81B64FD5F81C2481
:10CD00003B689A1A7C2A40F23281C5F81C3495F8A7
:10CD10002034013385F82034054605F12400AC4E5B
:10CD2000C0B2F5F74FFB06F5EC7333F91500FDF7CC
:10CD300065FFA94B81461888FDF760FF014648460C
:10CD4000FEF764F8A549FDF7ADFFFEF771F901356F
:10CD500000B2F5F763FB032DDFD13020F5F732FB8E
:10CD60000020F5F75BFBF5F73BFB96F8205415F038
:10CD700003051AD11020F5F725FB2846F5F74EFBE1
:10CD80002120F5F71FFB2846F5F748FB1420F5F79F
:10CD900019FBB6F90802F5F741FB1C20F5F712FB69
:10CDA0002846F5F73BFBF5F71BFB94F82034884D3C
:10CDB0005E0740F0B7800220F5F704FBB5F92204C6
:10CDC0000A2690FBF6F0F5F729FBD8F8083098070B
:10CDD00065D5DFF8108295F8242498F8003040F6E5
:10CDE0003401B2FBF3F24A432A21B2FBF1F2B5F867
:10CDF0002614062091FBF3F903FB19194FEA0919D0
:10CE00001FFA89F949EA02291FFA89F9C2F30322B4
:10CE100049EA0209F5F7D6FA0FFA89F0F5F7FEFAB2
:10CE2000B5F8262498F80030013292B292FBF3F163
:10CE300003FB1123A5F8263495F824344FF06E082F
:10CE400008FB03F8152398FBF3F83A204FF0640A27
:10CE5000F5F7B8FAB8FBFAF94846F5F7DFFA3B20E0
:10CE6000F5F7B0FA0AFB198080B2053090FBF6F0B6
:10CE700000B2F5F7D3FA2820F5F7A4FAD5F828047C
:10CE800090FBF6F000B2F5F7C9FA0420F5F79AFA2C
:10CE9000D5F82C0480F3100000B2F5F7BFFAD4F8EF
:10CEA00078314B4D99063BD50FA9D5F83004F5F7ED
:10CEB000C1FD1320F5F786FABDF93C00F5F7AEFA8F
:10CEC0001B20F5F77FFABDF93E00F5F7A7FA2320FE
:10CED000F5F778FAD5F83034002BACBF4E2053204C
:10CEE000F5F79CFA0FA9D4F83404F5F7A3FD122046
:10CEF000F5F768FABDF93C00F5F790FA1A20F5F756
:10CF000061FABDF93E00F5F789FA2220F5F75AFAE1
:10CF1000D4F83434002BACBF45205720F5F77EFA07
:10CF2000F5F75EFA94F82034282B20D1284B002204
:10CF30003F6883F820244FF47A73B7FBF3F73C255E
:10CF40001720F5F73FFAB7FBF5F6B6FBF5F005FB52
:10CF50001060000200B2F5F761FA1820F5F732FA16
:10CF600005FB167000B2F5F759FAF5F739FAD4F85F
:10CF70001434174D1B78012B40F01481F5F704F899
:10CF8000D5F83834164AC31A9342064640F2A880B0
:10CF900095F82424002385F85A2485F8502495F820
:10CFA000EE2185F83E3485F8403485F85B3485F809
:10CFB000513495F86834920785F8833414D42D23BE
:10CFC00085F884348AE000BF0C170020DB1C0020A9
:10CFD000F0000020081700200000002000007A4424
:10CFE0003F0D030074000020042B8CBF3323322339
:10CFF00085F88434CB48D4F83054DFF860C395FB0F
:10D00000F0F70CFB07584FF0060E0EFB08F8C64B66
:10D0100007EB870798FBF3F903FB198807EB8707F2
:10D020004FFA89F9D4F8341409EB8707BFB291FBA2
:10D03000F0F084F873743F0A84F874740CFB0017E2
:10D040000EFB07F7ED0F84F8725497FBF3F503FB23
:10D050001573642293FBF2F384F87A341B1284F87C
:10D060007B34B4F8963498FBF2F8B3FBF2F202EB9F
:10D07000C202920092B2B4F8983484F87024120A72
:10D0800084F8712484F87C34B4F89A241B0A84F858
:10D090007D340A23B2FBF3F300EB800003F5FA734F
:10D0A0009BB26DB200EB800005EB800084F87E340B
:10D0B0001B0A80B284F87F34B4F89C3484F87584F9
:10D0C000C90F4FEA282884F87804000A84F8768487
:10D0D00084F8771484F8790484F88534C4F83864C3
:10D0E00094F89E84914DB8F1000F0DD1D5F8A404A9
:10D0F000F5F7A8F8012807D902288D4F00F0A08283
:10D10000F5F7A5F801237B74D4F8A824874D002AED
:10D1100048D095F89E743FB1D5F8B03440F6B73199
:10D12000F31A8B420BD83DE00123D5F8A404022169
:10D1300085F89E34F5F772F885F8B47430E095F808
:10D14000AC345BB9D5F8A4040121C5F8A83485F83E
:10D150009E34F5F763F8F5F77AF821E0013BDBB28E
:10D1600085F8AC3495F8B41495F8B50443B901309A
:10D170004B1C85F8B50485F8B434D5F8A4040DE04B
:10D18000134613F8012B0130114485F8B504D5F886
:10D19000A40485F8B414C5F8A8341146F5F764F86A
:10D1A000C4F8B064D4F81434604D1B78022B1BD142
:10D1B000D5F8B834C3B1C5F8BC341B685D4AC5F8AE
:10D1C000C034D5F8C43413449878F6F70DFFD5F879
:10D1D000BC349879F5F74DF8D5F8C4340133092BF0
:10D1E00088BF0023C5F8C434DFF874A1DAF808302A
:10D1F000DD037EF5A6AA94F8C8344C4E002B3EF40D
:10D20000A0AA4D4B1B78002B7EF49BAAF4F7BCFE22
:10D21000D6F8CC340546C31A6FEA0308D6F8D034E2
:10D220004FEAD878C31A6FEA0309D6F8D4344FEA24
:10D23000D979C3EB000B6FEA0B0B4FEADB7BBBF139
:10D24000000F06D1B9F1000F03D1B8F1000F3EF481
:10D2500078AA0027DFF8D4C0FEB2624692F85C35A7
:10D260009E423AD23549DCF8D834B20009681344FA
:10D270006244C2F8DC145988C8050BD48B052AD542
:10D280002F4B1B785E0754BF2E4B2F4B1B68C2F8E9
:10D29000DC3420E019462D4A30460393CDF808C00F
:10D2A000F7F746FCDDF808C0039BBCF8522212F0E9
:10D2B000400F03D030461946254A0AE0900703D5AF
:10D2C00030461946234A04E0D10704D5224A3046A5
:10D2D0001946F7F72DFC0137BCE79E000023B34247
:10D2E00040D01249D1F8D8241A445288520516D594
:10D2F00001F2DC42D0580890B1F9D0037821A0F5B2
:10D300007A7048434FF47A7190FBF1F000F22B10E1
:10D3100040F2671190FBF1F701FB170199520433BA
:10D32000DDE700BF8096980040420F00F00000202B
:10D330000000002020F20008DA1C00205408010838
:10D34000DC1C00202CF2000830F2000834F2000847
:10D350003AF2000840F2000846F20008806967FFD0
:10D360000C170020BBF1000F27D005F5C333A03305
:10D37000C4F8D43494F85D35B54EDBB986F85E3523
:10D38000DAF8083001279B0786F85D7504D5F4F7B5
:10D390003FFD08B186F85E75D4F86035AC4E1B6869
:10D3A0009B68984748B196F85E3543F0020386F8CB
:10D3B0005E3502E0002386F85D3594F85E25A44BC7
:10D3C0001AB9B9F1000F39D15CE093F85D7537B146
:10D3D00093F86415013101F0030183F86415002608
:10D3E0009B4BF1B293F85C058842EAD9D3F8D80494
:10D3F00089000844408800061ED593F8640567B983
:10D4000020B9D00718D50B44924912E0012813D94E
:10D41000900711D50B4490490BE020B9D0070BD5EC
:10D420000B448E4905E0012806D9900704D50B442A
:10D430008B490968C3F8DC140136D1E7B4F9CC3262
:10D44000B4F9CA223221002AB8BF5242002BB8BF19
:10D450005B4293FBF1F392FBF1F1DBB2C9B28B4279
:10D4600038BF0B467F4A0BB192FBF3F22A44C4F853
:10D47000D02494F86525764B0AB9012200E00022F9
:10D4800083F8652594F86525714B22B9764AC3F86F
:10D490006825002009E0714AF9E7D3F8D814940010
:10D4A0000E197688760607D40130694BC2B293F81C
:10D4B0005C159142F1D89FE0B3F9CA62322E21DDAA
:10D4C00011F8227093F86CE507F00F0CF445D3F8CF
:10D4D000686508DC93F86DE5BEEB171F03DC234499
:10D4E0003468C3F8DC445A4B11F8224093F86EC5F7
:10D4F00004F00F0EE6452DDB93F86D75B7EB141FA6
:10D5000028DC22E0323625DA11F8227093F86CE537
:10D5100007F00F0CF445D3F8686508DC93F86FE565
:10D52000BEEB171F03DB23443468C3F8DC44484BCD
:10D5300011F8224093F86EC504F00F0EE64509DBA2
:10D5400093F86F75B7EB141F04DB346803EB8203A9
:10D55000C3F8DC443E4BB3F9CC42322C21DD11F848
:10D56000227093F86C6507F00F0EB645D3F8684546
:10D5700009DC93F86DE5BEEB171F04DC276803EBAD
:10D580008203C3F8DC7411F8223003F00F01B142BA
:10D590008ADC2F4E96F86F15B1EB131F84DB3346F0
:10D5A00024E0323480DA11F8227093F86E6507F0C7
:10D5B0000F0EB645D3F8684509DB93F86DE5BEEB71
:10D5C000171F04DC276803EB8203C3F8DC7411F82F
:10D5D000223003F00F01B142FFF666AF1C4F97F8FF
:10D5E0006F15B1EB131FFFF65FAF3B4603EB8202F3
:10D5F0002368C2F8DC3457E7B8F1000F1CD093F869
:10D60000712593F8701505F543458818013890FB8E
:10D61000F2F402FB140083F87315013183F87205EC
:10D6200091FBF2F002FB10125035D2B2C3F8CC5489
:10D6300083F8742583F87025F7F7ADFFFEF781B8FE
:10D640007B7C9BB1C5F8A06487F811805CE500BFC6
:10D65000F00000204CF2000850F2000854080108C5
:10D6600054F20008400D030058F20008D5F8A03429
:10D67000F31AB3F57A6FFFF447AD0123D5F8A4048C
:10D680007B74F4F7DAFD0746D5F8A404F4F7D5FD6A
:10D69000802F7FF439AD8A2802D08E280DD033E553
:10D6A000D5F878319F067FF52FAD95F89E34002B85
:10D6B0007FF42AAD05F2694306E095F89E34002B0D
:10D6C0007FF422AD05F23C43C5F8A8342D2385F83C
:10D6D000AC3419E5AFF3008010B50023934203D0BA
:10D6E000CC5CC4540133F9E710BD024403469342B5
:10D6F00002D003F8011BFAE7704700000D4B70B52C
:10D700001D680022845C2B195B7803F00303012B56
:10D710008B5C08BF2034EE18767806F00306012EE5
:10D7200008BF2033E41A02D10132002BEAD120468F
:10D7300070BD00BF8000002010B50446224613785B
:10D740000134002BFAD1CC5CD4540133002CFAD133
:10D7500010BDC9B2024610F8013B1BB18B42F9D192
:10D76000104670470029FBD018467047034613F84F
:10D77000012B002AFBD1181A013870470F4BF0B566
:10D780001E680023934215D0C55C7419647804F0B8
:10D790000304012CCC5C08BF203537197F7807F0D3
:10D7A0000307012F08BF20342D1B04D10133002CA7
:10D7B000E8D100E000252846F0BD00BF8000002031
:10D7C00010B5034632B111F8014B013A03F8014B91
:10D7D000002CF7D11A44934203D0002103F8011B17
:10D7E000F9E710BD30B503780BB1044604E00B78BF
:10D7F000002B18BF002030BD22461078013438B10C
:10D800000023C85C28B1D55C8542F5D10133F8E727
:10D8100030BD104630BD00210A2200F001B92DE9CB
:10D82000F04E82468B461F46144612B90020BDE8D2
:10D83000F08E002BFAD00026A642F7D2A5196D086B
:10D8400007FB05B950464946089B9847002802DB6C
:10D8500003D06E1C25462C46EEE74846BDE8F08E08
:10D86000174B2DE9F0411D680646AC6D0F46FCB91B
:10D87000502000F0E3F8A8658460AB6D046044605C
:10D880001C61DC60AB6D9C615C61AB6DDC629C62B9
:10D89000AB6D5C631C63AB6DDC639C63AB6D5C6404
:10D8A0001C64AB6DDC649C64AB6D1C77AB6D5C621F
:10D8B00030463946AA6D0123BDE8F04100F002B8B8
:10D8C000E4000020F0B508B9106828B3044614F845
:10D8D000015B0F4617F8016B3EB1B542FAD10BB1AF
:10D8E0002046F3E714600370F0BD4DB9156028467B
:10D8F000F0BD17F8016BAE4207D0002EF9D11C46DF
:10D90000234613F8015B0F46F3E715B100212170A0
:10D9100000E02B461360F0BDF0BD000084463F4898
:10D920002DE9F04FD0F800800E46344614F8015B24
:10D9300008EB0500407800F0080000F0FF0708B190
:10D940002646F2E72D2D03D1B41C7578012703E09C
:10D950002B2D04BF7578B41C33F010000DD1302D81
:10D9600008D1207800F0DF00582851D165781023C5
:10D97000023402E0002B08BF0A23002F0CBF6FF017
:10D98000004A4FF0004ABAFBF3F903FB19AA00263C
:10D99000304608EB050B9BF801B01BF0040F01D0DB
:10D9A000303D0BE01BF0030B1BD0BBF1010F14BF8C
:10D9B0004FF0570B4FF0370BCBEB05059D4210DABC
:10D9C000B6F1FF3F0AD0484506D801D1554503DCE2
:10D9D00003FB0050012601E04FF0FF3614F8015B15
:10D9E000D7E7731C0CD1002F4FF022030CBF6FF050
:10D9F00000404FF00040CCF800302AB9BDE8F08F6D
:10DA000007B1404242B106B1611E1160BDE8F08F1E
:10DA1000002B08BF0823B0E7BDE8F08F800000208E
:10DA200030B51346044A05460C461068294622467E
:10DA3000BDE83040FFF772BFE4000020024B014612
:10DA4000186800F003B800BFE400002070B5CD1CDA
:10DA500025F0030508350C2D38BF0C25002D064692
:10DA60003FDB8D423DD3214B1C6818462146A1B1B6
:10DA70000B685B1B0ED40B2B03D90B60CC18CD505D
:10DA80001FE08C4202D1626802601AE04B6863605A
:10DA90000C4616E00C464968E9E7154C23681BB9AB
:10DAA000304600F027F820602946304600F022F882
:10DAB000431C014615D0C41C24F0030484420AD13F
:10DAC000256004F10B00231D20F00700C31A0BD0C2
:10DAD0005A42E25070BD3046611A00F00BF8013036
:10DAE000EED10C233360002070BD00BFEC1C002081
:10DAF000E81C002038B5064C002305460846236084
:10DB000000F008F8431C02D1236803B12B6038BD34
:10DB1000F41C0020094A136863B11844694688421E
:10DB200002D8106018467047054B0C221A604FF05F
:10DB3000FF307047034B1360EFE700BFF01C00207D
:10DB4000F41C0020F81C002000B5194A20F0004306
:10DB5000934283B0014617DDB3F1FF4F04DBFCF7BE
:10DB600097FF03B05DF804FB694600F037FB00F057
:10DB70000302012A0098019911D0022A0AD09AB111
:10DB8000012201F0EFF8ECE7002100F0EFFC03B018
:10DB90005DF804FB00F0EAFC00F10040E1E701F071
:10DBA000E1F800F10040DCE700F0E0FCD9E700BF5D
:10DBB000D80F493F30B5C0F3C754A4F17F031E2BE3
:10DBC00083B0014620DC581C1BDB162B4FEAD175B5
:10DBD00009DDC1F3160040F40000963CA04005B1F9
:10DBE000404203B030BD114B53F825402046FCF7AE
:10DBF00051FF019001982146FCF74AFF20F00043B5
:10DC000033B9002003B030BDFDF712FA03B030BDC8
:10DC1000C0F31604C0F3C75044F40004C0F19600EA
:10DC200024FA00F0002DDCD0DAE700BF501C010818
:10DC300000B51D4A20F00043934283B0014618DD31
:10DC4000B3F1FF4F04DBFCF723FF03B05DF804FBE7
:10DC5000694600F0C3FA00F00300012818D002283A
:10DC60000ED0D0B10098019900F080FC00F1004086
:10DC7000EBE70021002201F075F803B05DF804FB2A
:10DC800000980199012201F06DF800F10040DCE7F5
:10DC90000098019900F06AFCD7E7009801990122E9
:10DCA00001F060F8D1E700BFD80F493F70B58AB0E6
:10DCB000054600F09BF8224C064694F900300133EB
:10DCC00003D0284601F02CFA10B930460AB070BDD6
:10DCD000284601F0DBF94FF07E51FDF79FF900284F
:10DCE000F3D018490122002328460092089301919D
:10DCF000FCF7F4FB02460B461348CDE90423CDE9BB
:10DD0000022301F0A7F894F90030CDE90601022BB7
:10DD10000BD0684601F09CF838B1089B53B9DDE997
:10DD20000601FCF761FE0AB070BD01F073FA212311
:10DD30000360F2E701F06EFA089B0360EFE700BFB3
:10DD4000E8000020581C0108601C010800F0B6B96A
:10DD500070B58AB0054600F0B5FB224C064694F932
:10DD60000030013308D0284601F0DAF920B1284606
:10DD70000021FDF735F910B930460AB070BD1A49D7
:10DD8000012200232846019100920893FCF7A6FB8C
:10DD90002478CDE90401CDE902017CB900220023F9
:10DDA000CDE90623684601F053F888B1089BA3B972
:10DDB000DDE90601FCF718FE0AB070BD0020002165
:10DDC00002460B46FCF708FD022CCDE90601E9D11D
:10DDD00001F020FA21230360E8E701F01BFA089B19
:10DDE0000360E5E7E8000020641C0108F8B520F0B6
:10DDF0000043B3F17E5F044610D008DCB3F17C5FD2
:10DE000011DAB3F10C5F00F384809D48F8BD014640
:10DE1000FCF73EFE0146FCF7F9FFF8BD002840F391
:10DE2000CD800020F8BD0028C0F2CA8001464FF026
:10DE30007E50FCF72DFE4FF07C51FCF733FF04467B
:10DE400000F040FB8F4906462046FCF72BFF8E4929
:10DE5000FCF720FE2146FCF725FF8C49FCF718FE55
:10DE60002146FCF71FFF8A49FCF714FE2146FCF708
:10DE700019FF8849FCF70CFE2146FCF713FF864981
:10DE8000FCF708FE2146FCF70DFF844905462046B5
:10DE9000FCF708FF8249FCF7FBFD2146FCF702FF77
:10DEA0008049FCF7F7FD2146FCF7FCFE7E49FCF7B4
:10DEB000EFFD2146FCF7F6FE4FF07E51FCF7EAFD40
:10DEC00001462846FCF7A2FF3146FCF7EBFE26F49C
:10DED0007F6525F00F05074629462846FCF7E2FE38
:10DEE00001462046FCF7D4FD294604463046FCF79F
:10DEF000D1FD01462046FCF789FF01463846FCF774
:10DF0000C9FD01462846FCF7C5FD0146FCF7C2FDE8
:10DF1000F8BD0146FCF7C6FE5A490546FCF7C2FEAD
:10DF20005949FCF7B7FD2946FCF7BCFE5749FCF7F9
:10DF3000AFFD2946FCF7B6FE5549FCF7ABFD294677
:10DF4000FCF7B0FE5349FCF7A3FD2946FCF7AAFEF7
:10DF50005149FCF79FFD2946FCF7A4FE4F490646B0
:10DF60002846FCF79FFE4E49FCF792FD2946FCF738
:10DF700099FE4C49FCF78EFD2946FCF793FE4A4971
:10DF8000FCF786FD2946FCF78DFE4FF07E51FCF72D
:10DF900081FD01463046FCF739FF01462046FCF77B
:10DFA00081FE01464148FCF773FD01462046FCF71F
:10DFB0006FFD01463E48FCF76BFDF8BD3D48F8BDDE
:10DFC0004FF07E51FCF766FD4FF07C51FCF76AFE86
:10DFD0002C490446FCF766FE2B49FCF75BFD214605
:10DFE000FCF760FE2949FCF753FD2146FCF75AFE79
:10DFF0002749FCF74FFD2146FCF754FE2549FCF765
:10E0000047FD2146FCF74EFE2349FCF743FD214620
:10E01000FCF748FE0646204600F054FA1F49054624
:10E020002046FCF73FFE1E49FCF732FD2146FCF777
:10E0300039FE1C49FCF72EFD2146FCF733FE1A4938
:10E04000FCF726FD2146FCF72DFE4FF07E51FCF734
:10E0500021FD01463046FCF7D9FE2946FCF722FE99
:10E060001249FCF715FD01462846FCF713FD014651
:10E07000FCF710FD01461048FCF70AFDF8BD00BF93
:10E08000DB0FC93F08EF1138047F4F3A4611243D9A
:10E09000A80A4E3E90B0A63EABAA2A3E2EC69D3D93
:10E0A0006133303F2D57014039D119406821A233E7
:10E0B000DA0FC93FDB0F4940DA0F494021F0004237
:10E0C000B2F1FF4FF8B5044614DC20F00045B5F17D
:10E0D000FF4F06460EDCB1F17E5F3AD08F1707F096
:10E0E000020747EAD07755B9022F2FD0032F2FD13F
:10E0F0003148F8BD08462146FCF7CCFCF8BDFAB122
:10E10000B2F1FF4F29D0B5F1FF4F19D0AA1AD2159D
:10E110003C2A19DC002938DB2046FCF777FE00F0AA
:10E12000B5FF00F09DFE012F2CD0022F22D0002F32
:10E130002FD02249FCF7AEFC2149FCF7A9FCF8BD21
:10E14000002E15DB1F48F8BD1E48ECE71C48F8BD43
:10E15000F8BDBDE8F84000F083BEB5F1FF4F19D01F
:10E16000022FF3D0032FC3D0012F1BD00020F8BD06
:10E170001548F8BD1149FCF78DFC01461048FCF725
:10E1800087FCF8BD00F10040F8BD3C32C4DA002045
:10E19000C9E7F8BD022F0CD0032F08D0012F04D0FF
:10E1A0000A48F8BD4FF00040F8BD0948F8BD0948DD
:10E1B000F8BD0948F8BD00BFDB0F49C02EBDBB3319
:10E1C000DB0F4940DB0FC93FDB0FC9BFDB0F493F06
:10E1D000DB0F49BFE4CB16C0E4CB16402DE9F04F6E
:10E1E000AB4A20F00044944289B006460D4664DDF7
:10E1F000A84A94421CDC0028A74940F3EC80FCF7B5
:10E2000047FCA64B24F00F049C42064664D0A44968
:10E21000FCF73EFC014628603046FCF739FCA0497B
:10E22000FCF736FC01236860184609B0BDE8F08FA2
:10E230009C4A944262DDB4F1FF4F46DAE715863F0F
:10E24000A4EBC7542046FCF7F3FEFCF7D7FC0346CB
:10E25000014620460593FCF71BFC4FF08741FCF775
:10E2600021FD8046FCF7E4FEFCF7C8FC01460446AD
:10E2700040460694FCF70CFC4FF08741FCF712FD7A
:10E2800000210790FCF7A2FE002800F0C580204680
:10E290000021FCF79BFE002814BF012302238248C3
:10E2A0000221019000913A4605A8294600F022FA81
:10E2B000002EC0F2A780034603E00022286000235E
:10E2C0004A60184609B0BDE8F08F0146FCF7E0FB54
:10E2D000002368602860F4E77449FCF7D9FB7449AF
:10E2E0000446FCF7D5FB014628602046FCF7D0FB2E
:10E2F0006F49FCF7CDFB01236860E2E700F0C6FE42
:10E300006C490746FCF7CEFC4FF07C51FCF7C2FB92
:10E31000FCF78EFE8246FCF771FC5F498346FCF7F2
:10E32000C1FC01463846FCF7B3FB5D4980465846C0
:10E33000FCF7B8FCBAF11F0F81464946404618DC8D
:10E340005D4B0AF1FF3253F8223024F0FF029A426B
:10E350000FD0FCF79DFB07462F6039464046FCF77F
:10E3600097FB4946FCF794FB002E686056DB53464A
:10E37000A7E7FCF78DFBE315C0F3C7529A1A082AEA
:10E380000746E9DD494958460393FCF78BFC0746ED
:10E3900039464046FCF77CFB044621464046FCF7E4
:10E3A00077FB3946FCF774FB414907465846FCF7B2
:10E3B00079FC3946FCF76CFB814649462046FCF760
:10E3C00067FB039BC0F3C7529B1A192B074641DC1E
:10E3D0002860A046C1E7FCF75DFB304B24F00F043A
:10E3E0009C42064623D02E49FCF754FB0146286088
:10E3F0003046FCF74DFB2A49FCF74CFB4FF0FF334E
:10E4000068605EE795E80C0003F1004102F100420C
:10E4100043422A60696054E7032340E707F100475D
:10E4200000F100402F606860CAF1000349E71F490E
:10E43000FCF730FB1E490446FCF72CFB0146286024
:10E440002046FCF725FB1A49FCF724FB4FF0FF336D
:10E45000686036E719495846FCF724FC07463946F8
:10E460002046FCF715FB804641462046FCF710FB92
:10E470003946FCF70DFB124904465846FCF712FCDE
:10E480002146FCF705FB81464946404661E700BF4F
:10E49000D80F493FE3CB1640800FC93FD00FC93F8B
:10E4A00043443537800F4943EC1C0108004435379D
:10E4B00008A3852E84F9223F6C1C010800A3852E39
:10E4C00032318D2420F00042B2F1FF4FF8B50446FE
:10E4D00003462DD25AB300283DDBB2F5000F4FEAB8
:10E4E000E0502CD37F38C3F31603C20743F4000374
:10E4F00048BF5B00002740105B003E4619244FF0E8
:10E500008072B5189D4202DC5B1BAE181744013CBB
:10E510004FEA43034FEA5202F3D113B107F001036C
:10E520001F447F1007F17C5707EBC050F8BDF8BDC2
:10E530000146FCF7B7FB2146FCF7ACFAF8BD14F432
:10E5400000020FD15B00190202F10102FAD5C2F1FB
:10E5500001021044C6E70146FCF79AFA0146FCF7AF
:10E5600055FCF8BD01221044BCE700BF2DE9F8437B
:10E5700020F00046B6F1485F05460F4649DAFCF741
:10E5800057FD002800F09D8029462846FCF78AFBAD
:10E590004E490446FCF786FB4D49FCF77BFA2146C1
:10E5A000FCF780FB4B49FCF773FA2146FCF77AFB3A
:10E5B0004949FCF76FFA2146FCF774FB4749FCF721
:10E5C00067FA2146FCF76EFB4549FCF763FA2146E2
:10E5D000FCF768FB804620464FF07C51FCF762FB5D
:10E5E000414606462046FCF75DFB39460446284670
:10E5F000FCF758FB01462046FCF74AFA0146304634
:10E60000FCF746FA01464FF07E50FCF741FABDE8B0
:10E61000F8830146FCF746FB2C490446FCF742FB15
:10E620002B49FCF737FA2146FCF73CFB2949FCF75C
:10E630002FFA2146FCF736FB2749FCF72BFA214637
:10E64000FCF730FB2549FCF723FA2146FCF72AFBAF
:10E650002349FCF71FFA2146FCF724FB214B804697
:10E660009E42B8DD204B9E4227DC06F17F463146B4
:10E670004FF07E50FCF70CFA814620464FF07C515B
:10E68000FCF710FB3146FCF703FA414606462046EC
:10E69000FCF708FB394604462846FCF703FB014615
:10E6A0002046FCF7F5F901463046FCF7F1F9014642
:10E6B0004846FCF7EDF9BDE8F883DFF834900B4EDF
:10E6C000DBE74FF07E50BDE8F88300BF4ED747AD83
:10E6D000F6740F317CF29334010DD037610BB63AEA
:10E6E000ABAA2A3D9999993E0000483F0000903E10
:10E6F0000000383F2DE9F04FDFB00B93013B029350
:10E70000D31E48BF131DB84C06466898DB1054F85A
:10E71000204023EAE3730C93DB4302EBC30308942A
:10E720000693089C029B0C9A1D190991C3EB0207E2
:10E730001DD4699C3D4404EB870901354FF0000866
:10E7400022AC0AE059F80800FCF758FA0137AF424A
:10E7500044F8080008F1040809D0002FF2DA013764
:10E760000020AF4244F8080008F10408F5D1089AE7
:10E77000002AC0F2DF82089A0B9B02F101089C007C
:10E7800022AF4FEA880827440025029A002AC0F2E7
:10E79000F28105EB070B4FF000094FF0000A56F825
:10E7A00009005BF8041DFCF77DFA01465046FCF7B2
:10E7B00071F909F10409A1458246F0D14AA840F84F
:10E7C00005A004354545E0D1089A0EAB03EB820362
:10E7D0000D9391464FEA89030793079A5EAB134462
:10E7E000B9F1000F53F850AC23DD0DF134084AAFF6
:10E7F000174490440DAD4FF06E515046FCF752FA5D
:10E80000FCF716FCFCF7FAF94FF087418346FCF75A
:10E8100049FA01465046FCF73BF9FCF709FC59461A
:10E8200045F8040F57F8040DFCF734F945458246C6
:10E83000E1D15046069900F08DFC4FF07851054625
:10E84000FCF730FA00F026FC4FF08241FCF72AFA80
:10E8500001462846FCF71CF90546FCF7E9FB824611
:10E86000FCF7CCF901462846FCF712F9069A8046D7
:10E87000002A40F3678109F1FF310EA850F82130DA
:10E88000C2F1080043FA00F202FA00F01B1A0698DF
:10E890009244C0F1070743FA07F70EA840F8213069
:10E8A000002F32DDB9F1000F0AF1010A40F3758142
:10E8B0000EAB079A19461144002507E0C2F5807097
:10E8C00012B143F8040C01258B420BD053F8042BF2
:10E8D000002DF3D0C2F1FF028B4243F8042C4FF01D
:10E8E0000105F3D1069B002B0DDD012B00F03281D9
:10E8F000022B08D109F1FF330EA951F8232002F0B1
:10E900003F0241F82320022F70D040460021FCF73F
:10E910005DFB002800F08380089A09F1FF35AA42C8
:10E920000DDC079A0EAB0D981344002253F8041D1A
:10E93000834242EA0102F9D1002A40F0E481089BB7
:10E940000EA85A1E50F82230002B40F0F18100EB47
:10E950008202012352F8041D01330029FAD04B44EE
:10E9600099450A933DDADDF82CA022AACA44DDF8C5
:10E97000308002EB8A02C844C9EB0309131D0392DD
:10E980000593699A079B4FEA89094AAF02EB880809
:10E99000CDF810901F44002558F8040FFCF72EF90D
:10E9A000029B039A002B50514FF0000B13DBDDF854
:10E9B00014A04FF00009AA4456F809005AF8041DA3
:10E9C000FCF770F901465846FCF764F809F10409B0
:10E9D000A1458346F0D1049A0435954247F804BF17
:10E9E000DAD1DDF82890F5E60420010841464FF021
:10E9F0007E50FCF74DF88046002D86D006994FF0EA
:10EA00007E5000F0A7FB01464046FCF741F88046E7
:10EA100040460021FCF7DAFA00287FF47DAF069B20
:10EA200040465942CDF808A000F094FB4FF08741D2
:10EA30000446FCF7E9FA002800F07F814FF06E51A0
:10EA40002046FCF72FF9FCF7F3FAFCF7D7F84FF064
:10EA500087410546FCF726F901462046FCF718F8E1
:10EA6000FCF7E6FA0EAB43F829002846FCF7E0FA7B
:10EA7000069C09F1010508340EA9069441F8250009
:10EA800006994FF07E5000F065FB002D04464FDBE9
:10EA90006E1C4FEA8508C6EB867A0DF138094AAB41
:10EAA000C1444FEA8A0A98444FF0000B59F80B0012
:10EAB000FCF7A4F82146FCF7F5F84FF06E5148F842
:10EAC0000B002046FCF7EEF8ABF1040BD3450446EF
:10EAD000ECD1DFF88C92DDF820A00024B34603953A
:10EAE0000497BAF1000FB8BF002515DB00263746A2
:10EAF000002501E0A7420FDC58F8061059F806007F
:10EB0000FCF7D0F801462846FBF7C4FF0137BA45A9
:10EB1000054606F10406EDDA5EA800EB8403013435
:10EB2000A345A8F1040843F8A05CDAD1039D049F33
:10EB3000689C032C00F29880DFE814F0CB009C0066
:10EB40009C00310010D109F1FF330EA951F8237058
:10EB50003F12A5E609F1FF330EA850F8232002F07A
:10EB60007F0240F82320CEE64FF07C51FCF74CFAB0
:10EB700058B90746C9E64FF0000A4AA840F805A070
:10EB8000043545457FF401AE1EE6B9F1000F4FF0A4
:10EB900002070AF1010A3FF78BAE0025A2E6002D1D
:10EBA00040F3DC804FEA850B5EAB36AE05F1FF3AF1
:10EBB0005B4406EB8A0A53F8A08C54465B4635AAA0
:10EBC000BB462F4600E0C84654F804594146284643
:10EBD00001920093FBF75EFF814649462846FBF70A
:10EBE00057FF4146FBF756FF019AC4F80490944240
:10EBF000A060009BE7D13D46012D5F469B4640F358
:10EC0000AD805EAB9B445BF8A04C00E044465AF8F4
:10EC1000049921464846FBF73DFF80464146484659
:10EC2000FBF736FF2146FBF735FF5645CAF804804F
:10EC3000CAF80800EAD16C1C06EB840400200836F0
:10EC400054F8041DFBF726FFB442F9D1002F7ED003
:10EC5000369A379B099C00F1004002F1004203F113
:10EC60000043A06022606360029A02F007005FB078
:10EC7000BDE8F08F002DB8BF00200ADB36AE6C1C5B
:10EC8000002006EB840454F8041DFBF703FFB44294
:10EC9000F9D1002F35D000F10043099C01462360D3
:10ECA0003698FBF7F5FE002D08DD36AC04EB850544
:10ECB00054F8041FFBF7EEFEAC42F9D10FB100F19E
:10ECC0000040099A5060029A02F007005FB0BDE868
:10ECD000F08F002D39DB6C1C36AE002006EB84046F
:10ECE00054F8041DFBF7D6FEB442F9D10FB100F180
:10ECF0000040099A1060029A02F007005FB0BDE878
:10ED0000F08F0346C9E7069A0EAC54F82530083A4E
:10ED1000CDF808A00692002B7FF4B2AE04EB850379
:10ED200053F8041D013D083A0029F9D00692A7E6E0
:10ED3000012314E60B9B9C0046E52046FCF778F97E
:10ED40000EAA4D4642F829009AE60020CEE7099C1B
:10ED5000369A379BA0602260636085E7002075E7E4
:10ED6000102001082DE9F84320F00043B3F1485F7B
:10ED700004460F46904603DAFCF75AF9002857D0AC
:10ED800021462046FBF78EFF21460546FBF78AFF0A
:10ED9000294906462846FBF785FF2849FBF778FEF8
:10EDA0002946FBF77FFF2649FBF774FE2946FBF750
:10EDB00079FF2449FBF76CFE2946FBF773FF2249D4
:10EDC000FBF768FE8146B8F1000F22D038464FF0BD
:10EDD0007C51FBF767FF494680463046FBF762FFF0
:10EDE00001464046FBF754FE2946FBF75BFF3946D8
:10EDF000FBF74EFE154905463046FBF753FF01462B
:10EE00002846FBF747FE01462046FBF741FEBDE8DA
:10EE1000F88349462846FBF745FF0C49FBF738FEC7
:10EE20003146FBF73FFF2146FBF734FEBDE8F88390
:10EE30002046BDE8F88300BFD3C92E2F342FD73228
:10EE40001BEF3836010D50398988083CABAA2A3EA1
:10EE50000020704700200149704700BF0000F87F84
:10EE60002DE9F04120F00045B5F1A14F04460646DA
:10EE700008DBB5F1FF4F6FDC002840F3A0806F483E
:10EE8000BDE8F0816E4B9D4277DCB5F1445F68DBF5
:10EE90004FF0FF3721462046FBF704FF014680462E
:10EEA000FBF700FF67490546FBF7FCFE6649FBF7E9
:10EEB000F1FD2946FBF7F6FE6449FBF7EBFD294619
:10EEC000FBF7F0FE6249FBF7E5FD2946FBF7EAFE9A
:10EED0006049FBF7DFFD2946FBF7E4FE5E49FBF7DF
:10EEE000D9FD4146FBF7DEFE5C4980462846FBF72C
:10EEF000D9FE5B49FBF7CCFD2946FBF7D3FE594908
:10EF0000FBF7C6FD2946FBF7CDFE5749FBF7C0FDD1
:10EF10002946FBF7C7FE5549FBF7BAFD2946FBF723
:10EF2000C1FE7B1C014640464CD0FBF7B3FD214699
:10EF3000FBF7B8FE4E4B4F4D53F82710FBF7A8FDDB
:10EF40002146FBF7A5FD014655F82700FBF7A0FD7C
:10EF5000002E30DBBDE8F0810146FBF79BFDBDE8EC
:10EF6000F0814549FBF796FD4FF07E51FCF756F8CE
:10EF700000288DD02046BDE8F08100F087F83F4B97
:10EF800004469D4229DCA3F5D0039D4244DC0146A2
:10EF9000FBF780FD4FF07E51FBF77AFD4FF080418B
:10EFA00005462046FBF776FD01462846FBF72EFF77
:10EFB000002704466EE700F10040BDE8F0813048CC
:10EFC000BDE8F081FBF766FD2146FBF76BFE0146CD
:10EFD0002046FBF75DFDBDE8F0812A4B9D4214DC25
:10EFE0004FF07F51FBF754FD4FF07F51054620460F
:10EFF000FBF758FE4FF07E51FBF74CFD01462846CB
:10F00000FBF704FF0227044644E701461E48FBF7CE
:10F01000FDFE032704463DE74FF07E51FBF738FD28
:10F020004FF07E5105462046FBF734FD0146284649
:10F03000FBF7ECFE012704462CE700BFDB0FC93FBE
:10F04000FFFFDF3ED769853C59DA4B3D356B883D84
:10F050006E2EBA3D2549123EABAAAA3E21A215BD8D
:10F060006BF16E3D95879D3D388EE33DCDCC4C3E9A
:10F070003C2001084C200108CAF24971FFFF973F6C
:10F08000DB0FC9BFFFFF1B40000080BF20F0004026
:10F09000704700BF2DE9F04120F00047FD0D7F3D96
:10F0A000162D064613DC002D80461BDB194F2F4121
:10F0B000074214D01849FBF7EDFC0021FBF7AEFF27
:10F0C00068B1002E1BDB28EA0700BDE8F081B7F12C
:10F0D000FF4F04D30146FBF7DDFCBDE8F08130466D
:10F0E000BDE8F0810C49FBF7D5FC0021FBF796FF4A
:10F0F0000028F4D0002E08DB0020BDE8F0814FF49A
:10F10000000343FA05F5A844DDE7002FE7D00348E4
:10F11000BDE8F081FFFF7F00CAF24971000080BFA7
:10F1200030F0004001D102207047A0F50003B3F198
:10F13000FE4F01D204207047054B421E9A4201D86F
:10F1400003207047B0F1FF4358425841704700BF59
:10F15000FEFF7F0038B530F00044024603460D46FE
:10F1600014D0B4F1FF4F0DD2B4F5000F0FD3E40D5E
:10F170002C44FE2C2EDC002C1DDD23F0FF4343EA43
:10F18000C45038BD0146FBF785FC38BD38BD4FF093
:10F190009841FBF787FD194B02469D4207DBC0F300
:10F1A000C7540346193CE3E7154800F02DF814490D
:10F1B000FBF778FD38BD14F1160F13DA4CF250331B
:10F1C0009D421146F0DD0F4800F01EF80D49FBF797
:10F1D00069FD38BD11460B4800F016F80949FBF7E8
:10F1E00061FD38BD04F1190023F0FF4343EAC0502C
:10F1F0004FF04C51FBF756FD38BD00BFB03CFFFF50
:10F200006042A20DCAF2497101F0004120F00040B5
:10F2100008437047014B1868704700BFE4000020A6
:10F220000001746564666D6A69736C67780000FF3D
:10F23000F00000FF010B020D0A03050B030D0A038A
:10F240000A0B040D0A03080B040D0A03000000FF5B
:10F25000D20000FF5A0000FF1E0000FF4A0100FF1D
:10F260002C0100FF0E0100FFB40000FF960000FF1C
:10F270003C0000FF0000FFFF5408010874F2000882
:10F280004CF2000858F2000870F2000854F200082E
:10F290002CF200086CF2000868F2000850F2000836
:10F2A00030F2000864F2000860F200085CF2000826
:10F2B00000000000000C014008001002000801409E
:10F2C00000801402000C0140040014020000000041
:10F2D000000000000301000014F900080400000011
:10F2E000D4F800080400000094F8000802010000AF
:10F2F00074F8000800010000000000000600000093
:10F3000014F8000806000000B4F70008010100002E
:10F31000000000000400000074F700080600000070
:10F3200014F700080800000094F600080800000028
:10F3300014F600080800000094F500080101000020
:10F3400000000000000100000000000000010000BB
:10F35000000000000400000054F500080600000052
:10F36000F4F40008000100000000000002010000A9
:10F37000D4F40008010100000000000000000000BB
:10F3800000000000020000008025000000C2010013
:10F3900000000000100000008025000000C20100F5
:10F3A00001000000200000008025000000C20100D4
:10F3B00000000000010000008025000000C20100E4
:10F3C00000000000080000008025000000C20100CD
:10F3D000000300000400000080250000004B000036
:10F3E00000000000BAF40008A0F4000886F4000849
:10F3F0006CF4000811190008CD180008A9180008BD
:10F40000811800087118000879270008FD18000805
:10F4100019180008F1180008E3180008000000009F
:10F4200000C20100180901083B09010801000000A1
:10F4300000E1000050090108720901080200000003
:10F440000096000086090108A809010803000000D1
:10F45000004B0000BC090108DE090108040000009F
:10F4600080250000F60F0108F60F010800010603D1
:10F470000703080409040A040B040104020403043A
:10F4800004040504FFFF0002010202020302040259
:10F49000050206030703080409040A040B04FFFF1E
:10F4A000000106030703080309030A030B03010312
:10F4B0000203030304030503FFFF0002010202022B
:10F4C00003020402050206030703080309030A03F3
:10F4D0000B03FFFF0000803F000000000000000061
:10F4E000000080BF0000803F00000000000000001E
:10F4F0000000803F0000803F000080BF0000803F90
:10F50000000080BF0000803F000080BF000080BF7F
:10F510000000803F0000803F0000803F0000803FEF
:10F520000000803F0000803F0000803F000080BF5F
:10F53000000080BF0000803F0000000000000000CD
:10F54000000000000000803F0000000000000000FC
:10F55000000000000000803F000000000000803F2D
:10F560000000803F0000803F000080BF000080BF9F
:10F57000000000000000803F000000000000803F0D
:10F58000000080BF0000803F0000803F000080BF7F
:10F59000000000800000803F0000803F000000BFAE
:10F5A0000000803F0000803F000000BF000080BFDF
:10F5B0000000803F0000803F000080BF0000003F4F
:10F5C0000000803F0000803F0000003F0000803FBF
:10F5D0000000803F0000803F0000003F000080BF2F
:10F5E000000080BF0000803F000080BF000000BF1F
:10F5F000000080BF0000803F000000BF0000803F8F
:10F60000000080BF0000803F0000803F0000003FFE
:10F61000000080BF0000803FF704353FF70435BF8E
:10F620000000803F0000803FF70435BFF70435BF7E
:10F630000000803F0000803FF70435BFF704353FEE
:10F640000000803F0000803FF704353FF704353F5E
:10F650000000803F0000803F00000000000080BFED
:10F66000000080BF0000803F000080BF000000005D
:10F67000000080BF0000803F000000000000803FCD
:10F68000000080BF0000803F0000803F00000000BD
:10F69000000080BF0000803F000080BF0000803F6E
:10F6A000000080BF0000803F000080BF000080BFDE
:10F6B0000000803F0000803F0000803F0000803F4E
:10F6C0000000803F0000803F0000803F000080BFBE
:10F6D000000080BF0000803F000080BF0000803F2E
:10F6E0000000803F0000803F000080BF000080BF1E
:10F6F000000080BF0000803F0000803F0000803F8E
:10F70000000080BF0000803F0000803F000080BFFD
:10F710000000803F0000803F000000BFD0B35D3F8D
:10F720000000803F0000803F000000BFD0B35DBFFD
:10F730000000803F0000803F0000003FD0B35D3FED
:10F74000000080BF0000803F0000003FD0B35DBFDD
:10F75000000080BF0000803F000080BF000000006C
:10F76000000080BF0000803F0000803F00000000DC
:10F770000000803F0000803F000000000000803F4C
:10F78000000080BF0000803F000080BF000080BFFD
:10F79000000000000000803F000000000000803FEB
:10F7A0000000803F0000803F0000803F000080BFDD
:10F7B000000000000000803FD0B35DBF0000003FAC
:10F7C0000000803F0000803FD0B35DBF000000BF5D
:10F7D000000080BF0000803FD0B35D3F0000003FCD
:10F7E0000000803F0000803FD0B35D3F000000BFBD
:10F7F000000080BF0000803F00000000000080BFCC
:10F800000000803F0000803F000000000000803FBB
:10F81000000080BF0000803F00000000A8AAAA3FAF
:10F820000000803F0000803F000080BFB0AA2ABFD8
:10F83000000080BF0000803F0000803FB0AA2ABFC8
:10F84000000080BF0000803F00000000A8AAAA3F7F
:10F85000000080BF0000803F000080BFB0AA2ABF28
:10F860000000803F0000803F0000803FB0AA2ABF18
:10F870000000803F0000803F0000803F000000004B
:10F88000000000000000803F000080BF000000007A
:10F89000000000000000803F000080BF0000803FAB
:10F8A000000080BF0000803F000080BF000080BFDC
:10F8B0000000803F0000803F0000803F0000803F4C
:10F8C0000000803F0000803F0000803F000080BFBC
:10F8D000000080BF0000803F000000000000803F6B
:10F8E000000080BF0000803F000080BF00000000DB
:10F8F0000000803F0000803F0000803F00000000CB
:10F900000000803F0000803F00000000000080BF3A
:10F91000000080BF0000803F00000000A8AAAA3FAE
:10F92000000000000000803F000080BFB0AA2ABF96
:10F93000000000000000803F0000803FB0AA2ABF06
:10F9400000000000000000008025000000C201004F
:10F9500002000000020000008025000000C201003B
:10F9600003000000002C01400000004000040040A3
:10F9700000080040B56206010300F00500FF19B55C
:10F980006206010300F00300FD15B56206010300E5
:10F99000F00100FB11B56206010300F00000FA0F50
:10F9A000B56206010300F00200FC13B56206010314
:10F9B00000F00400FE17B562060103000102010E0B
:10F9C00047B562060103000103010F49B562060154
:10F9D0000300010601124FB5620601030001120186
:10F9E0001E67B56206080600C80001000100DE6A55
:10F9F00000B562061608000307030000000000318E
:10FA0000E501B5620616080003070300510800006F
:10FA10008A4102B562061608000307030004E004E9
:10FA200000199D03B56206160800030703000002D3
:10FA3000020035EF04B562061608000307030080D4
:10FA4000010000B2E8000000524F4C4C3B504954BA
:10FA500043483B5941573B414C543B506F733B50DB
:10FA60006F73523B4E6176523B4C4556454C3B4D75
:10FA700041473B56454C3B0000000000170A010877
:10FA800000000000010000001C0A01080100000045
:10FA900002000000230A0108020000000300000029
:10FAA0002C0A01080300000004000000320A0108CB
:10FAB0000500000005000000370A010806000000EC
:10FAC00006000000410A01080700000007000000CE
:10FAD0004A0A01080800000008000000530A010853
:10FAE00009000000090000005C0A01080A0000008B
:10FAF0000A000000660A01080B0000000B0000006D
:10FB0000700A01080C0000000C0000007A0A0108CD
:10FB10000D0000000D000000820A01080E00000028
:10FB20000E0000008A0A01080F0000000F0000000C
:10FB3000920A010810000000100000009B0A010852
:10FB40001100000011000000A20A010812000000CC
:10FB500012000000AC0A01081300000013000000AE
:10FB6000B40A01081400000014000000BF0A0108D4
:10FB7000150000001500000000000000FF0000005C
:10FB80000000040008000C00A50B0108AA0B0108E6
:10FB9000AE0B0108C10B0108B30B0108B90B01083A
:10FBA000BD0B010800000000F60F0108690B0108F9
:10FBB000710B0108790B0108810B0108880B010802
:10FBC000930B01089B0B0108A00B0108000000002B
:10FBD00000540040000C0140400080001F20000045
:10FBE0000000200000580040000C01400004000804
:10FBF00021220000000040009001C800C800C80099
:10FC0000C800C800C800C800C80064000000C800E0
:10FC1000C800C800C8003200400080000001000297
:10FC2000000449574641540102040810204E455330
:10FC30005755442C3A3A000000011E1E6464646467
:10FC40006464220046022100820120004302100069
:10FC50000101000049020100880102004C0212006B
:10FC6000840111009001110090011100A001110008
:10FC7000A001000081920008591900082719000806
:10FC8000659F000875190008619F00083C10010875
:10FC900040100108D1580008671001086C100108D5
:10FCA000055F000880100108861001085D990008B2
:10FCB0000D10010897100108C1740008B410010864
:10FCC000B9100108DD870008E8100108F60F0108E7
:10FCD000ED680008ED100108F51001083962000810
:10FCE000091101080D110108215D0008201101080A
:10FCF0002F110108497A000849110108F60F01087F
:10FD0000995B00084E11010852110108655900085D
:10FD10006111010865110108956100087A10010858
:10FD200081110108C55B0008941101089A110108AE
:10FD300039630008B5110108BD1101089187000859
:10FD4000CC110108D1110108D56800088A0D0108FD
:10FD5000E1110108815D00080F120108031201087A
:10FD6000195000083E170108F60F0108B95800089D
:10FD70009B1301089F130108A5130108AB13010889
:10FD8000AE130108B5130108B8130108BD1301082B
:10FD9000C9130108CC130108D2130108D9130108B3
:10FDA000E3130108ED130108F61301080414010818
:10FDB00010140108171401081D1401082A14010861
:10FDC0003514010842140108000000000013010866
:10FDD000071301080C1301081D130108271301085C
:10FDE000321301083D130108B90B0108481301083B
:10FDF000B30B0108511301085B1301085F0F0108E1
:10FE00006913010879130108801301088913010897
:10FE1000931301080000000095140108440000003D
:10FE20001817002000000000282300009E1401087D
:10FE3000410000001A17002000000000010000002F
:10FE4000AC1401084400000024180020B004000095
:10FE5000A4060000B3140108440000002618002086
:10FE600000000000D0070000BD140108440000009D
:10FE70002818002000000000D0070000C714010867
:10FE8000420000002A1800200000000012000000BC
:10FE9000D4140108420000002C18002000000000CB
:10FEA00001000000E914010844000000DC170020F4
:10FEB00000000000D0070000F61401084400000014
:10FEC000DE17002000000000D00700000315010825
:10FED00044000000E017002000000000D0070000F0
:10FEE0000F15010844000000E21700200000000088
:10FEF000D00700001F15010844000000E41700208F
:10FF000000000000D0070000301501084400000088
:10FF1000E617002000000000D00700003B15010894
:10FF200044000000E817002000000000D007000097
:10FF30005015010844000000EA17002032000000BC
:10FF4000007D00005F15010844000000EC17002050
:10FF500032000000F20100006E15010841000000AF
:10FF60002D18002000000000010000007B15010892
:10FF7000410000002E1800200000000001000000D9
:10FF80008E150108410000002F180020000000001D
:10FF9000B40000009A15010841000000301800204C
:10FFA0000000000064000000A615010842000000E7
:10FFB00031180020FFFFFFFF01000000BC15010801
:10FFC000410000003418002000000000080000007C
:10FFD000D315010841000000351800200000000082
:10FFE00008000000EA150108410000004818002040
:10FFF000300000007E000000FB15010850000000EA
:020000040801F1
:1000000038180020B004000000C2010008160108E2
:10001000500000003C180020B004000000C20100A5
:1000200015160108500000004018002000000000D4
:1000300000C20100221601085000000044180020F0
:10004000B004000000C201003B160108410000009E
:1000500032180020000000000100000048160108CE
:1000600041000000331800200000000004000000E0
:100070005616010881000000181900200000000039
:10008000C80000006016010881000000221900204D
:1000900000000000C80000006A160108810000008E
:1000A0002C19002000000000C80000007416010890
:1000B000810000001919002000000000C8000000A5
:1000C0007F160108810000002319002000000000B5
:1000D000C80000008A160108810000002D190020C8
:1000E00000000000C8000000951601088100000013
:1000F0001A19002000000000C80000009F16010827
:10010000810000002419002000000000C800000049
:10011000A9160108810000002E190020000000002F
:10012000C8000000B316010884000000381A00203F
:1001300000000000D0070000C11601088100000087
:100140003C1A00200000000001000000D616010843
:10015000840000003E1A00200A000000D0070000C2
:10016000E416010884000000401A00200A00000084
:10017000D0070000F2160108810000003B1A0020A1
:1001800000000000640000000017010841000000AA
:1001900022180020000000000300000012170108D0
:1001A000410000004C180020000000000200000088
:1001B00025170108410000004D1800200000000034
:1001C0000100000036170108410000004E18002011
:1001D0000000000001000000461701084100000077
:1001E000101800200A000000C80000005117010884
:1001F00041000000111800200A0000003200000039
:100200006717010841000000121800200A000000D2
:10021000320000007D17010844000000141800207F
:1002200001000000102700009117010844000000A1
:10023000161800200000000072060000A617010832
:10024000410000001818002000000000010000001C
:10025000C417010841000000EE1700200000000054
:1002600008000000CF17010841000000EF17002030
:100270000000000008000000D9170108410000003C
:10028000F01700200000000008000000E31701083C
:1002900048000000F21700204CFFFFFF680100003B
:1002A000F417010848000000F41700204CFFFFFF7E
:1002B000680100000618010848000000F617002039
:1002C0004CFFFFFF68010000161801084400000001
:1002D0000218002064000000840300002C180108AC
:1002E00044000000FA170020000000000001000098
:1002F000351801084100000000180020000000002F
:10030000800000004518010844000000FC17002090
:1003100064000000E80300005618010844000000D3
:10032000FE17002064000000E803000068180108C0
:1003300081000000E619002001000000FA00000022
:100340007A18010881000000E71900200000000071
:10035000010000008F18010881000000EA19002048
:100360000000000096000000A918010884000000A9
:10037000E819002001000000840300007118010842
:1003800081000000E41900200000000020000000AF
:10039000C318010881000000E519002000000000DA
:1003A00064000000D018010842000000F817002087
:1003B000FFFFFFFF01000000E618010882000000B7
:1003C000341A0020FFFFFFFF01000000F4180108AD
:1003D00082000000351A002000000000010000002B
:1003E00006190108810000006019002000000000CB
:1003F000FA0000000E1901088100000061190020B8
:1004000000000000640000001619010881000000CF
:100410006219002000000000640000001E1901089D
:10042000810000006319002000000000640000004B
:100430002719010881000000641900200000000055
:1004400064000000371901088100000065190020D0
:100450000000000064000000401901088100000055
:10046000661900200000000064000000491901081E
:100470008400000068190020E8030000D007000095
:1004800058190108810000002C1A0020000000000B
:10049000C800000067190108810000002D1A002023
:1004A00000000000C80000007A1901088400000064
:1004B0002E1A0020E8030000D00700008C19010864
:1004C00084000000301A002064000000D007000003
:1004D0009E19010884000000321A00206400000008
:1004E000B80B0000B019010881000000361A002086
:1004F00000000000FF000000BD19010841000000DD
:10050000F91700200000000005000000CA190108CA
:10051000810000007019002000000000FA000000B7
:10052000D91901088100000078190020000000009E
:1005300064000000E819010881000000791900201A
:100540000000000064000000F6190108A00000008F
:10055000741900200100000014000000061A0108B0
:10056000810000008C190020000000000100000044
:10057000151A0108880000006E190020D4FEFFFF44
:100580002C010000241A0108880000006C190020CA
:10059000D4FEFFFF2C010000321A01088100000088
:1005A0007C1900200000000030000000401A010803
:1005B000A0000000801900200000000001000000E1
:1005C0004F1A0108A000000084190020000000005C
:1005D000010000005B1A0108A0000000881900203B
:1005E0000000000001000000671A010888000000F8
:1005F0006A190020B0B9FFFF50460000771A0108C1
:10060000810000001019002000000000020000001E
:10061000861A010881000000151900200000000062
:10062000C80000008E1A0108810000001F19002078
:1006300000000000C8000000FE1701088100000053
:100640002919002000000000C8000000961A0108C7
:10065000810000001419002000000000C800000004
:100660009D1A0108810000001E19002000000000F2
:10067000C8000000ED1701088100000028190020C3
:1006800000000000C8000000A41A0108810000005A
:100690001619002000000000C8000000AA1A010876
:1006A000810000002019002000000000C8000000A8
:1006B00010180108810000002A1900200000000025
:1006C000C8000000B01A0108A0000000381900207E
:1006D0000000000064000000B91A0108A00000003A
:1006E000441900200000000064000000C21A010844
:1006F000A00000005019002000000000640000006D
:10070000CB1A0108A00000003419002000000000EE
:1007100064000000D31A0108A00000004019002066
:100720000000000064000000DB1A0108A0000000C7
:100730004C1900200000000064000000E31A0108CA
:10074000A00000003C190020000000006400000030
:10075000EA1A0108A000000048190020000000006B
:1007600064000000F11A0108A000000054190020E4
:100770000000000064000000F81A0108A00000005A
:100780005C190020000000000A000000061B0108A0
:10079000A000000058190020000000000A0000001E
:1007A000121B010881000000171900200000000042
:1007B000C8000000181B010881000000211900205A
:1007C00000000000C80000001E1B0108810000009E
:1007D0002B19002000000000C8000000241B0108A5
:1007E000810000001B19002000000000C80000006C
:1007F0002C1B0108810000002519002000000000CA
:10080000C8000000341B0108810000002F190020DF
:1008100000000000C80000003C1B0108810000002F
:100820001D19002000000000C8000000421B010844
:10083000810000002719002000000000C80000000F
:10084000481B010881000000311900200000000051
:10085000C80000000000000000080040000C01403B
:1008600040000000001E002800040040000C014071
:1008700020000000041D002800040040000C01407E
:1008800001000000081D002800040040000C014089
:10089000020000000C1D002800000040000801407C
:1008A00001000000001C002800000040000801407A
:1008B00002000000041C002800080040000C014059
:1008C000000200000C1E011800080040000C01404E
:1008D00000010000081E011800080040000C014043
:1008E00080000000041E0118002C01400008014097
:1008F00000010000001B011800040040000C014032
:1009000010000000001D0118000000400008014018
:1009100004000000081C011824505542582C3431A2
:100920002C312C303030332C303030312C313135CB
:100930003230302C302A31450D0A0024504D544BB2
:100940003235312C3131353230302A31460D0A0002
:1009500024505542582C34312C312C303030332C2B
:10096000303030312C35373630302C302A32440D8F
:100970000A0024504D544B3235312C353736303047
:100980002A32430D0A0024505542582C34312C3160
:100990002C303030332C303030312C333834303050
:1009A0002C302A32360D0A0024504D544B3235314A
:1009B0002C33383430302A32370D0A002450554257
:1009C000582C34312C312C303030332C3030303105
:1009D0002C31393230302C302A32330D0A00245079
:1009E0004D544B3235312C31393230302A32320DC0
:1009F0000A003031323334353637383941424344D6
:100A000045464748494A4B4C4D4E4F50515253541E
:100A100055565758595A0041524D3B00414E474C8C
:100A2000453B00484F52495A4F4E3B004241524FBE
:100A30003B004D41473B0048454144465245453BFC
:100A4000004845414441444A3B0043414D535441D1
:100A5000423B0043414D545249473B0047505320CD
:100A6000484F4D453B0047505320484F4C443B00B6
:100A700050415353544852553B004245455045520E
:100A80003B004C45444D41583B004C45444C4F576E
:100A90003B004C4C49474854533B0043414C49426E
:100AA0003B00474F5645524E4F523B004F53442058
:100AB00053573B0054454C454D455452593B00411A
:100AC00055544F54554E453B0053797374656D2012
:100AD000557074696D653A202564207365636F6E87
:100AE00064732C20566F6C746167653A202564200E
:100AF0002A20302E315620282564532062617474D8
:100B0000657279290D0A004350552025644D487AB5
:100B10002C2064657465637465642073656E736FFF
:100B200072733A20002573200041434348573A200E
:100B30002573002E2563004379636C652054696D2D
:100B4000653A2025642C20493243204572726F7229
:100B5000733A2025642C20636F6E66696720736981
:100B60007A653A2025640D0A004144584C333435E7
:100B7000004D505536303530004D4D4138343578C4
:100B800000424D41323830004C534D333033444CE9
:100B90004843004D5055363030300046414B4500FB
:100BA0004E6F6E65004759524F004143430042412A
:100BB000524F00534F4E415200475053004750533D
:100BC0002B4D414700436C65616E666C69676874C4
:100BD0002F25735365702032322032303134202F6C
:100BE0002031393A30323A303520282573290064D3
:100BF0003566356664620061757820257520257537
:100C00000D0A00496E76616C6964204665617475F1
:100C1000726520696E6465783A206D757374206220
:100C200065203C2025750D0A0025752C25753A2573
:100C3000733A2573006C65642025752025730D0AB1
:100C4000005061727365206572726F720D0A0049FF
:100C50006E76616C6964206C656420696E64657889
:100C60003A206D757374206265203C2025750D0A4D
:100C700000417661696C61626C6520636F6D6D61C6
:100C80006E64733A0D0A0025730925730D0A00433B
:100C9000757272656E74206D697865723A2025737D
:100CA0000D0A00417661696C61626C65206D69783E
:100CB0006572733A2000496E76616C6964206D69D3
:100CC00078657220747970650D0A004D69786572D7
:100CD0002073657420746F2025730D0A002025642D
:100CE00020256400556E6B6E6F776E207661726999
:100CF00061626C65206E616D650D0A0043757272EC
:100D0000656E742073657474696E67733A200D0A9A
:100D10000025732073657420746F200056616C7514
:100D2000652061737369676E6D656E74206F75748D
:100D3000206F662072616E67650D0A004E470900DC
:100D40004F4B0900437573746F6D206D6978657240
:100D50003A200D0A4D6F746F720954687209526F10
:100D60006C6C095069746368095961770D0A002336
:100D700025643A09002573090053616E697479206E
:100D8000636865636B3A09007265736574006C6F24
:100D90006164004C6F61646564202573206D69781F
:100DA0000D0A0057726F6E67206E756D6265722056
:100DB0006F6620617267756D656E74732C206E6549
:100DC000656473206964782074687220726F6C6C3B
:100DD000207069746368207961770D0A004D6F7423
:100DE0006F72206E756D626572206D75737420620E
:100DF00065206265747765656E203120616E6420C0
:100E000025640D0A004D75737420626520616E794A
:100E1000206F72646572206F6620414554523132F2
:100E200033340D0A0043757272656E7420617373FA
:100E300069676E6D656E743A2000456E61626C651F
:100E4000642066656174757265733A20004176614D
:100E5000696C61626C652066656174757265733A70
:100E60002000496E76616C696420666561747572F4
:100E700065206E616D650D0A00534F4E415220751D
:100E80006E617661696C61626C650D0A004469731C
:100E900061626C65642000456E61626C656420006F
:100EA00055736167653A0D0A6D6F746F7220696ED4
:100EB000646578205B76616C75655D202D207368B4
:100EC0006F77205B6F72207365745D206D6F746F38
:100ED000722076616C75650D0A004E6F2073756324
:100EE00068206D6F746F722C207573652061206EA1
:100EF000756D626572205B302C2025645D0D0A00E3
:100F00004D6F746F7220256420697320736574209F
:100F100061742025640D0A00496E76616C69642055
:100F20006D6F746F722076616C75652C2031303076
:100F3000302E2E323030300D0A0053657474696ED5
:100F400067206D6F746F7220256420746F20256494
:100F50000D0A00736574202573203D200043433340
:100F600044000D0A5265626F6F74696E67005361C9
:100F700076696E67000D0A4C656176696E6720437D
:100F80004C49206D6F64650D0A000D0A456E74654D
:100F900072696E6720434C49204D6F64652C207444
:100FA0007970652027657869742720746F207265D1
:100FB0007475726E2C206F72202768656C70270D17
:100FC0000A000D0A2320000D1B5B4B001B5B324AFD
:100FD0001B5B313B314800556E6B6E6F776E206343
:100FE0006F6D6D616E642C20747279202768656C5A
:100FF0007027000820080041455452313233340034
:10100000526573657474696E6720746F20646566D9
:1010100061756C7473004572726F723A20456E612F
:10102000626C6520616E6420706C756720696E204B
:101030004750532066697273740D0A006175780019
:10104000666561747572655F6E616D652061757846
:10105000666C6167206F7220626C616E6B20666FD8
:1010600072206C69737400636D69780064657369DC
:10107000676E20637573746F6D206D69786572009B
:10108000636F6C6F7200636F6E666967757265205F
:10109000636F6C6F727300726573657420746F2078
:1010A00064656661756C747320616E64207265623C
:1010B0006F6F740064756D70007072696E74206378
:1010C0006F6E666967757261626C652073657474B2
:1010D000696E677320696E2061207061737461624C
:1010E0006C6520666F726D00657869740066656175
:1010F00074757265006C697374206F72202D76614F
:101100006C206F722076616C00676574006765748F
:10111000207661726961626C652076616C7565002C
:10112000677073706173737468726F75676800704D
:101130006173737468726F75676820677073207469
:101140006F2073657269616C0068656C70006C6516
:101150006400636F6E666967757265206C656473A1
:10116000006D6170006D617070696E67206F662040
:101170007263206368616E6E656C206F7264657265
:10118000006D69786572206E616D65206F72206CEC
:10119000697374006D6F746F72006765742F736587
:1011A00074206D6F746F72206F7574707574207613
:1011B000616C75650070726F66696C6500696E645C
:1011C000657820283020746F20322900736176659D
:1011D000007361766520616E64207265626F6F7462
:1011E000006E616D653D76616C7565206F72206281
:1011F0006C616E6B206F72202A20666F72206C69A2
:1012000073740073686F772073797374656D2073DE
:1012100074617475730070726F66696C6520256403
:101220000D0A006D6173746572000D0A23207665E6
:101230007273696F6E0D0A000D0A232064756D705C
:10124000206D61737465720D0A000D0A23206D69AB
:101250007865720D0A006D697865722025730D0A34
:1012600000636D697820256400636D6978202564CA
:1012700020302030203020300D0A000D0A0D0A23C6
:1012800020666561747572650D0A00666561747526
:101290007265202D25730D0A00666561747572658F
:1012A0002025730D0A000D0A0D0A23206D61700DB3
:1012B0000A006D61702025730D0A000D0A0D0A23C6
:1012C000206C65640D0A000D0A0D0A2320636F6C03
:1012D0006F720D0A000D0A232064756D7020707204
:1012E0006F66696C650D0A000D0A232070726F66C7
:1012F000696C650D0A000D0A23206175780D0A00DE
:1013000052585F50504D005642415400494E464C91
:10131000494748545F4143435F43414C0052585F43
:1013200053455249414C004D4F544F525F53544F17
:101330005000534552564F5F54494C5400534F464A
:101340005453455249414C004641494C534146454E
:101350000054454C454D4554525900435552524551
:101360004E545F4D455445520052585F50415241D2
:101370004C4C454C5F50574D0052585F4D535000F8
:10138000525353495F414443004C45445F535452C8
:10139000495000444953504C41590054524900515E
:1013A0005541445000515541445800424900474975
:1013B0004D42414C005936004845583600464C597C
:1013C000494E475F57494E47005934004845583603
:1013D00058004F43544F5838004F43544F464C41E8
:1013E0005450004F43544F464C41545800414952C9
:1013F000504C414E450048454C495F3132305F43C7
:1014000043504D0048454C495F39305F44454700E3
:10141000565441494C340048455836480050504DC8
:101420005F544F5F534552564F004455414C434F14
:10143000505445520053494E474C45434F50544534
:101440005200435553544F4D0041455254313233AD
:101450003400002710080423022001636F6C6F72B0
:101460002025752025642C25752C25750D0A00492D
:101470006E76616C696420636F6C6F7220696E6454
:1014800065783A206D757374206265203C2025755F
:101490000D0A002E006C6F6F7074696D6500656DCC
:1014A000665F61766F6964616E6365006D69645F34
:1014B0007263006D696E5F636865636B006D617870
:1014C0005F636865636B00727373695F6368616E05
:1014D0006E656C00696E7075745F66696C746572B8
:1014E000696E675F6D6F6465006D696E5F746872C9
:1014F0006F74746C65006D61785F7468726F74747A
:101500006C65006D696E5F636F6D6D616E64003355
:10151000645F6465616462616E645F6C6F77003301
:10152000645F6465616462616E645F6869676800D6
:1015300033645F6E65757472616C0033645F6465FB
:10154000616462616E645F7468726F74746C65006C
:101550006D6F746F725F70776D5F72617465007329
:101560006572766F5F70776D5F726174650072652A
:101570007461726465645F61726D00646973617245
:101580006D5F6B696C6C5F73776974636800736D12
:10159000616C6C5F616E676C6500666C6170735F37
:1015A000737065656400666978656477696E675F06
:1015B000616C74686F6C645F6469720073657269F2
:1015C000616C5F706F72745F315F7363656E6172BF
:1015D000696F0073657269616C5F706F72745F32FE
:1015E0005F7363656E6172696F007265626F6F74BD
:1015F0005F636861726163746572006D73705F62CE
:101600006175647261746500636C695F62617564C1
:1016100072617465006770735F6261756472617492
:1016200065006770735F706173737468726F75675C
:10163000685F6261756472617465006770735F7082
:10164000726F7669646572006770735F736261734D
:101650005F6D6F6465006770735F706F735F7000BC
:101660006770735F706F735F69006770735F706F2F
:10167000735F64006770735F706F73725F70006791
:1016800070735F706F73725F69006770735F706F04
:1016900073725F64006770735F6E61765F7000677E
:1016A00070735F6E61765F69006770735F6E6176FD
:1016B0005F64006770735F77705F726164697573F0
:1016C000006E61765F636F6E74726F6C735F6865D6
:1016D0006164696E67006E61765F73706565645FF3
:1016E0006D696E006E61765F73706565645F6D61D4
:1016F00078006E61765F736C65775F726174650008
:1017000073657269616C72785F70726F7669646517
:10171000720074656C656D657472795F70726F7656
:10172000696465720074656C656D657472795F7368
:101730007769746368006672736B795F696E76654A
:101740007273696F6E00766261745F7363616C655A
:1017500000766261745F6D61785F63656C6C5F7663
:101760006F6C7461676500766261745F6D696E5F4E
:1017700063656C6C5F766F6C74616765006375722E
:1017800072656E745F6D657465725F7363616C65BD
:101790000063757272656E745F6D657465725F6FFC
:1017A0006666736574006D756C74697769695F63EB
:1017B000757272656E745F6D657465725F6F757456
:1017C00070757400616C69676E5F6779726F006134
:1017D0006C69676E5F61636300616C69676E5F6D02
:1017E000616700616C69676E5F626F6172645F72EE
:1017F0006F6C6C00616C69676E5F626F6172645FD1
:10180000706974636800616C69676E5F626F6172B2
:10181000645F796177006D61785F616E676C655FA9
:10182000696E636C696E6174696F6E006779726F5F
:101830005F6C7066006D6F726F6E5F746872657357
:10184000686F6C64006779726F5F636D70665F6666
:101850006163746F72006779726F5F636D70666D3C
:101860005F666163746F7200616C745F686F6C6453
:101870005F6465616462616E6400616C745F686F6F
:101880006C645F666173745F6368616E6765007442
:1018900068726F74746C655F636F7272656374698C
:1018A0006F6E5F76616C7565007468726F74746CCE
:1018B000655F636F7272656374696F6E5F616E6797
:1018C0006C65007961775F6465616462616E640074
:1018D0007961775F636F6E74726F6C5F6469726554
:1018E0006374696F6E007961775F646972656374B0
:1018F000696F6E007472695F756E61726D65645FA9
:10190000736572766F0072635F72617465007263F3
:101910005F6578706F007468725F6D6964007468E9
:10192000725F6578706F00726F6C6C5F7069746362
:10193000685F72617465007961775F7261746500D8
:101940007470615F72617465007470615F6272656A
:10195000616B706F696E74006661696C7361666556
:101960005F64656C6179006661696C736166655F6F
:101970006F66665F64656C6179006661696C73614E
:1019800066655F7468726F74746C65006661696C1B
:10199000736166655F6D696E5F757365630066612F
:1019A000696C736166655F6D61785F75736563000F
:1019B00067696D62616C5F666C6167730061636328
:1019C0005F6861726477617265006163635F6C7008
:1019D000665F666163746F720061636378795F64E8
:1019E00065616462616E64006163637A5F6465610E
:1019F0006462616E64006163637A5F6C70665F63EA
:101A000075746F6666006163635F756E61726D65A4
:101A10006463616C006163635F7472696D5F7069B8
:101A2000746368006163635F7472696D5F726F6C89
:101A30006C006261726F5F7461625F73697A6500E6
:101A40006261726F5F6E6F6973655F6C7066006272
:101A500061726F5F63665F76656C006261726F5F73
:101A600063665F616C74006D61675F6465636C6978
:101A70006E6174696F6E007069645F636F6E74721B
:101A80006F6C6C657200705F706974636800695F89
:101A9000706974636800705F726F6C6C00695F726C
:101AA0006F6C6C00705F79617700695F79617700B6
:101AB000705F70697463686600695F7069746368F9
:101AC0006600645F70697463686600705F726F6C53
:101AD0006C6600695F726F6C6C6600645F726F6C3D
:101AE0006C6600705F7961776600695F796177661F
:101AF00000645F79617766006C6576656C5F686F1E
:101B000072697A6F6E006C6576656C5F616E676C8A
:101B10006500705F616C7400695F616C7400645F84
:101B2000616C7400705F6C6576656C00695F6C65F4
:101B300076656C00645F6C6576656C00705F7665D9
:101B40006C00695F76656C00645F76656C000020F0
:101B5000202020202020202028282828282020205D
:101B6000202020202020202020202020202020880D
:101B70001010101010101010101010101010100471
:101B800004040404040404040410101010101010C1
:101B900041414141414101010101010101010101B5
:101BA00001010101010101010101101010101010CB
:101BB0004242424242420202020202020202020285
:101BC00002020202020202020202101010102000A1
:101BD0000000000000000000000000000000000005
:101BE00000000000000000000000000000000000F5
:101BF00000000000000000000000000000000000E5
